:020000040800F2
:10000000D0120020F1080008250700082707000883
:100010002B0700082F070008330700080000000026
:10002000000000000000000000000000370700088A
:1000300039070008000000003B0700083D070008E2
:100040000B0900080B0900080B0900080B09000840
:100050000B0900080B0900080B0900080B09000830
:100060000B0900080B0900080B0900080B09000820
:100070000B0900080B0900080B0900080B09000810
:100080000B0900080B0900080B0900080B09000800
:100090000B0900080B0900080B0900080B090008F0
:1000A0000B0900080B0900080B0900080B090008E0
:1000B0000B0900080B0900080B0900080B090008D0
:1000C0000B0900080B0900080B0900080B090008C0
:1000D0000B0900080B0900080B0900081B2D00087C
:1000E0000B0900080B0900080B0900080B090008A0
:1000F0000B0900080B0900080B0900080B09000890
:100100000B0900080B0900080B0900080B0900087F
:100110000B0900080B0900080B0900080B0900086F
:100120000B0900080B0900080B090008230500084B
:10013000DFF80CD002F016FF004800476501000808
:10014000D0120020EFF30980704780F309887047D0
:10015000EFF30880704780F30888704740BA704713
:10016000C0BA70471CB500241EA103C9CDE9000127
:100170004FF000601D49086000F03CF802F00CFEF2
:1001800002F0C6FE4FF4E13000F0FEF802F02CFB66
:1001900001201749086002F027FB21E002F095FDDD
:1001A000012803D102F020FB012406E002F0BCFC90
:1001B000012801D1022400E0002402F015FB012CEB
:1001C00006D102F011FB02F068FD02F00DFB07E022
:1001D000022C05D102F008FB02F032FD02F004FB14
:1001E000DCE700000301050A035C370008ED00E0CE
:1001F0008481224210B5042000F0DCFB2E48006808
:1002000000EB400080002D49B0FBF1F02C49087054
:100210000846007800EB4001C1EBC0104FF6FF71BB
:1002200001EAC0002749088010BD0146244A12781F
:100230004A434FF0E0235A6100229A611A4612693C
:1002400042F001021A6100BF4FF0E022106910F085
:10025000010F02D010F4803FF6D04FF0E022126977
:1002600022F001024FF0E0231A6100229A617047E8
:100270000146144A12884A434FF0E0235A61002293
:100280009A611A46126942F001021A6100BF4FF0EA
:10029000E022106910F0010F02D010F4803FF6D078
:1002A0004FF0E022126922F001024FF0E0231A61C0
:1002B00000229A617047000004000020001BB70074
:1002C000000000200200002010B590B0044601217B
:1002D000880300F0A3FE0121084600F092FE0C9472
:1002E0000020ADF83400ADF83600ADF83800ADF8B8
:1002F0003C000C20ADF83A000CA9204801F0C3F8EE
:1003000001211E4801F04BF91D4801F07DFA1B4800
:10031000001D01901B48029000200390642004906F
:100320000020059080200690002007900890202053
:10033000099000020A9000200B9001A9104801F0DA
:1003400005FB012240210D4801F05AF901210C481A
:1003500001F027FB10B010BD10B5044600BF4021CE
:10036000064801F0F7F90028F9D04021034801F0D0
:10037000FEF92146014801F07FF910BD0038014027
:10038000580002404400002010B586B00446012108
:10039000682000F043FE0121880400F04CFE744800
:1003A00001F02EF8734801F02FFA0420ADF8140084
:1003B00010208DF8170003208DF8160005A96E484F
:1003C00000F076FB4FF48060ADF8140018208DF833
:1003D000170005A9694800F06BFB4FF40060ADF809
:1003E000140004208DF8170005A9644800F060FB94
:1003F00001940020ADF80800ADF80A00ADF80C003B
:10040000ADF810000C20ADF80E0001A9584801F01D
:100410003AF827208DF8000001208DF80100022015
:100420008DF8020001208DF80300684600F077FA8D
:10043000012240F225514E4801F0BDF801214C48FF
:1004400001F0ADF800204E49086006B010BD30B58F
:100450008DB005460C464748143801F0D5F944489C
:10046000001D029003951020049005940020069032
:10047000802007900020089009900A904FF40050C7
:100480000B9000200C9002A93A48143801F05EFA53
:1004900001228021364801F0B3F8012202213948B7
:1004A00001F08BFA3B208DF8040002208DF8050046
:1004B00001208DF806008DF8070001A800F02FFA42
:1004C0000DB030BD70B505460E4601202C490860C0
:1004D0004FF000040CE000BF4021254801F03AF93C
:1004E0000028F9D0295D224801F0C6F8601C84B2CA
:1004F000B442F0DB00BF40211D4801F02BF9002879
:10050000F9D000201E49086070BD10B503460020D8
:1005100000BF03E00C5C1C54441CE0B29042F9DBC9
:1005200010BD10B5184801F06AFA002111481438BE
:1005300001F037FA4FF49670FFF777FE002010496C
:10054000086010BD70B5044601200D4908602046C2
:1005500002F000FDC5B229462046FFF7B3FF012097
:10056000FFF786FE00200949C1F8880170BD000030
:10057000004800403000024000180140000C0140DB
:100580008801234258040240000002100000234268
:1005900000B585B00020ADF800004FF48270ADF8D2
:1005A00002000020ADF80400ADF80600ADF8080028
:1005B0004FF40070ADF80A000020ADF80C00ADF863
:1005C0000E000720ADF810006946534800F0B8FD52
:1005D0000121514800F059FE05B000BD70B5054637
:1005E0000E46002405E0601CC4B2C82C01DD0020CA
:1005F00070BD0221284600F0CCFE0028F3D0314621
:10060000284600F073FE002405E0601CC4B2C82C2C
:1006100001DD0020ECE70121284600F0BAFE0028A9
:10062000F3D0284600F064FEC0B2E1E770B505469D
:10063000002405E0601CC4B2C82C01DD002070BDA0
:100640000221364800F0A5FE0028F3D029463348A1
:1006500000F04CFE002405E0601CC4B2C82C01DD93
:100660000020ECE701212D4800F093FE0028F3D094
:100670002A4800F03DFEC0B2E1E770B5054600240F
:1006800005E0601CC4B2C82C01DD002070BD022151
:10069000214800F07EFE0028F3D029461E4800F0D5
:1006A00025FE002405E0601CC4B2C82C01DD00203A
:1006B000ECE70121184800F06CFE0028F3D0164842
:1006C00000F016FEC0B2E1E770B50546002405E073
:1006D000601CC4B2C82C01DD002070BD022110488E
:1006E00000F057FE0028F3D029460D4800F0FEFD2B
:1006F000002405E0601CC4B2FF2C01DD0020ECE703
:100700000121074800F045FE0028F3D0044800F01E
:10071000EFFDC0B2E1E70000003C004000300140C6
:1007200000380040704700BFFEE700BFFEE700BF93
:10073000FEE700BFFEE77047704770477047000054
:100740000CB50020019000905E48006840F48030B5
:100750005C49086000BF5B48006800F4003000900E
:100760000198401C0190009818B90198B0F5A06F4D
:10077000F1D15448006810F4003F02D001200090ED
:1007800001E0002000900098012828D14E48006820
:1007900040F010004C4908600846006820F0030053
:1007A0000860084600680860464840684549486057
:1007B0000846406848600846406848600846406807
:1007C00020F0030048600846406840F0010048609F
:1007D00000BF3C48406800F00C000428F9D10CBD73
:1007E00010B5FFF7ADFF10BD10B53648006840F0FA
:1007F00001003449086008464068344908403149DE
:10080000486008460068324908402E49086008469A
:10081000006820F4802008600846406820F4FE004C
:1008200048604FF41F008860FFF7DAFF4FF0006068
:100830002849086010BD10B5002100200022214B7E
:100840005B6803F00C0121B1042906D0082928D1E6
:1008500007E0214B214C236027E0214B1F4C2360F4
:1008600023E0184B5B6803F47010164B5B6803F4CD
:100870008032022303EB904022B91A4B4343174CBA
:1008800023600DE00F4B5B6813F4003F04D0164B60
:100890004343124C236003E0114B43430F4C23604E
:1008A00003E00D4B0D4C236000BF00BF054B5B68A0
:1008B000C3F303130D4CE15C084B1B68CB40074CA2
:1008C000236010BD00100240002002400000FFF82D
:1008D000FFFFF6FE08ED00E000127A0004000020A1
:1008E000001BB70000093D00808D5B000800002060
:1008F0000648804706480047FEE7FEE7FEE7FEE7BA
:10090000FEE7FEE7FEE7FEE7FEE7FEE7E907000891
:100910003101000831490143314A1160704770B517
:10092000002100230F22C4780CB32D4C246804F45A
:10093000E064C4F5E064210AC1F10403CA404478CC
:1009400004FA03F18478144021430901254C067808
:10095000A155047804F01F050124AC4005786D1101
:100960004FF0E02606EB8505C5F8004109E0047864
:1009700004F01F050124AC401B4D0678761145F8A4
:10098000264070BD194A0A400243154B1B1F1A60CE
:10099000704739B1124A121D12680243104B1B1DD9
:1009A0001A6006E00E4A121D126882430C4B1B1D92
:1009B0001A607047042808D14FF0E021096941F01E
:1009C00004014FF0E022116107E04FF0E0210969D6
:1009D00021F004014FF0E022116170470000FA0598
:1009E0000CED00E000E400E080E100E080FFFF1F8C
:1009F00010B50446CA48844208D10121042000F001
:100A000027FB0021042000F023FB46E0C548844278
:100A100008D10121082000F01BFB0021082000F074
:100A200017FB3AE0C048844208D10121102000F0B1
:100A30000FFB0021102000F00BFB2EE0BB4884428E
:100A400008D10121202000F003FB0021202000F02C
:100A5000FFFA22E0B648844208D10121402000F08C
:100A6000F7FA0021402000F0F3FA16E0B148844282
:100A700008D10121802000F0EBFA0021802000F055
:100A8000E7FA0AE0AC48844207D10121801500F062
:100A9000DFFA0021A01500F0DBFA10BD10B501212E
:100AA000084600F0D5FA0021012000F0D1FA10BD6F
:100AB0002DE9F041024600250026002000230024F5
:100AC000002791F803C00CF00F0591F803C01CF04B
:100AD000100F03D091F802C04CEA050591F800C050
:100AE000BCF1000F31D0146800202BE04FF0010C56
:100AF0000CFA00F3B1F800C00CEA03069E4220D1C4
:100B000083004FF00F0C0CFA03F7BC4305FA03FC0B
:100B10004CEA040491F803C0BCF1280F06D14FF051
:100B2000010C0CFA00FCC2F814C00AE091F803C0F2
:100B3000BCF1480F05D14FF0010C0CFA00FCC2F8D3
:100B400010C0401C0828D1D31460B1F800C0BCF11B
:100B5000FF0F34DD546800202EE000F1080C4FF048
:100B6000010808FA0CF3B1F800C00CEA03069E4233
:100B700021D183004FF00F0C0CFA03F7BC4305FAA8
:100B800003FC4CEA040491F803C0BCF1280F05D122
:100B900000F1080C08FA0CF8C2F8148091F803C0B0
:100BA000BCF1480F07D100F1080C4FF0010808FA1A
:100BB0000CF8C2F81080401C0828CED35460BDE861
:100BC000F0814FF6FF710180022181700421C17014
:100BD00070470246002093680B4201D0012000E0DC
:100BE000002070470146886880B2704702460020A6
:100BF000D3680B4201D0012000E00020704701467D
:100C0000C86880B2704701617047416170470AB19E
:100C1000016100E041617047C16070474FF480326C
:100C20000A438261816182618269826970470246FA
:100C30000020424B18684FF68073184040EA0210BB
:100C400008433E4B186070473D49C8617047F0B596
:100C50000A46002300240021002500F00046B6F1DA
:100C6000004F02D1354EF16901E0344E7168C0F396
:100C7000034583B200F44016B6F5401F08D121F0B9
:100C800070612E4E766826F070662C4F7E6012E002
:100C900000F48016B6F5801F06D1032606FA05F487
:100CA000A14341F0706106E0460D360103FA06F6F5
:100CB000B14341F0706122B1460D360103FA06F6E8
:100CC000314300F00046B6F1004F02D11B4EF161F6
:100CD00001E01A4E7160F0BD30B500228B071C0F89
:100CE0000F2303FA04F2154B08338C1053F8243009
:100CF0009343124C08348D1044F8253023468C1051
:100D000053F824308C07240F00FA04F423430B4CCF
:100D100008348D1044F8253030BD0A49086070470A
:100D200000080140000C0140001001400014014087
:100D300000180140001C014000200140000001405B
:100D400000002042DC002042DD48006840F0010045
:100D5000DB49086008464068DA490840D8494860DD
:100D600008460068D8490840D54908600846006828
:100D700020F4802008600846406820F4FE004860A7
:100D80004FF41F0088607047CD49096821F4803115
:100D9000CB4A11601146096821F480211160B0F539
:100DA000803F03D0B0F5802F0ED106E0C44909681A
:100DB00041F48031C24A116007E0C149096841F439
:100DC000A021BF4A116000E000BF00BF704710B50E
:100DD00001460022002300204A11012A02D1B84C0A
:100DE000236806E0022A02D1B54C236A01E0B44C24
:100DF000636A01F01F02012494401C4201D00120CB
:100E000000E0002010BD38B500200090002400252F
:100E100000BF3120FFF7DBFF05460098401C009023
:100E20000098B0F5A06F01D0002DF2D03120FFF76F
:100E3000CEFF08B1012400E00024204638BD014661
:100E400000209F4A106820F0F80040EAC1001060BE
:100E500070479E490860704702460020984B5868CA
:100E600020F47C1042EA01031843954B5860704708
:100E700096490866704701460020914A506820F064
:100E800003000843506070478D48406800F00C0034
:100E90007047014600208A4A506820F0F00008435D
:100EA0005060704701460020854A506820F4E06099
:100EB00008435060704701460020814A506820F482
:100EC000605040EAC1005060704729B17C4A527AB4
:100ED00002437B4B5A7204E0794A527A8243784B40
:100EE0005A7270477A490860704701460020744A78
:100EF000506820F440400843506070470021754A14
:100F000011706F4A82F82010012802D0042808D1FD
:100F100003E001216F4A117004E005216D4A117050
:100F200000E000BF00BF70476B490860704764492C
:100F3000096A0143624A116270476749443908608F
:100F4000704730B500210022002400235C4D6D68FD
:100F500005F00C0121B1042905D0082923D105E0B1
:100F60005E4D056022E05E4D05601FE0544D6D68EA
:100F700005F47012524D6D6805F48034022505EBBE
:100F800092421CB9574D554305600BE04C4D6D68BE
:100F900015F4003F03D0544D5543056002E0504D19
:100FA0005543056002E04D4D056000BF00BF444D54
:100FB0006D6805F0F00109094C4D6B5C0568DD407A
:100FC00045603F4D6D6805F4E061090A474D6B5C73
:100FD0004568DD4085603A4D6D6805F46051C90A89
:100FE000424D6B5C4568DD40C560354D6D6805F46C
:100FF0004041890B3E4D6B5CC568B5FBF3F505615F
:1010000030BD29B12E4A526902432D4B5A6104E08A
:101010002B4A526982432A4B5A61704729B1284AA8
:1010200092690243264B9A6104E0254A9269824301
:10103000234B9A61704729B1214AD2690243204B60
:10104000DA6104E01E4AD26982431D4BDA617047BF
:1010500029B11B4AD2680243194BDA6004E0184AEE
:10106000D2688243164BDA60704729B1144A12697C
:101070000243134B1A6104E0114A12698243104B78
:101080001A61704714494039086070470F49C864B5
:1010900070470B49C87170470948406A40F080703A
:1010A00007494862704701460020054A92680A4293
:1010B00001D0012000E0002070470149887270478C
:1010C000001002400000FFF8FFFFF6FE0000424261
:1010D000D8004242201002408004424200127A00AE
:1010E000001BB70000093D00808D5B001800002048
:1010F0002800002010B50446BE48844208D10121D2
:101100008014FFF7A5FF0021A014FFF7A1FF16E050
:10111000B948844208D101210014FFF7A6FF00213D
:101120002014FFF7A2FF0AE0B448844207D101214E
:10113000C013FFF79AFF0021E013FFF796FF10BDE1
:1011400010B50022028802F441520B884C882343D8
:101150008C882343CC8823430C8923434C89234325
:101160008C892343CC8923431A430280838B4FF21B
:10117000FF74234083830B8A038210BD2DE9F04F57
:1011800085B005460C464FF0000902274FF00008D5
:101190004FF0010B0026B246A88B4FF240010840E9
:1011A000A88302202884B5F81C90A068022801D1E9
:1011B00000BF38E0A08810B94FF0010B01E04FF0FC
:1011C000020B8D48854200D100E000BF6846FFF762
:1011D000B8FEDDF800A0E088B0F5007F0AD14FEA44
:1011E0001A2000EB80004000A168B0FBF1F0401D28
:1011F00086B20BE04FEA4B10BAFBF0F000EB800038
:101200004000A168B0FBF1F0401D86B20A20B6FB99
:10121000F0F606F00108A6EB0800C0F34F074FF602
:10122000FF7000EA0828022F01DBFF2F02DD0227F2
:101230004FF00008E08840EA080038432884A0887E
:10124000A1890843618808432188084340F400606D
:1012500040EA0909A5F81C9005B0BDE8F08F00210F
:10126000018041808180C180018141818181C18172
:101270000721018270470021018041808180C18067
:101280000221816000218181704721B1028842F0F2
:101290004002028004E002884FF6BF731A400280C9
:1012A000704721B1828B42F48062828304E0828B9A
:1012B0004FF6FF331A408283704730B50024002375
:1012C0000C110125A540ABB21AB185881D4385805C
:1012D00002E085889D43858030BD1AB183880B4329
:1012E000838002E083888B438380704781817047CD
:1012F000014688897047A1F57E42FF3A04D00288F2
:1013000042F48072028004E002884FF6FF631A40C4
:101310000280704721B1828842F00402828004E09A
:1013200082884FF6FB731A408280704702884FF222
:10133000FF731A40028002880A43028070470188C6
:1013400041F480510180704721B1028842F400527B
:10135000028004E002884DF6FF731A400280704755
:1013600002460020012901D0108B00E0908A7047CE
:101370000146088A7047B1F5804F04D1028842F4D3
:101380008042028004E002884BF6FF731A4002801C
:1013900070470246002013890B4201D0012000E073
:1013A00000207047CA4302817047F0B50246002012
:1013B00000240023002501F00F070126BE40B4B22F
:1013C0000B1101269E40B3B2968806EA03051689E2
:1013D000264202D00DB1012000E00020F0BD10B582
:1013E000002201F00F040123A3409AB2D3430381EA
:1013F00010BD00000030014000380040003C0040BB
:1014000010B50446FB48844209D101218803FFF747
:101410001FFE00214FF48040FFF71AFE32E0F6482D
:10142000844209D101214804FFF71FFE00214FF437
:101430000030FFF71AFE25E0F048844209D101216F
:101440008804FFF712FE00214FF48020FFF70DFE05
:1014500018E0EB48844209D10121C804FFF705FEDA
:1014600000214FF40020FFF700FE0BE0E548844226
:1014700008D101210805FFF7F8FD00214FF4801085
:10148000FFF7F3FD10BD2DE9F04786B005460E4687
:101490000024A24600BFA1460027B08900B100BFCA
:1014A0002F462C8A4CF6FF700440F08804432C82AF
:1014B000AC894EF6F3100440B08831890843718935
:1014C00008430443AC81AC8A4FF6FF400440B08926
:1014D0000443AC8201A8FFF734FDC648874202D11D
:1014E000DDF810A001E0DDF80CA0A88910F4004F91
:1014F00008D00AEBCA0000EB0A1031684900B0FBC3
:10150000F1F807E00AEBCA0000EB0A103168890025
:10151000B0FBF1F86420B8FBF0F00401200964216D
:1015200001FB1089A88910F4004F08D0322000EB8D
:10153000C900B0FBF1F000F00700044308E03220DE
:1015400000EB09106421B0FBF1F000F00F00044340
:101550002C8106B0BDE8F0874FF4165101600021E0
:101560008180C18001810C214181002181817047EE
:1015700010B502460020108A4FF2FF0318400B8876
:101580004C8823438C882343CC8823431843108200
:1015900010BD0021018041808180C180704721B150
:1015A000828942F40052828104E082894DF6FF7301
:1015B0001A4082817047F0B50346002400260025BA
:1015C0000020A1F510676A3F00D100BF1846C1F3A3
:1015D000421401F01F06012707FA06F5012C01D17C
:1015E0000C3004E0022C01D1103000E014301AB1AC
:1015F00007682F43076002E00768AF430760F0BD4C
:101600001AB1838A0B43838202E0838A8B438382ED
:101610007047028A4FF6F0731A400282028A0A4328
:101620000282704782894FF2FF731A408281828959
:101630000A438281704721B1828942F0020282818D
:1016400004E082894FF6FD731A4082817047028A56
:101650004FF6DF731A400282028A0A430282704701
:1016600021B1028A42F48042028204E0028A4BF6EF
:10167000FF731A4002827047C1F3080282807047EC
:1016800001468888C0F308007047818941F0010154
:1016900081817047028BD2B20283028B42EA01221F
:1016A00002837047028B02F47F420283028B0A435B
:1016B0000283704721B1828A42F02002828204E0D4
:1016C000828A4FF6DF731A408282704721B1828A84
:1016D00042F01002828204E0828A4FF6EF731A40D1
:1016E0008282704721B1828A42F00802828204E03D
:1016F000828A4FF6F7731A408282704721B182893D
:1017000042F40042828103E08289C2F30E028281A8
:10171000704721B1828A42F40062828204E0828AA8
:101720004FF2FF731A4082827047828A4FF6FB7332
:101730001A408282828A0A438282704721B1828A59
:1017400042F00202828204E0828A4FF6FD731A4060
:101750008282704702460020B1F5007F00D100BFB1
:1017600013880B4201D0012000E00020704701F4F3
:101770000072B2F5007F00D100BFCA4302807047FB
:1017800070B502460024002300250020A1F5106654
:101790006A3E00D100BFC1F3421501F01F030126CC
:1017A00006FA03F3012D02D19689334006E0022D9B
:1017B00002D1168A334001E0968A33400C1201268A
:1017C00006FA04F41688344013B10CB1012000E08D
:1017D000002070BD10B500220023A1F510646A3C02
:1017E00000D100BF0A1201249440A3B2DC4304805C
:1017F00010BD000000380140004400400048004097
:10180000004C00400050004001684FF6FE7211404D
:1018100001600021016041608160C1608C498842A3
:1018200008D18B490839496841F00F01884A083AC4
:1018300051608AE086491431884208D184490839C8
:10184000496841F0F001824A083A51607DE08049E0
:101850002831884208D17E490839496841F47061CD
:101860007B4A083A516070E079493C31884208D19E
:1018700077490839496841F47041754A083A51601E
:1018800063E073495031884208D171490839496889
:1018900041F470216E4A083A516056E06C49643157
:1018A000884208D16A490839496841F47001684A98
:1018B000083A516049E066497831884208D1644964
:1018C0000839496841F07061614A083A51603CE06A
:1018D0006049884206D1011F096841F00F01021FCB
:1018E000116032E05B491431884208D15949091F1F
:1018F000096841F0F001574A121F116025E055496F
:101900002831884208D15349091F096841F47061A0
:10191000504A121F116018E04E493C31884208D1EC
:101920004C49091F096841F470414A4A121F11606D
:101930000BE048495031884207D14649091F0968E0
:1019400041F47021434A121F1160704710B5002204
:10195000026847F6F0739A430C6A8B6823430C695C
:1019600023434C6923438C692343CC6923434C6A4A
:1019700023438C6A23431A430260CB6843600B689D
:1019800083604B68C36010BD0021016041608160CD
:10199000C160016141618161C16101624162816235
:1019A000704721B1026842F00102026004E002685F
:1019B0004FF6FE731A40026070471AB103680B437A
:1019C000036002E003688B43036070474160704727
:1019D0000146486880B2704701460020002211F09D
:1019E000805F03D01B4B083B1A6802E0184B083B92
:1019F0001A680A4201D0012000E00020704710F070
:101A0000805F03D01349091F086002E010490839BC
:101A10004860704701460020002211F0805F03D02B
:101A20000C4B083B1A6802E0094B083B1A680A4253
:101A300001D0012000E00020704710F0805F03D04B
:101A40000449091F086002E00149083948607047ED
:101A5000080002400804024001460020FE4A1068C7
:101A600000F03800084310607047FB49096821F016
:101A70000801F94A11601146096801431160704775
:101A8000F549096821F01001F34A1160114609680F
:101A9000014311607047F148EF494860F0484860E1
:101AA0007047EE48EC494860ED4848607047EA48A6
:101AB000006940F08000E84908617047E648006925
:101AC00040F08000E449086170470420E249C96899
:101AD00011F0010F01D001200EE0DF49C96811F0BB
:101AE000040F01D0022007E0DB49C96811F0100F94
:101AF00001D0032000E00420704700B50246042313
:101B0000FFF7E3FF034603E0FFF7DFFF0346521E44
:101B1000012B01D1002AF7D102B90523184600BDD7
:101B200030B5044604254FF43020FFF7E6FF0546A4
:101B3000042D17D1C848006940F00200C649086169
:101B400008464461006940F0400008614FF43020CD
:101B5000FFF7D3FF0546C048006941F6FD71084014
:101B6000BD490861284630BD10B504244FF430202B
:101B7000FFF7C3FF0446042C16D1B748006940F0B4
:101B80000400B54908610846006940F0400008615A
:101B90004FF43020FFF7B1FF0446AF48006941F62B
:101BA000FB710840AC490861204610BD00B50246F3
:101BB0000423FFF78AFF034603E0FFF786FF03468F
:101BC000521E012B01D1002AF7D102B90523184674
:101BD00000BD10B504244FF43020FFF7E7FF0446A2
:101BE000042C16D19C48006940F004009A49086111
:101BF0000846006940F0400008614FF43020FFF7CC
:101C0000D5FF04469448006941F6FB7108409249AB
:101C10000861204610BD00208F49C96911F0020FEC
:101C200001D0012000E00020704730B5A525042434
:101C3000FFF7F1FF00B100254FF43020FFF75DFF03
:101C40000446042C3AD185488349886084488860DA
:101C50000846006940F0200008610846006940F02D
:101C6000400008614FF43020FFF747FF0446042C82
:101C70001BD17948006941F6DF7108407649086157
:101C80000846006940F01000086176480580E002CF
:101C9000FFF733FF0446052C10D06F48006941F66A
:101CA000EF7108406C49086108E0052C06D06A48CD
:101CB000006941F6EF71084067490861204630BD70
:101CC00078B506460C46042500200090E802FFF790
:101CD00014FF0546042D24D15F48006940F001003F
:101CE0005D4908613480E802FFF707FF0546042DCF
:101CF00010D1B01C0090200C00990880E802FFF77A
:101D0000FCFE05465448006941F6FE710840524900
:101D1000086106E05048006941F6FE7108404E49EE
:101D20000861284678BD70B504460D460426F002C9
:101D3000FFF7E3FE0646042E11D14748006940F044
:101D40000100454908612580F002FFF7D6FE0646EE
:101D50004148006941F6FE7108403F49086130463C
:101D600070BD70B505460E460424E002FFF7C5FEBF
:101D70000446042C17D139483749886038488860B0
:101D80000846006940F0100008612E80E002FFF76D
:101D9000B4FE0446052C06D02F48006941F6EF71C9
:101DA00008402D490861204670BD2DE9F0430446E6
:101DB0004FF6FF763746B046B1460425E443E6B217
:101DC000C4F30727C4F307484FEA1469E802FFF792
:101DD00094FE0546042D49D120481F4988602048BB
:101DE00088600846006940F010000861FF2E06D0A8
:101DF0001C4808300680E802FFF77FFE0546042DE8
:101E000008D1FF2F06D017480A300780E802FFF7F5
:101E100074FE0546042D0AD1B8F1FF0F07D0114812
:101E20000C30A0F80080E802FFF767FE0546042D9D
:101E30000AD1B9F1FF0F07D00A480E30A0F8009080
:101E4000E802FFF75AFE0546052D0FD0024800694B
:101E500041F6EF71084007E000200240230167458A
:101E6000AB89EFCD00F8FF1F664908612846BDE841
:101E7000F08330B5054604244FF43020FFF73DFED3
:101E80000446042C41D160485E4988605F48886000
:101E90000846006940F0200008610846006940F0EB
:101EA000400008614FF43020FFF727FE0446042C61
:101EB00022D15448006941F6DF7108405149086158
:101EC0000846006940F0100008611DB1002050492B
:101ED000088002E0A5204E4908804FF43020FFF72B
:101EE0000CFE0446052C10D04648006941F6EF71FF
:101EF00008404449086108E0052C06D041480069C3
:101F000041F6DF7108403F490861204630BDF0B519
:101F100005460E46174604243B483A4988603B482C
:101F20008860E002FFF7E9FD0446042C19D135482A
:101F3000006940F010003349086147F0F800304371
:101F400028433349891C0880E002FFF7D6FD044688
:101F5000052C06D02B48006941F6EF71084029494D
:101F600008612046F0BD2748C069800870472548B1
:101F7000006A704700202349096811F0200F01D042
:101F8000012000E00020704729B11E4A1269024377
:101F90001C4B1A6104E01B4A12698243194B1A61F7
:101FA000704701460020012908D1164AD26912F073
:101FB000010F01D0012008E0002006E0114AD2689C
:101FC0000A4201D0012000E0002070470D49C8609E
:101FD000704704200B49C96811F0010F01D001209E
:101FE0000EE00849C96811F0040F01D0022007E093
:101FF0000449C96811F0100F01D0032000E004204B
:10200000704700000020024023016745AB89EFCDF7
:1020100000F8FF1F0E49086070470D49486070477F
:102020000B49886070474AF6AA2009490860704742
:102030004CF6CC4006490860704701460020044A2F
:10204000D2680A4201D0012000E000207047000061
:102050000030004008B54FF48070ADF8000010204B
:102060008DF8030003208DF802006946FE48FEF754
:102070001FFD0020FD49086008BD08B54FF48060D1
:10208000ADF8000010208DF8030003208DF8020049
:102090006946F748FEF70CFD4FF40060ADF800000C
:1020A00010208DF8030003208DF802006946F048E7
:1020B000FEF7FEFC4FF48050ADF8000010208DF8C4
:1020C000030003208DF802006946E948FEF7F0FCA2
:1020D00008BD08B54020ADF8000010208DF80300C1
:1020E00003208DF802006946E248FEF7E1FC4FF458
:1020F0000040ADF8000010208DF8030003208DF89B
:1021000002006946DA48FEF7D3FC08BD08B538205E
:10211000ADF8000018208DF8030003208DF80200B0
:102120006946D548FEF7C4FC8020ADF800001020B9
:102130008DF8030003208DF802006946CE48FEF7B3
:10214000B7FC8021CC48FEF75EFD8020ADF8000092
:1021500010208DF8030003208DF802006946C44862
:10216000FEF7A6FC8021C248FEF74DFD08BD08B56C
:102170000820ADF8000010208DF8030003208DF832
:1021800002006946BD48FEF793FC0020BC49086088
:1021900008BD08B50820ADF8000000208DF8030048
:1021A00003208DF802006946B448FEF781FC08BDA3
:1021B00008B50120ADF8000010208DF803000320C1
:1021C0008DF802006946AD48FEF772FC0220ADF8BA
:1021D000000010208DF8030003208DF802006946EE
:1021E000A648FEF765FC4FF48070ADF800001020A3
:1021F0008DF8030003208DF8020069469E48FEF723
:1022000057FC4FF40070ADF8000010208DF803006B
:1022100003208DF8020069469748FEF749FC01212A
:102220009648FEF7F0FC08BD08B50120ADF80000A7
:1022300028208DF8030003208DF8020069468F489E
:10224000FEF736FC0220ADF8000028208DF80300D0
:1022500003208DF8020069468848FEF729FC4FF4F8
:102260008070ADF8000028208DF8030003208DF861
:10227000020069468048FEF71BFC4FF40070ADF881
:10228000000028208DF8030003208DF80200694625
:102290007948FEF70DFC08BD08B501210420FEF7C2
:1022A000BDFEFF20ADF8000010208DF803000320D4
:1022B0008DF8020069466C48FEF7FAFB0121082000
:1022C000FEF7ACFE4FF44050ADF8000028208DF82A
:1022D000030003208DF8020069466748FEF7E8FB1B
:1022E0004FF44040ADF8000010208DF803000320AB
:1022F0008DF8020069466048FEF7DAFB01214020B4
:10230000FEF78CFE4020ADF8000010208DF8030091
:1023100003208DF8020069465848FEF7C9FB0020EB
:10232000584908605849C1F8B801584908605849E7
:10233000086001F10401086001F10401086001F185
:102340000401086001F10401086001F10401086062
:1023500001F10401086001F10401086008BD08B53D
:1023600001210420FEF75AFEFF20ADF800000020F6
:102370008DF8030003208DF8020069463A48FEF705
:1023800097FB01210820FEF749FE4FF44050ADF8BD
:10239000000000208DF8030003208DF8020069463C
:1023A0003548FEF785FB4FF44040ADF800000020B3
:1023B0008DF8030003208DF8020069462E48FEF7D1
:1023C00077FB01214020FEF729FE4020ADF80000F8
:1023D00000208DF8030003208DF80200694627488D
:1023E000FEF766FB08BD08B50220ADF8000000202E
:1023F0008DF8030069461F48FEF75AFB0120ADF82F
:10240000000000208DF8030069461A48FEF750FBD3
:1024100008BD08B50220ADF8000000208DF80300CB
:1024200069461448FEF744FB08BD08B50120ADF825
:10243000000000208DF8030069460E48FEF738FBC7
:1024400008BD08B58020ADF8000028208DF80300F5
:1024500069460848FEF72CFB4FF48070ADF8000089
:102460006946044816E0000000080140A00121422E
:102470000014014000100140000C01400018014010
:102480008C0123429801234200802142BC812142D9
:1024900080012142FEF70CFB4FF40070ADF8000004
:1024A0006946FE48FEF704FB08BD08B50220ADF8FA
:1024B000000010208DF8030003208DF8020069460B
:1024C000F748FEF7F5FA0020F649086008BD08B5A0
:1024D0004FF40070ADF8000018208DF80300694635
:1024E000F148FEF7E5FA4FF48060ADF800000420F3
:1024F0008DF803006946EC48FEF7DAFA08BD08B526
:102500004FF40070ADF8000000208DF8030069461C
:10251000E548FEF7CDFA4FF48060ADF800000020EA
:102520008DF803006946E048FEF7C2FA4FF4807068
:10253000ADF8000000208DF8030003208DF80200A4
:102540006946D948FEF7B4FA08BD08B54FF4005003
:10255000ADF8000010208DF8030003208DF8020074
:102560006946D248FEF7A4FA4FF48040ADF8000067
:1025700010208DF8030003208DF802006946CB4837
:10258000FEF796FA4FF40060ADF8000028208DF8B1
:1025900003006946C548FEF78BFA4FF40051C34863
:1025A000FEF731FB4FF48041C048FEF72CFB08BD1D
:1025B00008B54FF40050ADF8000018208DF8030066
:1025C00003208DF802006946B548FEF771FA08BD90
:1025D00008B54FF40040ADF8000010208DF803005E
:1025E00003208DF802006946AD48FEF761FA4FF40A
:1025F0000041AB48FEF709FB08BD08B54FF4005099
:10260000ADF8000000208DF8030003208DF80200D3
:102610006946A348FEF74CFA08BD08B54FF40040E0
:10262000ADF8000010208DF8030003208DF80200A3
:1026300069469D48FEF73CFA00209D49086008BDA8
:1026400008B58020ADF8000010208DF803000320AD
:102650008DF8020069469548FEF72AFA0020954950
:10266000086008BD08B58020ADF8000010208DF886
:10267000030003208DF8020069468C48FEF718FA23
:1026800000208C49086008BD08B50220ADF80000A4
:1026900010208DF8030003208DF802006946804861
:1026A000FEF706FA00207F49086008BD08B54FF420
:1026B0008060ADF8000018208DF8030003208DF82D
:1026C000020069467C48FEF7F3F94FF40060ADF86C
:1026D000000004208DF8030003208DF802006946F5
:1026E0007548FEF7E5F94FF48070ADF80000102052
:1026F0008DF8030003208DF8020069466B48FEF751
:10270000D7F901206D49086008BD08B58020ADF8F3
:10271000000000208DF8030003208DF802006946B8
:102720006248FEF7C5F94FF48060ADF80000002064
:102730008DF8030003208DF8020069465E48FEF71D
:10274000B7F94FF40060ADF8000000208DF80300E9
:1027500069465948FEF7ACF94FF48070ADF80000B7
:1027600000208DF8030003208DF8020069464F48D1
:10277000FEF79EF901205149086008BD08B5012007
:10278000ADF8000010208DF8030003208DF8020042
:1027900069464948FEF78CF94FF40060ADF8000037
:1027A00010208DF8030003208DF8020069463F4891
:1027B000FEF77EF90020424908604249C1F88001D5
:1027C00008BD08B54FF40060ADF8000010208DF88A
:1027D000030003208DF8020069463348FEF768F9CC
:1027E00000203949086008BD10B54FF400612E483B
:1027F000FEF7FCF908B9012000E00020044622465B
:102800004FF400612848FEF702FA10BD08B52020F9
:10281000ADF8000010208DF8030003208DF80200B1
:1028200069461E48FEF744F900202849086008BDA3
:1028300008B54FF40060ADF8000010208DF80300DB
:1028400003208DF8020069461848FEF731F9002090
:102850001B49086008BD08B54FF40060ADF80000E2
:1028600004208DF8030003208DF8020069460E480D
:10287000FEF71EF908BD704708B54FF2FF70ADF8BE
:10288000000000208DF8030069460748FEF710F9A4
:102890004FF6FF70ADF80000002019E00010014075
:1028A00000140140848122420008014000180140C8
:1028B000BC0121429C012342000C0140A0012342A3
:1028C000AC01234200802142AC012142940122420A
:1028D0008DF8030069461748FEF7EAF84FF6F770DF
:1028E000ADF8000000208DF8030069461248FEF79D
:1028F000DFF80820ADF8000004208DF803006946D9
:102900000D48FEF7D5F84FF6FF70ADF80000002037
:102910008DF8030069460948FEF7CAF847F6F770D4
:10292000ADF8000000208DF8030069460448FEF76A
:10293000BFF808BD000C0140001001400014014028
:102940000018014070B504460D46002305E02678C6
:102950002E706D1C641C5E1CF3B29342F7DB70BDDD
:102960000146088870472DE9F04105460E46174696
:10297000002407E036F814102846FFF7D4F9AD1C00
:10298000601C84B2BC42F5DBBDE8F08130B5034683
:102990000C461546002207E01846FFF7E1FF24F831
:1029A00012009B1C501C82B2AA42F5DB30BD2DE9FF
:1029B000F04106460F461446204604EBD0714910FC
:1029C000A4EB4101012905D104EBD0714910491C48
:1029D0008DB203E0204604EBD0714D10FFF75BF899
:1029E0002A4631463846FFF7BEFFFFF760F8BDE8DC
:1029F000F08110B5D648006800285FD0D54800782F
:102A000000285CDD00BFD3480078401DD04909682C
:102A10008842F8D8CF48C078C8B9FFF7E5FE00244F
:102A20000DE0201DCB49085CCB49CC4A1268885484
:102A3000CA480068401CC9490860601CC4B2C54847
:102A40000078A042EDDC0020C149086013E0C148D5
:102A5000C07805280FD1BF480079C1490870BD482A
:102A600040794870BB4880798870BA48C079C8708E
:102A70000020B7490860B9480068B0F5006F13D16D
:102A8000FFF7B2FE4FF40062B6480168B248FFF7A4
:102A90008EFFB448006800F50060B249086000206D
:102AA000AE490860FFF7A0FEAA490978091DA94AA6
:102AB00088180121FDF706FDFFF796FE31E0A448D6
:102AC000006805282DD1A348407850BBA1488078E4
:102AD00038BBA048C078012823D19E480079FF2840
:102AE0001FD1FFF781FE9D48008882B29D48016892
:102AF0009948FFF75CFFFFF777FE9A48006897490F
:102B0000096808449749086000209449086001203A
:102B10009549087001218F48001DFDF7D3FCFFF790
:102B200063FEFFF761FE10BD10B5FFF75DFE88483C
:102B30000068002843D0874800788C49097888428B
:102B40003AD18348006807282ED1824840788749C7
:102B50004978884224D17F4880788449897888429E
:102B60001ED17C48C0788149C978884218D17948FB
:102B700000797E490979884212D1764840797B49AB
:102B8000497988420CD1734880797849897988429B
:102B900006D100206E490860FFF726FE012010BD17
:102BA00000206B4908600AE069480068072806D9D8
:102BB00000206749086002E00020654908600020A5
:102BC000EDE710B56A4CFEF766FFFFF70DFE00BF9C
:102BD00006E0FFF709FE2046FEF7A2FF04F50064B9
:102BE00064488442F5D3FFF7FFFDFEF760FF10BD98
:102BF00070B505460024FEF74EFFFFF7F5FD5E4871
:102C0000FEF78EFFFFF7F0FD10225C495A48FFF7F0
:102C1000AAFEFFF7E9FDFEF74AFF70BD10B50446B6
:102C2000206857490840B0F1005F08D160685549F5
:102C300008602068FDF78FFA52480068804710BD91
:102C400000BFFFF7D1FDFFF7BCFF0020404908603F
:102C500042490860464843490860002042490870DC
:102C600007214948FDF72EFC16E003E0FFF7BCFD05
:102C7000FFF7BFFE3C4800780028F7D008E0FFF7D8
:102C8000B3FD38480068FFF7B3FF3948FFF7C6FFC8
:102C9000354800780128F2D0E7E710B572B6002178
:102CA0003A48FEF77CFC0520FDF7E2FA002038499F
:102CB00008604FF00A00FDF7DBFA002080F310886F
:102CC00000BF2B48FFF7AAFF10BD10B5FFF78CFD22
:102CD000FEF7E1FE10222F492748FFF757FEFEF7C7
:102CE000E6FEFFF781FD00240AE02A4830F81400D0
:102CF000224931F81410884200D003E0601CC4B2AD
:102D0000102CF2DB00BF0F2C03DDFFF76DFD01205F
:102D100010BDFFF769FD0020FAE710B540F225511C
:102D20001A48FEF72DFD88B11848FEF7A9FC09499D
:102D3000074A1268885406480068401C0449086025
:102D400008460068642801D30020086010BD000018
:102D50003800002072010020420200203C000020C8
:102D6000300000202C00002034000020B42F000888
:102D7000008000080000080800780008BC2F000848
:102D80000000FE2F40000020A62F00080048004051
:102D900084812242A60A002010B501217C20FEF782
:102DA0003DF901210846FEF739F9FFF70AFD4FF416
:102DB00000616248FDF71AFF08B9012000E0002019
:102DC000044622464FF400615C48FDF720FFFFF700
:102DD0009DF9FFF76AFBFFF7CAF90120584908601F
:102DE000FFF7E6F9FFF7CAFCFFF7AFFBFFF7E0FBE1
:102DF000FFF7EEFBFFF725FBFFF70FFCFFF7AFFA3E
:102E0000FFF71EFCFFF737FD10BD08B5012150206C
:102E1000FEF704F903208DF8020048208DF8030026
:102E20000120ADF8000069464648FDF741FE4FF429
:102E30000070ADF8000069464348FDF739FE1020E8
:102E40008DF803000220ADF8000069463D48FDF70B
:102E50002FFE4FF48060ADF8000069463A48FDF758
:102E600027FE4FF480613848FDF7CDFE022135483A
:102E7000FDF7C9FE01203549086008BD10B50121E4
:102E80007C20FEF7CBF801210846FEF7C7F8FFF7D4
:102E90006EF901202A490860FFF78AF9FFF76EFCF6
:102EA000FFF753FBFFF7CDFAFFF7E5FC10BD10B5B8
:102EB0004FF48030FDF768FFFDF7A5FF0446012CB5
:102EC00010D10020FDF7E5FFA002FDF7EBFF002089
:102ED000FDF7F1FF0120FDF7CEFF00BFFDF7D4FFA6
:102EE0000428FBD110BD10B545F25550FFF792F8FC
:102EF0000520FFF792F84FF42F70FFF791F8FFF7D6
:102F000092F8FFF795F810BD10B5FFF78CF810BDDB
:102F100010B50121C803FEF78EF801210846FEF71F
:102F20007DF801210A48FDF792FEFDF731FB10BD47
:102F300010B54FF4E130FDF7C7F910BD00080140AE
:102F40008C012342001001400018014094012242EC
:102F500000023000421C10F8011B0029FBD1801A2E
:102F600070470000064C074D06E0E06840F00103A2
:102F700094E8070098471034AC42F6D3FDF7DCF82C
:102F8000DC2F0008FC2F000802E008C8121F08C14F
:102F9000002AFAD170477047002001E001C1121FDA
:102FA000002AFBD170470301AA55038D3E0301059A
:102FB0000A035C37040255AA03C9FA000000110095
:102FC0002200330044005500660077008800990015
:102FD000AA00BB00CC00DD00EE00FF00FC2F0008C3
:102FE0000000002044000000882F00084030000846
:102FF000440000208C120000982F00080000000000
:10300000001BB700000000000000000001020304E4
:10301000060708090000000001020304010203047E
:10302000060708090204060800000000000000006E
:103030000000000000000000000000000000000090
:0400000508000131BD
:020000040800F2
:10780000000011002200330044005500660077009C
:1078100088009900AA00BB00CC00DD00EE00FF004C
:020000040800F2
:10800000A8520020E90501081D0401081F04010809
:1080100023040108270401082B04010800000000C4
:108020000000000000000000000000002F04010814
:108030003104010800000000330401083504010880
:1080400003060108030601080306010803060108E8
:1080500003060108030601080306010803060108D8
:1080600003060108030601080306010803060108C8
:1080700003060108030601080306010803060108B8
:1080800003060108030601080306010803060108A8
:10809000030601080306010803060108FD8900081C
:1080A0000306010803060108030601080306010888
:1080B0009589000803060108F77104080306010802
:1080C0000306010803060108030601080306010868
:1080D0000306010803060108030601080306010858
:1080E000498A00080306010803060108030601087F
:1080F0000306010803060108030601080306010838
:108100000306010803060108030601080306010827
:10811000C77004080F62020803060108030601087D
:10812000030601080306010803060108E39200089C
:10813000DFF80CD03FF086FE00480047958100082C
:10814000A8520020EFF30980704780F30988704738
:10815000EFF30880704780F30888704740BA704793
:10816000C0BA70474FF0010080F3138801480249FC
:108170000160FEE70CED00E00400FA054FF001009D
:1081800080F31388014802490160FEE70CED00E02E
:108190000400FA059D489E4908600BF03AFC34E162
:1081A00000F049FE6DE00EF058F94FF40061994877
:1081B00008F0C2FD08B9012000E000200446224674
:1081C0004FF40061934808F0C8FD56E092484079AA
:1081D000012852D19148007C01284ED100208E49BF
:1081E000487100F039FE4FF400618A4808F0A4FDA0
:1081F00008B9012000E00020044622464FF4006147
:10820000844808F0AAFD01F09FFF17F0FBFB17F070
:10821000C3FC1DF081FC1DF0ABFC1AF0D0FA19F084
:108220004EFD00F019FE4FF400617A4808F084FD1D
:1082300008B9012000E00020044622464FF4006106
:10824000744808F08AFD0CF0CDFD07F0C9F81EF067
:10825000FDFA3AF035FF0EF0EEFA13F0D0F813F015
:10826000EEF93CF003FB0DF06DFC16F0F5FA0CF0A6
:10827000CDFE11F0CEFC0CF064FD684800780128BA
:10828000A4D06648007801288DD084E00EF055F91E
:108290004FF400615F4808F04FFD08B9012000E08D
:1082A0000020044622464FF400615A4808F055FD6C
:1082B0006DE059484079012869D15848007C002870
:1082C00065D15549487100F084FD00F0C5FD4FF4BB
:1082D0000061504808F030FD08B9012000E000209E
:1082E000044622464FF400614A4808F036FD01F08A
:1082F0002BFF17F051FC4A4991F8551041B14849FC
:1083000091F85510012902D14449088E00E000BFC0
:108310001AF055FA19F0D3FC07F062F800F09CFD52
:108320004FF400613B4808F007FD08B9012000E068
:108330000020044622464FF40061364808F00DFD47
:108340001EF084FA3AF0BCFE0EF075FA0CF01BFD3C
:1083500013F055F83CF08AFA0DF0F4FB16F07CFAB5
:108360002E48007C012801D02C4840790CF04EFEAC
:1083700011F04FFC0CF0E5FC0EF013F838B912F0D8
:1083800083FD012108460AF03BFB00F033FB234844
:10839000007802288DD02148007802283FF476AF7B
:1083A00021E00DF0CDFF18E00CF01CFD0A2000F0DC
:1083B00078F80EF042F800F04FFD4FF400611548D8
:1083C00008F0BAFC08B9012000E00020044622466B
:1083D0004FF400610F4808F0C0FC104800780328F3
:1083E000E2D00DF0B8FF0D4800780328D9D008E09E
:1083F00003E012F073FC16F089FA084800780428AC
:10840000F7D0064800780428F2D0C9E600800008BA
:1084100008ED00E00008014004000020A216002042
:108420004224002010B5042008F03FF92F480068CE
:1084300000EB400080002E49B0FBF1F02D490870A0
:108440000846007800EB4001C1EBC0104FF6FF7109
:1084500001EAC0002849088010BD0146254A12786B
:108460004A434FF0E0235A6100229A611A4612698A
:1084700042F001021A6100BF4FF0E022106900F0E3
:1084800001021AB100F48032002AF5D04FF0E02248
:10849000126922F001024FF0E0231A6100229A6172
:1084A00070470146144A12884A434FF0E0235A614C
:1084B00000229A611A46126942F001021A6100BF55
:1084C0004FF0E022106900F001021AB100F480328E
:1084D000002AF5D04FF0E022126922F001024FF09D
:1084E000E0231A6100229A617047000030000020EA
:1084F000001BB700000000200200002008B5012189
:10850000202008F035FE4FF4E050ADF800001020B8
:108510008DF8030003208DF8020069463D4808F0FD
:108520006BFB08BD10B5002404E00120FFF795FFA8
:10853000601CC4B2042CF8DB10BD2DE9FC5F83463F
:1085400058463FF0FEFA05460022334B3FF00CFB45
:1085500001D2DFF8C8B0324958463FF05BFB01D288
:10856000DFF8BCB058463FF0ECFA07462D4A2E4BD8
:108570003FF024F905462D4A2D4B3FF078F8CDE920
:1085800000013FF021FB8346254958463FF042FB5E
:1085900001D2DFF88CB058463FF0D3FA00221E4BD0
:1085A000CDE900013FF004F90546224A224B3FF095
:1085B00077F907463FF06FFA814609F5605A0024C3
:1085C00011E000201D490860C4F110002AFA00F0F3
:1085D0001B49C1F8A801FFF7A5FF01201749086052
:1085E000FFF7A0FF641C112CEBD300201349086097
:1085F0001349C1F8A801FFF795FF01200F49091D94
:108600000860FFF78FFF00200D49C1F8B001BDE8F9
:10861000FC9F00000014014000000C40000060407E
:108620000000C041A01A2FDD2406F03F7F87A24042
:108630009FC8933F74479CA1FAFF2F3FAC81224211
:108640000080224210B586B0044601214FF4047028
:1086500008F08EFD4FF4004008F0EEFC0820ADF865
:10866000000000208DF8030003208DF80200694609
:10867000A64808F0C1FA002001908DF808008DF896
:1086800009004FF460200390002004900D208DF825
:10869000140001A99E4808F04EF8012C02D10120D7
:1086A00008F006FA01219A4808F071F8984808F095
:1086B00090F800BF964808F091F80028FAD1944845
:1086C00008F096F800BF924808F097F80028FAD111
:1086D00006B010BD38B5044600214FF4007008F014
:1086E00047FD012C02D1002008F0E2F9884807F08C
:1086F000FBFF0021864808F04AF80820ADF800008A
:1087000000208DF8030003208DF8020069467F48A1
:1087100008F072FA38BD70B50446052301222146DF
:108720007B4808F0A0F80121794808F070F800BFF4
:108730000221774808F0DCF90028F9D0744808F0E5
:10874000F9F80546284670BD10B50121704808F0BB
:108750005EF800BF02216E4808F0CAF90028F9D07F
:108760006B4808F0E7F810BD2DE9F0478CB0824661
:10877000894600254846FFF765FF00240AE0504679
:10878000FFF7C9FF01A921F8140001A830F814006F
:108790000544641C142CF2D34846FFF79BFFBDF838
:1087A0000870BDF80880032410E001A830F8140018
:1087B000B84202D201A830F8147001A830F81400B1
:1087C000404502D901A830F81480641C132CECD366
:1087D0000025022604E001A830F816000544761CA6
:1087E000132EF8D3E81BA0EB08050F20B5FBF0F51E
:1087F000A8B20CB0BDE8F0872DE9F047AEB08046D6
:1088000000202B90FFF71EFF00251DE0D8F8001078
:1088100031F815003FF0D2F802AA02EBC50203C2FC
:108820002B983FF0CBF8CDE9000102A800EBC50082
:10883000D0E90063324600983EF019FF81463FF0D0
:108840002AF92B90681C85B2142DDFDB2B983FF0A2
:10885000B5F8064600222F4B3FF022F8CDE92C0157
:1088600000202B90DDE92C013FF0AEF90646DDE952
:108870002C013FF0A9F90746DDE9022110463FF03F
:10888000A3F98146DDE9042110463FF09DF98246B7
:1088900033463A46494616F0ECF8022425E002A891
:1088A00000EBC400D0E9002110463FF08DF90746E7
:1088B00016F0E9F806463FF044F902AA02EBC402BA
:1088C00003C22B983FF07AF8814602A800EBC4005F
:1088D000D0E90063324648463EF0C9FECDE90001CA
:1088E0003FF0D9F82B90601C84B2142CD7DB2B9866
:1088F0003FF064F806460022074B3EF0D1FFCDE979
:108900002C01DDE92C012EB0BDE8F08700100140FC
:1089100000240140000034400000324010B5012125
:108920007C2008F025FC0121084608F021FC0121EB
:10893000C80308F02AFC0121880408F026FC012164
:10894000084608F008FC0121102008F011FC012164
:10895000C80408F01AFC0121880308F009FC012171
:10896000080508F005FC10BD38B504461C208DF83C
:10897000000001208DF801008DF80200012C02D1C9
:108980008DF8030002E000208DF80300684607F030
:1089900042FE38BD10B50121880709F04AFB50B1ED
:1089A0000121880709F056FB0020FE498871FE4925
:1089B0000860FFF7D9FF10BD10B54FF4803008F004
:1089C00089FA08F0C6FA0446012C10D1002008F0FC
:1089D00006FBA00208F00CFBA00208F012FB01202D
:1089E00008F0EFFA00BF08F0F5FA0428FBD1FFF712
:1089F00095FF10BD10B5FFF7DFFF10BD10B540208B
:108A00000AF098FBF8B140200AF0A5FBFFF7F2FF4F
:108A100006F02AFBE548006858B90A20FFF741FD37
:108A2000E248006878B90120E149087302204873E0
:108A300009E00A20FFF735FDDC480068012802D173
:108A4000DB490873487310BD10B54FF400400AF0BD
:108A500071FBA0B14FF400400AF07DFBD54880784F
:108A6000012802D1D349487102E00120D14948715F
:108A7000D148D0F80500401CCF49C1F805004FF49B
:108A800000600AF057FB30B14FF400600AF063FB5E
:108A90000120CA49887410BD3EB504464FF080409D
:108AA00008F0CEFB0121084608F06FFB6000401E75
:108AB00080B2ADF8040041F26F70ADF80000002004
:108AC000ADF80600ADF8020069464FF0804008F0AE
:108AD0008BFC0121880709F0A9FA012211469007B1
:108AE00008F0F9FF0120FFF73FFF0121880708F098
:108AF000D7FF3EBD0EB54FF4E06007F087FD28209C
:108B00008DF8080000208DF809008DF80A0001207A
:108B10008DF80B0002A807F07EFD0F21042008F05D
:108B200081F94FF40040009000208DF804000C20E3
:108B30008DF8050001208DF8060068460AF094FAC9
:108B40000EBD0EB54FF4E06007F060FD28208DF8F3
:108B5000080000208DF809008DF80B0002A807F02E
:108B60005AFD0F21042008F05DF94FF400400090F9
:108B700000208DF804000C208DF8050000208DF8F1
:108B8000060068460AF070FA0EBD0EB517208DF883
:108B9000080001208DF8090000208DF80A0001204E
:108BA0008DF80B0002A807F036FD0621022008F020
:108BB00039F94020009000208DF8040010208DF835
:108BC000050001208DF8060068460AF04DFA0EBD3A
:108BD0000EB54FF4A06007F019FD17208DF80800BE
:108BE00001208DF8090000208DF80A008DF80B0097
:108BF00002A807F010FD0621022008F013F940201A
:108C0000009000208DF804000C208DF80500002055
:108C10008DF8060068460AF027FA0EBD0EB528202A
:108C20008DF8080001208DF809008DF80A008DF8F4
:108C30000B0002A807F0EFFC0B21022008F0F2F86D
:108C40004FF40060009000208DF804000C208DF897
:108C5000050001208DF8060068460AF005FA0EBDF1
:108C60000EB54FF4A06007F0D1FC28208DF8080065
:108C700001208DF809008DF80A0000208DF80B0006
:108C800002A807F0C8FC0B21022008F0CBF84FF433
:108C90000060009000208DF8040008208DF8050089
:108CA00000208DF8060068460AF0DEF90EBD10B50A
:108CB00080200AF03FFA044614B180200AF04BFAF3
:108CC00010BD10B5044607F0A3FBFFF713FFFFF735
:108CD0005CFFFFF7A3FF002080F3108800BF10BDEA
:108CE00010B504462046FFF7D7FE01202E49086044
:108CF00010BD10B501217C2008F03AFA0121084688
:108D000008F036FA11F0DAFF4FF400612C4808F051
:108D100013F808B9012000E00020044622464FF471
:108D20000061274808F019F811F0ADFC11F0DCFCE7
:108D300011F0F8FC06F07AF900201C49683108604F
:108D400011F065FF11F03AFE11F087FF00201D4978
:108D5000C1F8940111F06FFF002014496C310860D4
:108D600011F070FE12F03CF811F04EFC11F0F3FD22
:108D700011F09EFE11F0A7FD11F0ADFE11F0DBFE2B
:108D800021F071FB00201049C1F8840106F06CF954
:108D9000FFF7B4FB3AF03CFC3AF040FC3AF05EFCE2
:108DA00014E00000A2160020BC81224218012242D9
:108DB000F60F0020040000205F1A0020D947002091
:108DC00000080140000022420080224212F03FF8D9
:108DD00010BD10B501217C2008F0CAF90121084618
:108DE00008F0C6F911F06AFF4FF400611C4807F063
:108DF000A3FF08B9012000E00020044622464FF4FA
:108E00000061174807F0A9FF11F001FF11F0E8FF1A
:108E100011F0D4FD10BD10B50121C80308F0B5F95B
:108E20000121084608F0A4F901210E4807F0B5FF1A
:108E300000F08AFA10BD10B545F255500AF094F9C9
:108E400005200AF094F94FF4EA700AF093F90AF059
:108E500094F90AF097F910BD10B50AF08EF910BD1B
:108E6000000801400002300030B587B004460D46CE
:108E7000444808F0E5F90121042008F086F90121B1
:108E8000084608F075F90121080307F086FF601E07
:108E900080B2ADF81400681E80B2ADF8100000205A
:108EA000ADF81600ADF8120004A9364808F09CFA97
:108EB0006020ADF800000120ADF80200204604EB70
:108EC000D071C1F34F01ADF806100220ADF80800D3
:108ED00069462C4808F007FB08212A4808F019FFCA
:108EE0000121284808F0DCFE0121264808F0D8FDC1
:108EF00007B030BD30B587B005460C46224808F0B3
:108F00009FF90121022008F040F90121084608F0EC
:108F10002FF901211D4807F040FF4FF47A70ADF89A
:108F2000140040F6B830ADF810004FF40070ADF802
:108F300016000020ADF8120004A9134808F054FAF6
:108F40007020ADF800000120ADF80200ADF8064039
:108F50000020ADF8080069460B4808F0C4FA082163
:108F6000094808F0D6FE0821074809F009F806214B
:108F7000054809F017F80121034808F091FD07B0F2
:108F800030BD0000000800400004004000081A0046
:108F900070B50024012528E080214C4807F0BFFE71
:108FA00006464FF48071494807F0B9FE46EA0026AC
:108FB0004FF40071454807F0B2FE46EA0044012034
:108FC000FFF76FFA8021414807F0A9FE06464FF4EB
:108FD00080713E4807F0A3FE46EA00264FF4007178
:108FE0003A4807F09CFE46EA0045AC42D4D1204600
:108FF00070BD70B5002401250CE00121344807F054
:109000008EFE04460120FFF74CFA0121304807F09C
:1090100086FE0546AC42F0D1204670BD1CB5072146
:10902000022007F0FFFE8020009000208DF8040051
:109030000C208DF8050000208DF8060068460AF027
:1090400013F81CBD1CB50721022007F0EBFE8020A1
:10905000009000208DF804000C208DF80500002001
:109060008DF80600684609F0FFFF1CBD1FB5802083
:10907000ADF8000048208DF803006946134807F05A
:10908000BBFD4FF4E06007F0C1FA17208DF8040033
:1090900001208DF805008DF806008DF8070001A865
:1090A00007F0B9FA0721022007F0BCFE80200290E9
:1090B00000208DF80C000C208DF80D0001208DF89B
:1090C0000E0002A809F0D0FF1FBD000000100140F3
:1090D000000C014010B590B004460121880308F04F
:1090E00047F80121084608F036F80C940020ADF846
:1090F0003400ADF83600ADF83800ADF83C000C2077
:10910000ADF83A000CA9204809F071F901211E4878
:1091100009F0F9F91D4809F02BFB1B48001D0190CF
:109120001B48029000200390C82004900020059066
:1091300080200690002007900890202009900002CF
:109140000A9000200B9001A9104809F0B3FB0122FE
:1091500040210D4809F008FA01210C4809F0D5FB1F
:1091600010B010BD10B5044600BF4021064809F0FC
:10917000A5FA0028F9D04021034809F0ACFA2146AD
:10918000014809F02DFA10BD003801405800024096
:10919000EC09002010B590B004460121482007F0EA
:1091A000E7FF0121880407F0F0FF0121084607F0DE
:1091B000D2FF0C940020ADF83400ADF83600ADF8C5
:1091C0003800ADF83C000C20ADF83A000CA9584826
:1091D00009F00DF90121564809F095F9002055498B
:1091E0000860554809F0C4FA5148001D01905348E1
:1091F0000290002003904FF46170049000200590CD
:1092000080200690002007900890202009904FF4BD
:1092100040500A9000200B9001A9474809F04AFBF2
:1092200001224021424809F09FF90121424809F0FA
:109230006CFB10B010BD30B58BB005460C463E48F7
:10924000143809F095FA3A48001D00900195102055
:109250000290039400200490802005900020069046
:10926000079008904FF40050099000200A9069463A
:109270003148143809F01EFB012280212C4809F0E6
:1092800073F90BB030BD70B505460E460120294973
:10929000086000240CE000BF4021254809F00EFAC8
:1092A0000028F9D0295D224809F09AF9601C84B29F
:1092B000B442F0DB00BF40211D4809F0FFF900284F
:1092C000F9D000201B49086070BD10B5034600208E
:1092D00000BF03E00C5C1C54441CE0B29042F9DB7C
:1092E00010BD10B5164809F03FFB00211248143894
:1092F00009F00BFB4FF49670FFF7AFF800200D4913
:10930000086010BD70B5044601200A490860204677
:109310003EF0C2F8C5B229462046FFF7B4FF01204F
:10932000FFF7BFF800200749C1F8880170BD0000B1
:109330000048004088012342300002407E0B00209C
:10934000000002100000234200B585B00020ADF8F7
:1093500000004FF48270ADF802000020ADF8040068
:10936000ADF80600ADF808004FF40070ADF80A0043
:109370000020ADF80C00ADF80E000720ADF810008D
:109380006946534808F090FE0121514808F031FF2A
:1093900005B000BD70B505460E46002405E0601C12
:1093A000C4B2C82C01DD002070BD0221284608F09F
:1093B000A4FF0028F3D03146284608F04BFF0024D4
:1093C00005E0601CC4B2C82C01DD0020ECE70121DF
:1093D000284608F092FF0028F3D0284608F03CFF0A
:1093E000C0B2E1E770B50546002405E0601CC4B2D8
:1093F000C82C01DD002070BD0221364808F07DFF39
:109400000028F3D02946334808F024FF002405E063
:10941000601CC4B2C82C01DD0020ECE701212D48FE
:1094200008F06BFF0028F3D02A4808F015FFC0B2FF
:10943000E1E770B50546002405E0601CC4B2C82C05
:1094400001DD002070BD0221214808F056FF0028F0
:10945000F3D029461E4808F0FDFE002405E0601CFC
:10946000C4B2C82C01DD0020ECE70121184808F047
:1094700044FF0028F3D0164808F0EEFEC0B2E1E742
:1094800070B50546002405E0601CC4B2C82C01DD9F
:10949000002070BD0221104808F02FFF0028F3D0F3
:1094A00029460D4808F0D6FE002405E0601CC4B231
:1094B000FF2C01DD0020ECE70121074808F01DFF2B
:1094C0000028F3D0044808F0C7FEC0B2E1E700006E
:1094D000003C0040003001400038004010B50A2038
:1094E000FEF7BBFFF9480078012808D08021F84832
:1094F00007F031FC8021F74807F02BFC07E08021C2
:10950000F44807F028FC8021F14807F022FC0520F0
:10951000FFF78FFFFF20FFF78CFF04468021EC4808
:1095200007F017FC8021EB4807F013FC204610BD24
:1095300010B500BFFFF7D2FF00F001000028F9D1FD
:1095400010BD70B506460D462C46E048007801284F
:1095500008D08021DE4807F0FEFB8021DD4807F0BF
:10956000F8FB07E08021DB4807F0F5FB8021D848B5
:1095700007F0EFFB0620FFF75CFF8021D44807F0DF
:10958000E8FB8021D34807F0E4FBD04800780128AD
:1095900008D08021CE4807F0DEFB8021CD4807F0BF
:1095A000D8FB07E08021CB4807F0D5FB8021C848D5
:1095B00007F0CFFB0220FFF73CFFC4F30740FFF7A3
:1095C00038FFC4F30720FFF734FFE0B2FFF731FFA5
:1095D0003046FFF72EFF8021BD4807F0BAFB8021FF
:1095E000BC4807F0B6FBFFF7A3FF70BD70B505469A
:1095F0002C46B6480078012808D08021B44807F0EE
:10960000AAFB8021B34807F0A4FB07E08021B14802
:1096100007F0A1FB8021AE4807F09BFB0320FFF77A
:1096200008FFC4F30740FFF704FFC4F30720FFF768
:1096300000FFE0B2FFF7FDFEFF20FFF7FAFE06464F
:109640008021A34807F085FB8021A24807F081FB19
:10965000304670BD10B504469C480078012808D0FB
:1096600080219B4807F077FB80219A4807F071FB27
:1096700007E08021974807F06EFB8021944807F0AF
:1096800068FB0620FFF7D5FE8021914807F061FBBB
:109690008021904807F05DFB8C480078012808D0B5
:1096A00080218B4807F057FB80218A4807F051FB47
:1096B00007E08021874807F04EFB8021844807F0AF
:1096C00048FB0120FFF7B5FE2046FFF7B2FE8021E0
:1096D0007F4807F03EFB80217E4807F03AFB10BD33
:1096E00010B50A20FEF7B9FE78480078012808D0A6
:1096F0008021774807F02FFB8021764807F029FB6F
:1097000007E08021734807F026FB8021704807F0AE
:1097100020FBB920FFF78DFE80216D4807F019FB73
:1097200080216C4807F015FB10BD70B505460A2076
:10973000FEF793FE65480078012808D08021644830
:1097400007F009FB8021634807F003FB07E0802155
:10975000604807F000FB80215D4807F0FAFA9F207F
:10976000FFF767FE002405E0FF20FFF762FE2855A3
:10977000601CC4B2092CF7DB8021554807F0E9FAD8
:109780008021544807F0E5FA70BD38B504462046FC
:10979000FFF72CFF8DF80000601CFFF727FF8DF806
:1097A0000100A01CFFF722FF8DF80200E01CFFF76C
:1097B0001DFF8DF80300009838BD2DE9F74F82B0EA
:1097C00082469046B8F57A6F03DD002005B0BDE80B
:1097D000F08FD1464FF0000B039C46466EB101203E
:1097E00000EB1425C4EB0520B04201D3374601E05D
:1097F000C4EB05274FF0010B01E04FF0000B74E0C4
:1098000032480078012808D08021314807F0A3FAB7
:109810008021304807F09DFA07E080212D4807F0AD
:109820009AFA80212A4807F094FA0620FFF701FEF1
:109830008021274807F08DFA8021264807F089FA11
:1098400022480078012808D08021214807F083FAB7
:109850008021204807F07DFA07E080211D4807F0AD
:109860007AFA80211A4807F074FA0220FFF7E1FD26
:10987000C4F30740FFF7DDFDC4F30720FFF7D9FD70
:10988000E0B2FFF7D6FD0020019007E019F8010BC8
:10989000FFF7CFFD0198401C80B201900198B842BB
:1098A000F4D380210A4807F054FA8021094807F0D0
:1098B00050FA3C44F61BA6B1012000EB1425C4EB82
:1098C0000520B04208D3374608E000000A00002017
:1098D00000140140000C0140C4EB05274FF0010BC0
:1098E00001E04FF0000BFFF723FEBBF1000F87D123
:1098F00000206BE738B504460D460095042221464A
:109900006846FFF75AFF38BD1CB504462046FFF7EE
:109910006DFE8DF80000601CFFF768FE8DF80100F9
:10992000A01CFFF763FE8DF80200E01CFFF75EFE4F
:109930008DF80300201DFFF759FE8DF80400601D0F
:10994000FFF754FE8DF80500A01DFFF74FFE8DF8C0
:109950000600E01DFFF74AFE8DF807009DF80000A5
:10996000FF281ED19DF80100FF281AD19DF80200A2
:10997000FF2816D19DF80300FF2812D19DF804009E
:10998000FF280ED19DF80500FF280AD19DF806009A
:10999000FF2806D19DF80700FF2802D10021009181
:1099A0000191DDE900011CBD7CB5064614461D464B
:1099B000CDE90045082231466846FFF7FEFE7CBD32
:1099C00038B504462046FFF711FE8DF80000601CF4
:1099D000FFF70CFE8DF80100A01CFFF707FE8DF8C5
:1099E0000200E01CFFF702FE8DF80300009838BD6E
:1099F00038B504460D460095042221466846FFF717
:109A0000DCFE38BD38B504462046FFF7EFFD8DF883
:109A10000000601CFFF7EAFD8DF80100BDF80000B2
:109A200038BD38B504460D460095022221466846E9
:109A3000FFF7C3FE38BD2DE9F04106460C46174638
:109A400034480078012808D08021334807F083F992
:109A50008021324807F07DF907E080212F4807F088
:109A60007AF980212C4807F074F90320FFF7E1FC14
:109A7000C4F30740FFF7DDFCC4F30720FFF7D9FC70
:109A8000E0B2FFF7D6FC002505E0FF20FFF7D1FC90
:109A90007055681C85B2BD42F7DB80211E4807F077
:109AA00058F980211D4807F054F9FFF741FDBDE842
:109AB000F08170B504460D46164601201549087020
:109AC000324629462046FFF778FE002011490870EB
:109AD00070BD70B504460D46164601200D4908704C
:109AE000324629462046FFF7A6FF002009490870A4
:109AF00070BDADF5007D002000BF06E040AA105407
:109B000000210DF80010411C88B2FF28F6DD00BFCF
:109B1000FEE700000A00002000140140000C014094
:109B200070B50346A1F16400142590FBF5F503F12F
:109B30000A0000EB400606EB001005EB800452F82B
:109B4000240070BD2DE9F04780460E4617463F4978
:109B500040463EF05FF801D228250BE03C494046E4
:109B60003EF04EF802D26FF0090503E040463DF0AA
:109B700046FF0546374930463EF04CF802D24FF4D6
:109B8000C8640AE0344930463EF03AF801D2642411
:109B900003E030463DF033FF0446012F04D0022F8E
:109BA00009D0032F15D10DE02C4A21462846FFF796
:109BB000B7FF814614E02A4A21462846FFF7B0FF46
:109BC00081460DE0274A21462846FFF7A9FF814636
:109BD00006E0224A21462846FFF7A2FF814600BF41
:109BE00000BF4846BDE8F0872DE9FF4F87B08A46A1
:109BF000934650463DF0A5FF80464FF066321A4B23
:109C00003DF035FD04460D4658463DF09AFF0646A8
:109C100022462B463DF044FECDE9020107983DF077
:109C200090FF0446114A124B3DF0C8FDCDE90001FA
:109C3000DDE902233DF0C2FDCDE904013DF0C4FFA2
:109C4000069006980BB0BDE8F08F0000000020429F
:109C5000000020C10000C8440000C842588F04081A
:109C6000E8CB04087808050866127140FA74B4FB62
:109C70003325074010B5FE48006820F07060FC49AD
:109C800008600846006840F0407008600120F9490B
:109C90000860F949C1F8B8010A20FEF7DEFB002090
:109CA000F449091D08600A20FEF7D7FB0020F2499D
:109CB000C1F8B4010A20FEF7D0FB10BD10B5EC4886
:109CC000006820F07060EA4908600846006840F0CB
:109CD000407008600020E749091D08600A20FEF76F
:109CE000BCFB0120E449C1F8B4010A20FEF7B5FB32
:109CF0000120E049091D0860002404E00A20FEF765
:109D0000ACFB601CC4B2052CF8DB10BD10B5002400
:109D1000D748006820F07060D549086008460068A0
:109D200040F0006008600A20FEF797FB0A20FEF76B
:109D300094FB07E0601CC4B2FA2C03DDFFF7BEFF02
:109D4000012010BDCB487C3800680028F2D1C949F9
:109D5000086000BFF5E710B5C548006820F07060E6
:109D6000C34908600846006840F040700860002061
:109D7000C049091D08600A20FEF76FFB0120BE499B
:109D8000C1F8B4010A20FEF768FB0020B949086059
:109D90000A20FEF762FB10BD10B5B548006820F040
:109DA0007060B34908600846006840F04070086081
:109DB0000120B049091D08600A20FEF74EFB012072
:109DC000AD49C1F8B4010A20FEF747FB0020A949BC
:109DD00008600A20FEF741FB10BD70B50446A44898
:109DE000006820F07060A24908600846006840F0F2
:109DF0004070086000251CE004F0800020B10120C4
:109E00009C49091D086003E000209A49091D08606B
:109E10006006040E0A20FEF720FB01209549086029
:109E20000A20FEF71AFB00209349C1F8B401681C10
:109E3000C5B2082DE0DB0A20FEF70FFB01208D499B
:109E400008600A20FEF709FB00208B49C1F8B40125
:109E500070BD70B5064600248548006820F070602B
:109E6000834908600846006840F0006008600025EB
:109E700015E001207F4908600A20FEF7EEFA60062F
:109E8000040E7D48D0F8380108B144F001040020E8
:109E9000784908600A20FEF7E0FA681CC5B2082D70
:109EA000E7DB7348006820F070607149086008467D
:109EB000006840F040700860204670BD2DE9F04118
:109EC00007460D461646FFF7D5FE6420FFF785FFCF
:109ED0003846FFF782FFFFF7CDFE6520FFF77DFFD5
:109EE000002407E00120FFF7B4FF2855FFF733FFF8
:109EF000601CC4B2701EA042F4DC0020FFF7A9FF72
:109F00002855FFF749FFFFF7D9FEBDE8F0812DE99D
:109F1000F04107460D461646FFF7ACFE6420FFF7FA
:109F20005CFF3846FFF759FF002404E0285DFFF787
:109F300054FF601CC4B2B442F8DBFFF7BFFEBDE8BB
:109F4000F0811CB500208DF800008DF80100022082
:109F50008DF8020000208DF8030060208DF80400C9
:109F6000052269460B20FFF7D2FF1CBD2DE9FC47F7
:109F700004460D4616461F46DDE90B9ADDF828809B
:109F80000A209AFBF0F100FB11A00A219AFBF1F1E3
:109F900040EA0110C0B28DF800000A2099FBF0F1F0
:109FA00000FB11900A2199FBF1F140EA0110C0B2C7
:109FB0008DF801000A2098FBF0F100FB11800A21C6
:109FC00098FBF1F140EA0110C0B28DF802008DF863
:109FD00003700A2096FBF0F100FB11600A2196FB4A
:109FE000F1F140EA0110C0B28DF804000A2095FB9F
:109FF000F0F100FB11500A2195FBF1F140EA01104C
:10A00000C0B28DF805000A2094FBF0F100FB11406E
:10A010000A2194FBF1F140EA0110C0B28DF806006C
:10A02000072269460020FFF772FFBDE8FC872DE993
:10A03000FC4704460D4616461F46DDE90B9ADDF83F
:10A040002880642094FBF0F100FB114084B20A20C8
:10A050009AFBF0F100FB11A00A219AFBF1F140EA12
:10A060000110C0B28DF800000A2099FBF0F105E064
:10A0700004180140B40123420000234200FB119068
:10A080000A2199FBF1F140EA0110C0B28DF80100FC
:10A090000A2098FBF0F100FB11800A2198FBF1F1F6
:10A0A00040EA0110C0B28DF802008DF803700A205A
:10A0B00096FBF0F100FB11600A2196FBF1F140EAFA
:10A0C0000110C0B28DF804000A2095FBF0F100FBEE
:10A0D00011500A2195FBF1F140EA0110C0B28DF850
:10A0E00005000A2094FBF0F100FB11400A2194FBCB
:10A0F000F1F140EA0110C0B28DF80600072269466E
:10A100000020FFF704FFBDE8FC872DE9FC4704466B
:10A110000D4616461F46DDE90B9ADDF828808DF8BE
:10A1200000A08DF801908DF802808DF803708DF8F5
:10A1300004608DF805508DF806400722694600201E
:10A14000FFF7E5FEBDE8FC8710B50722384900207F
:10A15000FFF7B4FE364880793649087034484079B4
:10A16000487033480079887031488078C87030482A
:10A17000407808712E48007848712D48007800F02A
:10A180000F002B490978090901EB810100EB41001F
:10A19000294988702648407800F00F002449497802
:10A1A000090901EB810100EB410023494870204877
:10A1B000807800F00F001E498978090901EB8101C0
:10A1C00000EB41001C4908701948C07848711848D4
:10A1D000007900F00F0016490979090901EB8101A6
:10A1E00000EB4100144908711148407900F00F005C
:10A1F0000F494979090901EB810100EB41000E4942
:10A20000C8700B488079000900EB80004FF4FA61B8
:10A2100001EB40000649897901F00F010844064925
:10A22000C88010BD03E04FF45E70FEF73AF9FAE71C
:10A230001A000020140000200C00002010B5FB487C
:10A24000006820F00F00F94908600846006840F0F7
:10A25000030008600120F6490860F649C1F8A00132
:10A260000A20FEF7FAF80020F149091F08600A20C9
:10A27000FEF7F3F80020EF49C1F8A4010A20FEF729
:10A28000ECF810BD10B5E948006820F00F00E74970
:10A2900008600846006840F0030008600020E449B8
:10A2A000091F08600A20FEF7D8F80120E149C1F82B
:10A2B000A4010A20FEF7D1F80120DD49091F08603A
:10A2C000002404E00A20FEF7C8F8601CC4B2052C84
:10A2D000F8DB10BD10B50024D448006820F00F0052
:10A2E000D24908600846006840F0080008600A206B
:10A2F000FEF7B3F80A20FEF7B0F807E0601CC4B21E
:10A30000FA2C03DDFFF7BEFF012010BDC8488438DA
:10A3100000680028F2D1C649086000BFF5E710B513
:10A32000C248006820F00F00C04908600846006875
:10A3300040F0030008600020BD49091F08600A20A2
:10A34000FEF78BF80120BB49C1F8A4010A20FEF7F3
:10A3500084F80020B64908600A20FEF77EF810BD98
:10A3600010B5B248006820F00F00B04908600846F8
:10A37000006840F0030008600120AD49091F086033
:10A380000A20FEF76AF80120AA49C1F8A4010A20B0
:10A39000FEF763F80020A64908600A20FEF75DF882
:10A3A00010BD70B50446A148006820F00F009F4919
:10A3B00008600846006840F00300086000251CE0C3
:10A3C00004F0800020B101209949091F086003E0D2
:10A3D00000209749091F08606006040E0A20FEF756
:10A3E0003CF80120924908600A20FEF736F8002068
:10A3F0009049C1F8A401681CC5B2082DE0DB0A2011
:10A40000FEF72BF801208A4908600A20FEF725F89C
:10A4100000208849C1F8A40170BD70B5064600242B
:10A420008248006820F00F008049086008460068F4
:10A4300040F008000860002515E001207C49086014
:10A440000A20FEF70AF86006040E7A48D0F82001C8
:10A4500008B144F001040020754908600A20FDF7A6
:10A46000FCFF681CC5B2082DE7DB7048006820F0CF
:10A470000F006E4908600846006840F0030008605D
:10A48000204670BD2DE9F04107460D461646FFF700
:10A49000D5FE7C20FFF785FF3846FFF782FFFFF7E8
:10A4A000CDFE7D20FFF77DFF002407E00120FFF7B0
:10A4B000B4FF2855FFF733FF601CC4B2701EA042E2
:10A4C000F4DC0020FFF7A9FF2855FFF749FFFFF74D
:10A4D000D9FEBDE8F0812DE9F04107460D4616464C
:10A4E000FFF7ACFE7C20FFF75CFF3846FFF759FF13
:10A4F000002404E0285DFFF754FF601CC4B2B4429E
:10A50000F8DBFFF7BFFEBDE8F0812DE9F04107461B
:10A510000D461646FFF792FE7C20FFF742FF802093
:10A52000FFF73FFF3846FFF73CFF002404E0285DBB
:10A53000FFF737FF601CC4B2B442F8DBFFF7A2FE9E
:10A54000BDE8F081704710B5044623222146002063
:10A55000FFF7DBFF10BD10B5002404E000203649F2
:10A560000855601CC4B2232CF8DB3348FFF7EBFF1F
:10A5700010BD08B50220FDF794FF03208DF8000000
:10A58000012269468220FFF7A6FF08BD10B5012011
:10A590002A490860FFF7EDFFFFF7DDFF10BD70B53A
:10A5A00004460D461646324621462846FFF76AFF06
:10A5B00070BD002004E000211F4A1154411CC8B2A4
:10A5C0002328F8DB704730B5C31700EB5373DB105B
:10A5D000194CE35C0246C41700EB5474E410A0EB82
:10A5E000C4050124AC4023430146C41700EB547456
:10A5F000E410114D2B5530BD30B5C31700EB53732C
:10A60000DB100D4CE35C0246C41700EB5474E410FD
:10A61000A0EBC4050124AC40A3430146C41700EBE2
:10A620005474E410044D2B5530BD0000040C01405F
:10A63000A481214200802142D20F00208C012342BC
:10A6400030B505460C46152D82F08082DFE815F006
:10A650007E121500FF00E801D102BA03A3048C05A5
:10A660008A0673075C0845092E0A170B000C080DB3
:10A67000F10DDA0EC30FAC1095110A2C74D2DFE87D
:10A6800004F0051B31475D748AA0B6CC0F20FFF79C
:10A690009AFF1720FFF797FF1520FFF794FF0C2074
:10A6A000FFF791FF0D20FFF78EFF0E20FFF78BFFC6
:10A6B0001620FFF7A1FFC7E00F20FFF79DFF17202F
:10A6C000FFF781FF1520FFF77EFF0C20FFF794FFB7
:10A6D0000D20FFF791FF0E20FFF78EFF1620FFF7EA
:10A6E0008BFFB1E00F20FFF76EFF1720FFF76BFF26
:10A6F0001520FFF781FF0C20FFF765FF0D20FFF706
:10A7000062FF0E20FFF778FF1620FFF75CFF9BE04B
:10A710000F20FFF758FF1720FFF755FF1520FFF711
:10A7200052FF0C20FFF74FFF0D20FFF765FF0E20B3
:10A73000FFF762FF1620FFF746FF85E00F20FFF7C7
:10A740005BFF1720FFF73FFF1520FFF73CFF0C20B2
:10A75000FFF752FF0D20FFF74FFF0E20FFF733FFEB
:10A760001620FFF730FF6FE06DE00F20FFF72BFFA3
:10A770001720FFF741FF1520FFF725FF0C20FFF7FB
:10A7800022FF0D20FFF738FF0E20FFF71CFF1620D9
:10A79000FFF719FF58E00F20FFF715FF1720FFF70D
:10A7A0002BFF1520FFF70FFF0C20FFF70CFF0D20EC
:10A7B000FFF709FF0E20FFF706FF1620FFF703FF44
:10A7C00042E00F20FFF7FFFE1720FFF7FCFE1520E9
:10A7D000FFF7F9FE0C20FFF70FFF0D20FFF70CFF2E
:10A7E0000E20FFF709FF1620FFF706FF2CE00F20D1
:10A7F000FFF7E9FE1720FFF7E6FE1520FFF7E3FE5F
:10A800000C20FFF7E0FE0D20FFF7DDFE0E20FFF726
:10A81000DAFE1620FFF7D7FE16E00F20FFF7D3FE73
:10A820001720FFF7D0FE1520FFF7CDFE0C20FFF715
:10A83000CAFE0D20FFF7E0FE0E20FFF7C4FE162033
:10A84000FFF7C1FE00E000BF00BF02F07FB90A2C95
:10A8500074D2DFE804F0051B31475D748AA0B6CCE2
:10A860001F20FFF7B0FE3E20FFF7ADFE3D20FFF7B3
:10A87000AAFE1C20FFF7A7FE1420FFF7A4FE1E204F
:10A88000FFF7A1FE1D20FFF7B7FEC7E01F20FFF76F
:10A89000B3FE3E20FFF797FE3D20FFF794FE1C20FD
:10A8A000FFF7AAFE1420FFF7A7FE1E20FFF7A4FE65
:10A8B0001D20FFF7A1FEB1E01F20FFF784FE3E2020
:10A8C000FFF781FE3D20FFF797FE1C20FFF77BFE80
:10A8D0001420FFF778FE1E20FFF78EFE1D20FFF7E5
:10A8E00072FE9BE01F20FFF76EFE3E20FFF76BFE1F
:10A8F0003D20FFF768FE1C20FFF765FE1420FFF7E0
:10A900007BFE1E20FFF778FE1D20FFF75CFE85E032
:10A910001F20FFF771FE3E20FFF755FE3D20FFF799
:10A9200052FE1C20FFF768FE1420FFF765FE1E2074
:10A93000FFF749FE1D20FFF746FE6FE06DE01F2088
:10A94000FFF741FE3E20FFF757FE3D20FFF73BFE9D
:10A950001C20FFF738FE1420FFF74EFE1E20FFF7E5
:10A9600032FE1D20FFF72FFE58E01F20FFF72BFEC1
:10A970003E20FFF741FE3D20FFF725FE1C20FFF79C
:10A9800022FE1420FFF71FFE1E20FFF71CFE1D20D5
:10A99000FFF719FE42E01F20FFF715FE3E20FFF7EC
:10A9A00012FE3D20FFF70FFE1C20FFF725FE1420AE
:10A9B000FFF722FE1E20FFF71FFE1D20FFF71CFEE3
:10A9C0002CE01F20FFF7FFFD3E20FFF7FCFD3D20A0
:10A9D000FFF7F9FD1C20FFF7F6FD1420FFF7F3FD4C
:10A9E0001E20FFF7F0FD1D20FFF7EDFD16E01F20F4
:10A9F000FFF7E9FD3E20FFF7E6FD3D20FFF7E3FD11
:10AA00001C20FFF7E0FD1420FFF7F6FD1E20FFF7E6
:10AA1000DAFD1D20FFF7D7FD00E000BF00BF14E7FF
:10AA20000A2C74D2DFE804F0051B31475D748AA05C
:10AA3000B6CC5F20FFF7C7FD5E20FFF7C4FD5D20A9
:10AA4000FFF7C1FD5C20FFF7BEFD5420FFF7BBFD03
:10AA50005620FFF7B8FD5520FFF7CEFDC7E05F2079
:10AA6000FFF7CAFD5E20FFF7AEFD5D20FFF7ABFDEF
:10AA70005C20FFF7C1FD5420FFF7BEFD5620FFF715
:10AA8000BBFD5520FFF7B8FDB1E05F20FFF79BFD50
:10AA90005E20FFF798FD5D20FFF7AEFD5C20FFF71D
:10AAA00092FD5420FFF78FFD5620FFF7A5FD55209E
:10AAB000FFF789FD9BE05F20FFF785FD5E20FFF734
:10AAC00082FD5D20FFF77FFD5C20FFF77CFD5420B9
:10AAD000FFF792FD5620FFF78FFD5520FFF773FD1E
:10AAE00085E05F20FFF788FD5E20FFF76CFD5D20AD
:10AAF000FFF769FD5C20FFF77FFD5420FFF77CFD29
:10AB00005620FFF760FD5520FFF75DFD6FE06DE01B
:10AB10005F20FFF758FD5E20FFF76EFD5D20FFF719
:10AB200052FD5C20FFF74FFD5420FFF765FD5620D6
:10AB3000FFF749FD5520FFF746FD58E05F20FFF77E
:10AB400042FD5E20FFF758FD5D20FFF73CFD5C20D5
:10AB5000FFF739FD5420FFF736FD5620FFF733FD90
:10AB60005520FFF730FD42E05F20FFF72CFD5E200F
:10AB7000FFF729FD5D20FFF726FD5C20FFF73CFD78
:10AB80005420FFF739FD5620FFF736FD5520FFF71B
:10AB900033FD2CE05F20FFF716FD5E20FFF713FD6D
:10ABA0005D20FFF710FD5C20FFF70DFD5420FFF73F
:10ABB0000AFD5620FFF707FD5520FFF704FD16E0BC
:10ABC0005F20FFF700FD5E20FFF7FDFC5D20FFF733
:10ABD000FAFC5C20FFF7F7FC5420FFF70DFD562030
:10ABE000FFF7F1FC5520FFF7EEFC00E000BF00BFCF
:10ABF0002BE60A2C74D2DFE804F0051B31475D74A4
:10AC00008AA0B6CC5820FFF7DEFC5120FFF7DBFC12
:10AC10005320FFF7D8FC5B20FFF7D5FC5A20FFF745
:10AC2000D2FC5920FFF7CFFC5220FFF7E5FCC7E02C
:10AC30005820FFF7E1FC5120FFF7C5FC5320FFF738
:10AC4000C2FC5B20FFF7D8FC5A20FFF7D5FC592047
:10AC5000FFF7D2FC5220FFF7CFFCB1E05820FFF7FE
:10AC6000B2FC5120FFF7AFFC5320FFF7C5FC5B207F
:10AC7000FFF7A9FC5A20FFF7A6FC5920FFF7BCFC00
:10AC80005220FFF7A0FC9BE05820FFF79CFC5120CE
:10AC9000FFF799FC5320FFF796FC5B20FFF793FC2E
:10ACA0005A20FFF7A9FC5920FFF7A6FC5220FFF716
:10ACB0008AFC85E05820FFF79FFC5120FFF783FCBA
:10ACC0005320FFF780FC5B20FFF796FC5A20FFF72C
:10ACD00093FC5920FFF777FC5220FFF774FC6FE0DC
:10ACE0006DE05820FFF76FFC5120FFF785FC5320E3
:10ACF000FFF769FC5B20FFF766FC5A20FFF77CFC3E
:10AD00005920FFF760FC5220FFF75DFC58E0582007
:10AD1000FFF759FC5120FFF76FFC5320FFF753FC5E
:10AD20005B20FFF750FC5A20FFF74DFC5920FFF73E
:10AD30004AFC5220FFF747FC42E05820FFF743FC53
:10AD40005120FFF740FC5320FFF73DFC5B20FFF74D
:10AD500053FC5A20FFF750FC5920FFF74DFC5220BE
:10AD6000FFF74AFC2CE05820FFF72DFC5120FFF79D
:10AD70002AFC5320FFF727FC5B20FFF724FC5A2016
:10AD8000FFF721FC5920FFF71EFC5220FFF71BFCA8
:10AD900016E05820FFF717FC5120FFF714FC532052
:10ADA000FFF711FC5B20FFF70EFC5A20FFF724FC95
:10ADB0005920FFF708FC5220FFF705FC00E000BF18
:10ADC00000BF42E50A2C74D2DFE804F0051B3147CE
:10ADD0005D748AA0B6CC0B20FFF7F5FB1220FFF7BD
:10ADE000F2FB1020FFF7EFFB0820FFF7ECFB092038
:10ADF000FFF7E9FB0A20FFF7E6FB1120FFF7FCFB5A
:10AE0000C7E00B20FFF7F8FB1220FFF7DCFB102058
:10AE1000FFF7D9FB0820FFF7EFFB0920FFF7ECFB5A
:10AE20000A20FFF7E9FB1120FFF7E6FBB1E00B205A
:10AE3000FFF7C9FB1220FFF7C6FB1020FFF7DCFB72
:10AE40000820FFF7C0FB0920FFF7BDFB0A20FFF732
:10AE5000D3FB1120FFF7B7FB9BE00B20FFF7B3FB01
:10AE60001220FFF7B0FB1020FFF7ADFB0820FFF723
:10AE7000AAFB0920FFF7C0FB0A20FFF7BDFB11204A
:10AE8000FFF7A1FB85E00B20FFF7B6FB1220FFF7D1
:10AE90009AFB1020FFF797FB0820FFF7ADFB092076
:10AEA000FFF7AAFB0A20FFF78EFB1120FFF78BFBB1
:10AEB0006FE06DE00B20FFF786FB1220FFF79CFB95
:10AEC0001020FFF780FB0820FFF77DFB0920FFF72C
:10AED00093FB0A20FFF777FB1120FFF774FB58E084
:10AEE0000B20FFF770FB1220FFF786FB1020FFF707
:10AEF0006AFB0820FFF767FB0920FFF764FB0A20C5
:10AF0000FFF761FB1120FFF75EFB42E00B20FFF72C
:10AF10005AFB1220FFF757FB1020FFF754FB0820C5
:10AF2000FFF76AFB0920FFF767FB0A20FFF764FBC6
:10AF30001120FFF761FB2CE00B20FFF744FB1220F0
:10AF4000FFF741FB1020FFF73EFB0820FFF73BFB1C
:10AF50000920FFF738FB0A20FFF735FB1120FFF728
:10AF600032FB16E00B20FFF72EFB1220FFF72BFB26
:10AF70001020FFF728FB0820FFF725FB0920FFF72B
:10AF80003BFB0A20FFF71FFB1120FFF71CFB00E033
:10AF900000BF00BF59E40A2C74D2DFE804F0051B9F
:10AFA00031475D748AA0B6CC3B20FFF70CFB3A20FA
:10AFB000FFF709FB3920FFF706FB3820FFF703FBFB
:10AFC0001920FFF700FB1B20FFF7FDFA1A20FFF7FF
:10AFD00013FBC7E03B20FFF70FFB3A20FFF7F3FA24
:10AFE0003920FFF7F0FA3820FFF706FB1920FFF7AA
:10AFF00003FB1B20FFF700FB1A20FFF7FDFAB1E06F
:10B000003B20FFF7E0FA3A20FFF7DDFA3920FFF79F
:10B01000F3FA3820FFF7D7FA1920FFF7D4FA1B20EC
:10B02000FFF7EAFA1A20FFF7CEFA9BE03B20FFF782
:10B03000CAFA3A20FFF7C7FA3920FFF7C4FA3820D6
:10B04000FFF7C1FA1920FFF7D7FA1B20FFF7D4FA50
:10B050001A20FFF7B8FA85E03B20FFF7CDFA3A2037
:10B06000FFF7B1FA3920FFF7AEFA3820FFF7C4FA3C
:10B070001920FFF7C1FA1B20FFF7A5FA1A20FFF7E6
:10B08000A2FA6FE06DE03B20FFF79DFA3A20FFF750
:10B09000B3FA3920FFF797FA3820FFF794FA19200E
:10B0A000FFF7AAFA1B20FFF78EFA1A20FFF78BFA98
:10B0B00058E03B20FFF787FA3A20FFF79DFA392046
:10B0C000FFF781FA3820FFF77EFA1920FFF77BFAA5
:10B0D0001B20FFF778FA1A20FFF775FA42E03B20B1
:10B0E000FFF771FA3A20FFF76EFA3920FFF76BFA93
:10B0F0003820FFF781FA1920FFF77EFA1B20FFF7AF
:10B100007BFA1A20FFF778FA2CE03B20FFF75BFA76
:10B110003A20FFF758FA3920FFF755FA3820FFF7A1
:10B1200052FA1920FFF74FFA1B20FFF74CFA1A20AA
:10B13000FFF749FA16E03B20FFF745FA3A20FFF700
:10B1400042FA3920FFF73FFA3820FFF73CFA19207E
:10B15000FFF752FA1B20FFF736FA1A20FFF733FAEF
:10B1600000E000BF00BF5AE40A2C7CD2DFE804F004
:10B17000051D354D657F97AFC7DFFB20FFF723FA2D
:10B18000F320FFF720FAF920FFF71DFAF820FFF768
:10B190001AFA40F20110FFF716FA40F20310FFF717
:10B1A00012FAFA20FFF728FADAE0FB20FFF724FA78
:10B1B000F320FFF708FAF920FFF705FAF820FFF768
:10B1C0001BFA40F20110FFF717FA40F20310FFF7E5
:10B1D00013FAFA20FFF710FAC2E0FB20FFF7F3F9A9
:10B1E000F320FFF7F0F9F920FFF706FAF820FFF750
:10B1F000EAF940F20110FFF7E6F940F20310FFF719
:10B20000FBF9FA20FFF7DFF9AAE0FB20FFF7DBF9F3
:10B21000F320FFF7D8F9F920FFF7D5F9F820FFF769
:10B22000D2F940F20110FFF7E7F940F20310FFF7FF
:10B23000E3F9FA20FFF7C7F992E0FB20FFF7DCF90A
:10B24000F320FFF7C0F9F920FFF7BDF9F820FFF769
:10B25000D3F940F20110FFF7CFF940F20310FFF7E6
:10B26000B2F9FA2000E07AE0FFF7ADF978E0FB20D0
:10B27000FFF7A9F9F320FFF7BFF9F920FFF7A3F9CA
:10B28000F820FFF7A0F940F20110FFF7B5F940F2FE
:10B290000310FFF798F9FA20FFF795F960E0FB201B
:10B2A000FFF791F9F320FFF7A7F9F920FFF78BF9E2
:10B2B000F820FFF788F940F20110FFF784F940F217
:10B2C0000310FFF780F9FA20FFF77DF948E0FB2033
:10B2D000FFF779F9F320FFF776F9F920FFF773F913
:10B2E000F820FFF789F940F20110FFF785F940F2E5
:10B2F0000310FFF781F9FA20FFF77EF930E0FB2019
:10B30000FFF761F9F320FFF75EF9F920FFF75BF92A
:10B31000F820FFF758F940F20110FFF754F940F216
:10B320000310FFF750F9FA20FFF74DF918E0FB2062
:10B33000FFF749F9F320FFF746F9F920FFF743F942
:10B34000F820FFF740F940F20110FFF755F940F2FD
:10B350000310FFF738F9FA20FFF735F900E000BFD6
:10B3600000BF45E40A2C74D2DFE804F0051B314726
:10B370005D748AA0B6CCEB20FFF725F9E220FFF739
:10B3800022F9E120FFF71FF9E820FFF71CF9F1206F
:10B39000FFF719F9EA20FFF716F9E920FFF72CF972
:10B3A000C7E0EB20FFF728F9E220FFF70CF9E120D6
:10B3B000FFF709F9E820FFF71FF9F120FFF71CF963
:10B3C000EA20FFF719F9E920FFF716F9B1E0EB20C1
:10B3D000FFF7F9F8E220FFF7F6F8E120FFF70CF9A4
:10B3E000E820FFF7F0F8F120FFF7EDF8EA20FFF78B
:10B3F00003F9E920FFF7E7F89BE0EB20FFF7E3F81C
:10B40000E220FFF7E0F8E120FFF7DDF8E820FFF7A2
:10B41000DAF8F120FFF7F0F8EA20FFF7EDF8E9207D
:10B42000FFF7D1F885E0EB20FFF7E6F8E220FFF721
:10B43000CAF8E120FFF7C7F8E820FFF7DDF8F120B0
:10B44000FFF7DAF8EA20FFF7BEF8E920FFF7BBF8CC
:10B450006FE06DE0EB20FFF7B6F8E220FFF7CCF8E5
:10B46000E120FFF7B0F8E820FFF7ADF8F120FFF793
:10B47000C3F8EA20FFF7A7F8E920FFF7A4F858E09F
:10B48000EB20FFF7A0F8E220FFF7B6F8E120FFF786
:10B490009AF8E820FFF797F8F120FFF794F8EA20F0
:10B4A000FFF791F8E920FFF78EF842E0EB20FFF775
:10B4B0008AF8E220FFF787F8E120FFF784F8E82018
:10B4C000FFF79AF8F120FFF797F8EA20FFF794F8D2
:10B4D000E920FFF791F82CE0EB20FFF774F8E22069
:10B4E000FFF771F8E120FFF76EF8E820FFF76BF83F
:10B4F000F120FFF768F8EA20FFF765F8E920FFF789
:10B5000062F816E0EB20FFF75EF8E220FFF75BF849
:10B51000E120FFF758F8E820FFF755F8F120FFF792
:10B520006BF8EA20FFF74FF8E920FFF74CF800E04E
:10B5300000BF00BF45E40A2C74D2DFE804F0051B0D
:10B5400031475D748AA0B6CCDB20FFF73CF8D220EF
:10B55000FFF739F8D020FFF736F8D820FFF733F897
:10B56000D920FFF730F8DA20FFF72DF8D120FFF7C8
:10B5700043F8C7E0DB20FFF73FF8D220FFF723F8BE
:10B58000D020FFF720F8D820FFF736F8D920FFF7B2
:10B5900033F8DA20FFF730F8D120FFF72DF8B1E0CB
:10B5A000DB20FFF710F8D220FFF70DF8D020FFF7CF
:10B5B00023F8D820FFF707F8D920FFF704F8DA209E
:10B5C000FFF71AF8D120FEF7FEFF9BE0DB20FEF725
:10B5D000FAFFD220FEF7F7FFD020FEF7F4FFD820C5
:10B5E000FEF7F1FFD920FFF707F8DA20FFF704F89C
:10B5F000D120FEF7E8FF85E0DB20FEF7FDFFD2203B
:10B60000FEF7E1FFD020FEF7DEFFD820FEF7F4FFC3
:10B61000D920FEF7F1FFDA20FEF7D5FFD120FEF7A3
:10B62000D2FF6FE06DE0DB20FEF7CDFFD220FEF70A
:10B63000E3FFD020FEF7C7FFD820FEF7C4FFD920D4
:10B64000FEF7DAFFDA20FEF7BEFFD120FEF7BBFFE0
:10B6500058E0DB20FEF7B7FFD220FEF7CDFFD02069
:10B66000FEF7B1FFD820FEF7AEFFD920FEF7ABFF03
:10B67000DA20FEF7A8FFD120FEF7A5FF42E0DB208D
:10B68000FEF7A1FFD220FEF79EFFD020FEF79BFF22
:10B69000D820FEF7B1FFD920FEF7AEFFDA20FEF783
:10B6A000ABFFD120FEF7A8FF2CE0DB20FEF78BFFDD
:10B6B000D220FEF788FFD020FEF785FFD820FEF7C6
:10B6C00082FFD920FEF77FFFDA20FEF77CFFD12032
:10B6D000FEF779FF16E0DB20FEF775FFD220FEF7BC
:10B6E00072FFD020FEF76FFFD820FEF76CFFD92045
:10B6F000FEF782FFDA20FEF766FFD120FEF763FF38
:10B7000000E000BF00BF45E40A2C74D2DFE804F07B
:10B71000051B31475D748AA0B6CCC320FEF753FFEA
:10B72000C220FEF750FFC120FEF74DFFC020FEF7FC
:10B730004AFFC920FEF747FFCB20FEF744FFCA208F
:10B74000FEF75AFFC7E0C320FEF756FFC220FEF700
:10B750003AFFC120FEF737FFC020FEF74DFFC9209A
:10B76000FEF74AFFCB20FEF747FFCA20FEF744FF53
:10B77000B1E0C320FEF727FFC220FEF724FFC1205F
:10B78000FEF73AFFC020FEF71EFFC920FEF71BFFA1
:10B79000CB20FEF731FFCA20FEF715FF9BE0C32048
:10B7A000FEF711FFC220FEF70EFFC120FEF70BFFD0
:10B7B000C020FEF708FFC920FEF71EFFCB20FEF7D2
:10B7C0001BFFCA20FEF7FFFE85E0C320FEF714FF33
:10B7D000C220FEF7F8FEC120FEF7F5FEC020FEF7FE
:10B7E0000BFFC920FEF708FFCB20FEF7ECFECA20B6
:10B7F000FEF7E9FE6FE06DE0C320FEF7E4FEC22035
:10B80000FEF7FAFEC120FEF7DEFEC020FEF7DBFEEB
:10B81000C920FEF7F1FECB20FEF7D5FECA20FEF7C9
:10B82000D2FE58E0C320FEF7CEFEC220FEF7E4FEB3
:10B83000C120FEF7C8FEC020FEF7C5FEC920FEF7F6
:10B84000C2FECB20FEF7BFFECA20FEF7BCFE42E0E0
:10B85000C320FEF7B8FEC220FEF7B5FEC120FEF7FA
:10B86000B2FEC020FEF7C8FEC920FEF7C5FECB2001
:10B87000FEF7C2FECA20FEF7BFFE2CE0C320FEF793
:10B88000A2FEC220FEF79FFEC120FEF79CFEC02054
:10B89000FEF799FEC920FEF796FECB20FEF793FE39
:10B8A000CA20FEF790FE16E0C320FEF78CFEC220F1
:10B8B000FEF789FEC120FEF786FEC020FEF783FE5C
:10B8C000C920FEF799FECB20FEF77DFECA20FEF7C9
:10B8D0007AFE00E000BF00BF45E40A2C74D2DFE826
:10B8E00004F0051B31475D748AA0B6CCB320FEF787
:10B8F0006AFEAB20FEF767FEB120FEF764FEB020C3
:10B90000FEF761FEB920FEF75EFEBB20FEF75BFE90
:10B91000B220FEF771FEC7E0B320FEF76DFEAB204C
:10B92000FEF751FEB120FEF74EFEB020FEF764FE9A
:10B93000B920FEF761FEBB20FEF75EFEB220FEF7E7
:10B940005BFEB1E0B320FEF73EFEAB20FEF73BFE10
:10B95000B120FEF751FEB020FEF735FEB920FEF70C
:10B9600032FEBB20FEF748FEB220FEF72CFE9BE025
:10B97000B320FEF728FEAB20FEF725FEB120FEF730
:10B9800022FEB020FEF71FFEB920FEF735FEBB20D9
:10B99000FEF732FEB220FEF716FE85E0B320FEF77A
:10B9A0002BFEAB20FEF70FFEB120FEF70CFEB02001
:10B9B000FEF722FEB920FEF71FFEBB20FEF703FEB6
:10B9C000B220FEF700FE6FE06DE0B320FEF7FBFD56
:10B9D000AB20FEF711FEB120FEF7F5FDB020FEF71B
:10B9E000F2FDB920FEF708FEBB20FEF7ECFDB22009
:10B9F000FEF7E9FD58E0B320FEF7E5FDAB20FEF7CA
:10BA0000FBFDB120FEF7DFFDB020FEF7DCFDB92025
:10BA1000FEF7D9FDBB20FEF7D6FDB220FEF7D3FD21
:10BA200042E0B320FEF7CFFDAB20FEF7CCFDB12006
:10BA3000FEF7C9FDB020FEF7DFFDB920FEF7DCFD03
:10BA4000BB20FEF7D9FDB220FEF7D6FD2CE0B320D7
:10BA5000FEF7B9FDAB20FEF7B6FDB120FEF7B3FD52
:10BA6000B020FEF7B0FDB920FEF7ADFDBB20FEF71C
:10BA7000AAFDB220FEF7A7FD16E0B320FEF7A3FD56
:10BA8000AB20FEF7A0FDB120FEF79DFDB020FEF734
:10BA90009AFDB920FEF7B0FDBB20FEF794FDB22061
:10BAA000FEF791FD00E000BF00BF5AE40A2C74D2FB
:10BAB000DFE804F0051B31475D748AA0B6CCA320F3
:10BAC000FEF781FD9A20FEF77EFD9920FEF77BFDB3
:10BAD000A020FEF778FDA920FEF775FDA220FEF755
:10BAE00072FDA120FEF788FDC7E0A320FEF784FDCC
:10BAF0009A20FEF768FD9920FEF765FDA020FEF76D
:10BB00007BFDA920FEF778FDA220FEF775FDA120A0
:10BB1000FEF772FDB1E0A320FEF755FD9A20FEF777
:10BB200052FD9920FEF768FDA020FEF74CFDA920EC
:10BB3000FEF749FDA220FEF75FFDA120FEF743FDC1
:10BB40009BE0A320FEF73FFD9A20FEF73CFD9920E5
:10BB5000FEF739FDA020FEF736FDA920FEF74CFDCB
:10BB6000A220FEF749FDA120FEF72DFD85E0A320D0
:10BB7000FEF742FD9A20FEF726FD9920FEF723FDF1
:10BB8000A020FEF739FDA920FEF736FDA220FEF722
:10BB90001AFDA120FEF717FD6FE06DE0A320FEF770
:10BBA00012FD9A20FEF728FD9920FEF70CFDA0203B
:10BBB000FEF709FDA920FEF71FFDA220FEF703FDF9
:10BBC000A120FEF700FD58E0A320FEF7FCFC9A2020
:10BBD000FEF712FD9920FEF7F6FCA020FEF7F3FC1D
:10BBE000A920FEF7F0FCA220FEF7EDFCA120FEF755
:10BBF000EAFC42E0A320FEF7E6FC9A20FEF7E3FC15
:10BC00009920FEF7E0FCA020FEF7F6FCA920FEF745
:10BC1000F3FCA220FEF7F0FCA120FEF7EDFC2CE0E7
:10BC2000A320FEF7D0FC9A20FEF7CDFC9920FEF76A
:10BC3000CAFCA020FEF7C7FCA920FEF7C4FCA22086
:10BC4000FEF7C1FCA120FEF7BEFC16E0A320FEF724
:10BC5000BAFC9A20FEF7B7FC9920FEF7B4FCA020AE
:10BC6000FEF7B1FCA920FEF7C7FCA220FEF7ABFC53
:10BC7000A120FEF7A8FC00E000BF00BF5AE40A2C98
:10BC800074D2DFE804F0051B31475D748AA0B6CC9E
:10BC90009320FEF798FC8A20FEF795FC8820FEF79B
:10BCA00092FC9020FEF78FFC9120FEF78CFC9220F6
:10BCB000FEF789FC8920FEF79FFCC7E09320FEF782
:10BCC0009BFC8A20FEF77FFC8820FEF77CFC9020FE
:10BCD000FEF792FC9120FEF78FFC9220FEF78CFC81
:10BCE0008920FEF789FCB1E09320FEF76CFC8A20E6
:10BCF000FEF769FC8820FEF77FFC9020FEF763FCCE
:10BD00009120FEF760FC9220FEF776FC8920FEF77A
:10BD10005AFC9BE09320FEF756FC8A20FEF753FC6A
:10BD20008820FEF750FC9020FEF74DFC9120FEF796
:10BD300063FC9220FEF760FC8920FEF744FC85E05E
:10BD40009320FEF759FC8A20FEF73DFC8820FEF781
:10BD50003AFC9020FEF750FC9120FEF74DFC92201B
:10BD6000FEF731FC8920FEF72EFC6FE06DE093209A
:10BD7000FEF729FC8A20FEF73FFC8820FEF723FC13
:10BD80009020FEF720FC9120FEF736FC9220FEF773
:10BD90001AFC8920FEF717FC58E09320FEF713FCED
:10BDA0008A20FEF729FC8820FEF70DFC9020FEF784
:10BDB0000AFC9120FEF707FC9220FEF704FC892084
:10BDC000FEF701FC42E09320FEF7FDFB8A20FEF720
:10BDD000FAFB8820FEF7F7FB9020FEF70DFC912080
:10BDE000FEF70AFC9220FEF707FC8920FEF704FC10
:10BDF0002CE09320FEF7E7FB8A20FEF7E4FB882087
:10BE0000FEF7E1FB9020FEF7DEFB9120FEF7DBFB67
:10BE10009220FEF7D8FB8920FEF7D5FB16E0932091
:10BE2000FEF7D1FB8A20FEF7CEFB8820FEF7CBFB86
:10BE30009020FEF7C8FB9120FEF7DEFB9220FEF774
:10BE4000C2FB8920FEF7BFFB00E000BF00BF5AE441
:10BE50000A2C7DD2DFE804F0051E375069849DB6B8
:10BE6000CFE8FC20FEF7AFFBFD20FEF7ACFBFE2089
:10BE7000FEF7A9FBFF20FEF7A6FB40F20710FEF736
:10BE8000A2FB40F20510FEF79EFB4FF48370FEF715
:10BE9000B3FBE3E0FC20FEF7AFFBFD20FEF793FBD6
:10BEA000FE20FEF790FBFF20FEF7A6FB40F20710F6
:10BEB000FEF7A2FB40F20510FEF79EFB4FF48370E5
:10BEC000FEF79AFBCAE0FC20FEF77DFBFD20FEF7A3
:10BED0007AFBFE20FEF790FBFF20FEF774FB40F29A
:10BEE0000710FEF770FB40F20510FEF785FB4FF4DC
:10BEF0008370FEF768FBB1E0FC20FEF764FBFD20D9
:10BF0000FEF761FBFE20FEF75EFBFF20FEF75BFB0A
:10BF100040F20710FEF770FB40F20510FEF76CFBD5
:10BF20004FF48370FEF74FFB98E0FC20FEF764FBB4
:10BF3000FD20FEF748FBFE20FEF745FBFF20FEF745
:10BF40005BFB40F20710FEF757FB40F2051000E0E4
:10BF500083E0FEF738FB4FF48370FEF734FB7DE09F
:10BF6000FC20FEF730FBFD20FEF746FBFE20FEF72F
:10BF70002AFBFF20FEF727FB40F20710FEF73CFBF1
:10BF800040F20510FEF71FFB4FF48370FEF71BFB1A
:10BF900064E0FC20FEF717FBFD20FEF72DFBFE20E2
:10BFA000FEF711FBFF20FEF70EFB40F20710FEF735
:10BFB0000AFB40F20510FEF706FB4FF48370FEF714
:10BFC00002FB4BE0FC20FEF7FEFAFD20FEF7FBFA39
:10BFD000FE20FEF7F8FAFF20FEF70EFB40F20710F6
:10BFE000FEF70AFB40F20510FEF706FB4FF48370E4
:10BFF000FEF702FB32E0FC20FEF7E5FAFD20FEF73B
:10C00000E2FAFE20FEF7DFFAFF20FEF7DCFA40F24C
:10C010000710FEF7D8FA40F20510FEF7D4FA4FF4F5
:10C020008370FEF7D0FA19E0FC20FEF7CCFAFD2071
:10C03000FEF7C9FAFE20FEF7C6FAFF20FEF7C3FAA4
:10C0400040F20710FEF7D8FA40F20510FEF7BBFAEF
:10C050004FF48370FEF7B7FA00E000BF00BF3BE487
:10C060000A2C74D2DFE804F0051B31475D748AA006
:10C07000B6CCEC20FEF7A7FAE420FEF7A4FAEE20F7
:10C08000FEF7A1FAEF20FEF79EFAF620FEF79BFAE4
:10C09000F420FEF798FAED20FEF7AEFAC7E0EC20A8
:10C0A000FEF7AAFAE420FEF78EFAEE20FEF78BFAEE
:10C0B000EF20FEF7A1FAF620FEF79EFAF420FEF735
:10C0C0009BFAED20FEF798FAB1E0EC20FEF77BFA40
:10C0D000E420FEF778FAEE20FEF78EFAEF20FEF766
:10C0E00072FAF620FEF76FFAF420FEF785FAED20DB
:10C0F000FEF769FA9BE0EC20FEF765FAE420FEF714
:10C1000062FAEE20FEF75FFAEF20FEF75CFAF62007
:10C11000FEF772FAF420FEF76FFAED20FEF753FAFD
:10C1200085E0EC20FEF768FAE420FEF74CFAEE20FA
:10C13000FEF749FAEF20FEF75FFAF620FEF75CFA09
:10C14000F420FEF740FAED20FEF73DFA6FE06DE0D7
:10C15000EC20FEF738FAE420FEF74EFAEE20FEF768
:10C1600032FAEF20FEF72FFAF620FEF745FAF42018
:10C17000FEF729FAED20FEF726FA58E0EC20FEF74C
:10C1800022FAE420FEF738FAEE20FEF71CFAEF2040
:10C19000FEF719FAF620FEF716FAF420FEF713FA66
:10C1A000ED20FEF710FA42E0EC20FEF70CFAE42056
:10C1B000FEF709FAEE20FEF706FAEF20FEF71CFA6A
:10C1C000F620FEF719FAF420FEF716FAED20FEF736
:10C1D00013FA2CE0EC20FEF7F6F9E420FEF7F3F971
:10C1E000EE20FEF7F0F9EF20FEF7EDF9F620FEF76E
:10C1F000EAF9F420FEF7E7F9ED20FEF7E4F916E09E
:10C20000EC20FEF7E0F9E420FEF7DDF9EE20FEF782
:10C21000DAF9EF20FEF7D7F9F620FEF7EDF9F42072
:10C22000FEF7D1F9ED20FEF7CEF900E000BF00BF28
:10C230003BE40A2C74D2DFE804F0051B31475D743F
:10C240008AA0B6CCDC20FEF7BEF9D520FEF7BBF9FC
:10C25000D620FEF7B8F9DF20FEF7B5F9E620FEF7A5
:10C26000B2F9DD20FEF7AFF9DE20FEF7C5F9C7E031
:10C27000DC20FEF7C1F9D520FEF7A5F9D620FEF7A0
:10C28000A2F9DF20FEF7B8F9E620FEF7B5F9DD20C8
:10C29000FEF7B2F9DE20FEF7AFF9B1E0DC20FEF7E1
:10C2A00092F9D520FEF78FF9D620FEF7A5F9DF2009
:10C2B000FEF789F9E620FEF786F9DD20FEF79CF906
:10C2C000DE20FEF780F99BE0DC20FEF77CF9D5202C
:10C2D000FEF779F9D620FEF776F9DF20FEF773F93D
:10C2E000E620FEF789F9DD20FEF786F9DE20FEF76D
:10C2F0006AF985E0DC20FEF77FF9D520FEF763F9C7
:10C30000D620FEF760F9DF20FEF776F9E620FEF78B
:10C3100073F9DD20FEF757F9DE20FEF754F96FE0E0
:10C320006DE0DC20FEF74FF9D520FEF765F9D62049
:10C33000FEF749F9DF20FEF746F9E620FEF75CF943
:10C34000DD20FEF740F9DE20FEF73DF958E0DC2065
:10C35000FEF739F9D520FEF74FF9D620FEF733F96D
:10C36000DF20FEF730F9E620FEF72DF9DD20FEF79D
:10C370002AF9DE20FEF727F942E0DC20FEF723F958
:10C38000D520FEF720F9D620FEF71DF9DF20FEF7B5
:10C3900033F9E620FEF730F9DD20FEF72DF9DE2037
:10C3A000FEF72AF92CE0DC20FEF70DF9D520FEF788
:10C3B0000AF9D620FEF707F9DF20FEF704F9E62098
:10C3C000FEF701F9DD20FEF7FEF8DE20FEF7FBF8B0
:10C3D00016E0DC20FEF7F7F8D520FEF7F4F8D620BB
:10C3E000FEF7F1F8DF20FEF7EEF8E620FEF704F99D
:10C3F000DD20FEF7E8F8DE20FEF7E5F800E000BFFC
:10C4000000BFA3E30A2C74D2DFE804F0051B314718
:10C410005D748AA0B6CCCC20FEF7D5F8C520FEF717
:10C42000D2F8C720FEF7CFF8CF20FEF7CCF8CE2009
:10C43000FEF7C9F8CD20FEF7C6F8C620FEF7DCF8F7
:10C44000C7E0CC20FEF7D8F8C520FEF7BCF8C7201F
:10C45000FEF7B9F8CF20FEF7CFF8CE20FEF7CCF8E4
:10C46000CD20FEF7C9F8C620FEF7C6F8B1E0CC2013
:10C47000FEF7A9F8C520FEF7A6F8C720FEF7BCF81E
:10C48000CF20FEF7A0F8CE20FEF79DF8CD20FEF7D6
:10C49000B3F8C620FEF797F89BE0CC20FEF793F8A0
:10C4A000C520FEF790F8C720FEF78DF8CF20FEF7E5
:10C4B0008AF8CE20FEF7A0F8CD20FEF79DF8C62022
:10C4C000FEF781F885E0CC20FEF796F8C520FEF750
:10C4D0007AF8C720FEF777F8CF20FEF78DF8CE2048
:10C4E000FEF78AF8CD20FEF76EF8C620FEF76BF84F
:10C4F0006FE06DE0CC20FEF766F8C520FEF77CF813
:10C50000C720FEF760F8CF20FEF75DF8CE20FEF7DB
:10C5100073F8CD20FEF757F8C620FEF754F858E020
:10C52000CC20FEF750F8C520FEF766F8C720FEF7CE
:10C530004AF8CF20FEF747F8CE20FEF744F8CD208A
:10C54000FEF741F8C620FEF73EF842E0CC20FEF7A9
:10C550003AF8C520FEF737F8C720FEF734F8CF20A9
:10C56000FEF74AF8CE20FEF747F8CD20FEF744F854
:10C57000C620FEF741F82CE0CC20FEF724F8C520B9
:10C58000FEF721F8C720FEF71EF8CF20FEF71BF8B4
:10C59000CE20FEF718F8CD20FEF715F8C620FEF7DE
:10C5A00012F816E0CC20FEF70EF8C520FEF70BF8C7
:10C5B000C720FEF708F8CF20FEF705F8CE20FEF7DB
:10C5C0001BF8CD20FDF7FFFFC620FDF7FCFF00E0C4
:10C5D00000BF00BFBAE20A2C74D2DFE804F0051BEA
:10C5E00031475D748AA0B6CCB420FDF7ECFFB520CE
:10C5F000FDF7E9FFB620FDF7E6FFB720FDF7E3FF03
:10C60000BE20FDF7E0FFBC20FDF7DDFFBD20FDF7FC
:10C61000F3FFC7E0B420FDF7EFFFB520FDF7D3FF30
:10C62000B620FDF7D0FFB720FDF7E6FFBE20FDF7EF
:10C63000E3FFBC20FDF7E0FFBD20FDF7DDFFB1E02B
:10C64000B420FDF7C0FFB520FDF7BDFFB620FDF714
:10C65000D3FFB720FDF7B7FFBE20FDF7B4FFBC2026
:10C66000FDF7CAFFBD20FDF7AEFF9BE0B420FDF74C
:10C67000AAFFB520FDF7A7FFB620FDF7A4FFB7205E
:10C68000FDF7A1FFBE20FDF7B7FFBC20FDF7B4FF0B
:10C69000BD20FDF798FF85E0B420FDF7ADFFB52084
:10C6A000FDF791FFB620FDF78EFFB720FDF7A4FF41
:10C6B000BE20FDF7A1FFBC20FDF785FFBD20FDF7E3
:10C6C00082FF6FE06DE0B420FDF77DFFB520FDF740
:10C6D00093FFB620FDF777FFB720FDF774FFBE206C
:10C6E000FDF78AFFBC20FDF76EFFBD20FDF76BFF55
:10C6F00058E0B420FDF767FFB520FDF77DFFB620B9
:10C70000FDF761FFB720FDF75EFFBE20FDF75BFF81
:10C71000BC20FDF758FFBD20FDF755FF42E0B420D7
:10C72000FDF751FFB520FDF74EFFB620FDF74BFF9B
:10C73000B720FDF761FFBE20FDF75EFFBC20FDF7CF
:10C740005BFFBD20FDF758FF2CE0B420FDF73BFF59
:10C75000B520FDF738FFB620FDF735FFB720FDF710
:10C7600032FFBE20FDF72FFFBC20FDF72CFFBD20C0
:10C77000FDF729FF16E0B420FDF725FFB520FDF7F2
:10C7800022FFB620FDF71FFFB720FDF71CFFBE20DC
:10C79000FDF732FFBC20FDF716FFBD20FDF713FFAC
:10C7A00000E000BF00BFD1E10A2C74D2DFE804F042
:10C7B000051B31475D748AA0B6CCA420FDF703FFAA
:10C7C0009C20FDF700FFA620FDF7FDFEA720FDF74A
:10C7D000FAFEAE20FDF7F7FEAC20FDF7F4FEA52033
:10C7E000FDF70AFFC7E0A420FDF706FF9C20FDF738
:10C7F000EAFEA620FDF7E7FEA720FDF7FDFEAE202E
:10C80000FDF7FAFEAC20FDF7F7FEA520FDF7F4FEDC
:10C81000B1E0A420FDF7D7FE9C20FDF7D4FEA620B2
:10C82000FDF7EAFEA720FDF7CEFEAE20FDF7CBFE1A
:10C83000AC20FDF7E1FEA520FDF7C5FE9BE0A4209E
:10C84000FDF7C1FE9C20FDF7BEFEA620FDF7BBFE56
:10C85000A720FDF7B8FEAE20FDF7CEFEAC20FDF719
:10C86000CBFEA520FDF7AFFE85E0A420FDF7C4FEBA
:10C870009C20FDF7A8FEA620FDF7A5FEA720FDF74A
:10C88000BBFEAE20FDF7B8FEAC20FDF79CFEA52058
:10C89000FDF799FE6FE06DE0A420FDF794FE9C206B
:10C8A000FDF7AAFEA620FDF78EFEA720FDF78BFE62
:10C8B000AE20FDF7A1FEAC20FDF785FEA520FDF71B
:10C8C00082FE58E0A420FDF77EFE9C20FDF794FE3A
:10C8D000A620FDF778FEA720FDF775FEAE20FDF738
:10C8E00072FEAC20FDF76FFEA520FDF76CFE42E066
:10C8F000A420FDF768FE9C20FDF765FEA620FDF74D
:10C9000062FEA720FDF778FEAE20FDF775FEAC2095
:10C91000FDF772FEA520FDF76FFE2CE0A420FDF7C9
:10C9200052FE9C20FDF74FFEA620FDF74CFEA720EF
:10C93000FDF749FEAE20FDF746FEAC20FDF743FEB5
:10C94000A520FDF740FE16E0A420FDF73CFE9C204C
:10C95000FDF739FEA620FDF736FEA720FDF733FED2
:10C96000AE20FDF749FEAC20FDF72DFEA520FDF71A
:10C970002AFE00E000BF00BFE8E00A2C74D2DFE826
:10C9800004F0051B31475D748AA0B6CC9420FDF7F6
:10C990001AFE8D20FDF717FE8F20FDF714FE97205D
:10C9A000FDF711FE9E20FDF70EFE9520FDF70BFE14
:10C9B0009620FDF721FEC7E09420FDF71DFE8D2097
:10C9C000FDF701FE8F20FDF7FEFD9720FDF714FE19
:10C9D0009E20FDF711FE9520FDF70EFE9620FDF737
:10C9E0000BFEB1E09420FDF7EEFD8D20FDF7EBFD91
:10C9F0008F20FDF701FE9720FDF7E5FD9E20FDF756
:10CA0000E2FD9520FDF7F8FD9620FDF7DCFD9BE0AB
:10CA10009420FDF7D8FD8D20FDF7D5FD8F20FDF783
:10CA2000D2FD9720FDF7CFFD9E20FDF7E5FD952077
:10CA3000FDF7E2FD9620FDF7C6FD85E09420FDF7A9
:10CA4000DBFD8D20FDF7BFFD8F20FDF7BCFD97209E
:10CA5000FDF7D2FD9E20FDF7CFFD9520FDF7B3FD3C
:10CA60009620FDF7B0FD6FE06DE09420FDF7ABFD83
:10CA70008D20FDF7C1FD8F20FDF7A5FD9720FDF767
:10CA8000A2FD9E20FDF7B8FD9520FDF79CFD9620A8
:10CA9000FDF799FD58E09420FDF795FD8D20FDF7F9
:10CAA000ABFD8F20FDF78FFD9720FDF78CFD9E20BD
:10CAB000FDF789FD9520FDF786FD9620FDF783FDA6
:10CAC00042E09420FDF77FFD8D20FDF77CFD8F2057
:10CAD000FDF779FD9720FDF78FFD9E20FDF78CFD7A
:10CAE0009520FDF789FD9620FDF786FD2CE094202A
:10CAF000FDF769FD8D20FDF766FD8F20FDF763FDD5
:10CB00009720FDF760FD9E20FDF75DFD9520FDF768
:10CB10005AFD9620FDF757FD16E09420FDF753FDD2
:10CB20008D20FDF750FD8F20FDF74DFD9720FDF77F
:10CB30004AFD9E20FDF760FD9520FDF744FD9620FF
:10CB4000FDF741FD00E000BF00BF00BF00BF30BDEA
:10CB500010B50446152C7AD2DFE804F0790B2137A2
:10CB60004D637A90A8BED4F4F2F1F0EFEEEDECEB69
:10CB7000EA000F20FDF740FD1720FDF73DFD1520D1
:10CB8000FDF73AFD0C20FDF737FD0D20FDF734FDD4
:10CB90000E20FDF731FD1620FDF72EFDB2E11F201E
:10CBA000FDF72AFD3E20FDF727FD3D20FDF724FD82
:10CBB0001C20FDF721FD1420FDF71EFD1E20FDF7B2
:10CBC0001BFD1D20FDF718FD9CE15F20FDF714FD06
:10CBD0005E20FDF711FD5D20FDF70EFD5C20FDF7E9
:10CBE0000BFD5420FDF708FD5620FDF705FD5520EF
:10CBF000FDF702FD86E15820FDF7FEFC5120FDF710
:10CC0000FBFC5320FDF7F8FC5B20FDF7F5FC5A20F8
:10CC1000FDF7F2FC5920FDF7EFFC5220FDF7ECFC8C
:10CC200070E10B20FDF7E8FC1220FDF7E5FC102079
:10CC3000FDF7E2FC0820FDF7DFFC0920FDF7DCFC36
:10CC40000A20FDF7D9FC1120FDF7D6FC5AE158E186
:10CC50003B20FDF7D1FC3A20FDF7CEFC3920FDF753
:10CC6000CBFC3820FDF7C8FC1920FDF7C5FC1B20C4
:10CC7000FDF7C2FC1A20FDF7BFFC43E1FB20FDF7E6
:10CC8000BBFCF320FDF7B8FCF920FDF7B5FCF8205C
:10CC9000FDF7B2FC40F20110FDF7AEFC40F20310CC
:10CCA000FDF7AAFCFA20FDF7A7FC2BE1EB20FDF72E
:10CCB000A3FCE220FDF7A0FCE120FDF79DFCE820AD
:10CCC000FDF79AFCF120FDF797FCEA20FDF794FCB4
:10CCD000E920FDF791FC15E1DB20FDF78DFCD2206A
:10CCE000FDF78AFCD020FDF787FCD820FDF784FCF7
:10CCF000D920FDF781FCDA20FDF77EFCD120FDF77D
:10CD00007BFCFFE0C320FDF777FCC220FDF774FC3D
:10CD1000C120FDF771FCC020FDF76EFCC920FDF7B6
:10CD20006BFCCB20FDF768FCCA20FDF765FCE9E051
:10CD3000D1E0BAE0A3E08CE075E05EE044E02DE0F5
:10CD400016E0FFE7B320FDF757FCAB20FDF754FCDE
:10CD5000B120FDF751FCB020FDF74EFCB920FDF7E6
:10CD60004BFCBB20FDF748FCB220FDF745FCC9E0B9
:10CD7000A320FDF741FC9A20FDF73EFC9920FDF72A
:10CD80003BFCA020FDF738FCA920FDF735FCA220D4
:10CD9000FDF732FCA120FDF72FFCB3E09320FDF757
:10CDA0002BFC8A20FDF728FC8820FDF725FC90202D
:10CDB000FDF722FC9120FDF71FFC9220FDF71CFCE3
:10CDC0008920FDF719FC9DE0FC20FDF715FCFD20F6
:10CDD000FDF712FCFE20FDF70FFCFF20FDF70CFC19
:10CDE00040F20710FDF708FC40F20510FDF704FCC7
:10CDF0004FF48370FDF700FC84E0EC20FDF7FCFBB2
:10CE0000E420FDF7F9FBEE20FDF7F6FBEF20FDF740
:10CE1000F3FBF620FDF7F0FBF420FDF7EDFBED2032
:10CE2000FDF7EAFB6EE0DC20FDF7E6FBD520FDF721
:10CE3000E3FBD620FDF7E0FBDF20FDF7DDFBE6207E
:10CE4000FDF7DAFBDD20FDF7D7FBDE20FDF7D4FB95
:10CE500058E0CC20FDF7D0FBC520FDF7CDFBC72067
:10CE6000FDF7CAFBCF20FDF7C7FBCE20FDF7C4FBC3
:10CE7000CD20FDF7C1FBC620FDF7BEFB42E0B4208C
:10CE8000FDF7BAFBB520FDF7B7FBB620FDF7B4FB05
:10CE9000B720FDF7B1FBBE20FDF7AEFBBC20FDF7D0
:10CEA000ABFBBD20FDF7A8FB2CE0A420FDF7A4FB05
:10CEB0009C20FDF7A1FBA620FDF79EFBA720FDF718
:10CEC0009BFBAE20FDF798FBAC20FDF795FBA52062
:10CED000FDF792FB16E09420FDF78EFB8D20FDF709
:10CEE0008BFB8F20FDF788FB9720FDF785FB9E20AD
:10CEF000FDF782FB9520FDF77FFB9620FDF77CFB7D
:10CF000000E000BF00BF10BD0246F94812B1012A7F
:10CF100022D110E0012904D0022904D0032906D12E
:10CF200003E0F44805E0F24803E0F34801E0F0488C
:10CF300000BF00BF10E0012904D0022904D003295A
:10CF400006D103E0EA4805E0EB4803E0EB4801E0E6
:10CF5000E74800BF00BF00BF00BF70472DE9FF5F7B
:10CF600090B0824600200D900E900F90E4A00B90A0
:10CF700000200A90DDF8789000221346DDE91201C6
:10CF80003AF0F2FD09D201200A9000200146DDE9C5
:10CF900012233AF00DFCCDE912014FF0000B0AF11B
:10CFA00002003AF0FAFC02460B46CDE902010020ED
:10CFB000D4493BF0BFFACDE90401DDE912233AF090
:10CFC000FDFBCDE906013AF07FFD07468846642265
:10CFD0000023384641463AF0E5F963214A401A43B6
:10CFE00002D17F1C48F100080AF102003AF0D5FC9A
:10CFF00002460B46CDE900010020C2493BF09AFAF7
:10D00000CDE90401384641463AF0E5FCCDE902019C
:10D01000DDE904233AF044FCCDE906013AF054FD81
:10D0200004460D4651460A98FFF76EFF201A75F127
:10D0300000012CDBB448807AC0F34000F8B1B3485B
:10D04000407C012826D00120B049487406210A20DE
:10D0500030F0ECF8AE4890F87D00022802DA0120AA
:10D06000AB49C877AA4890F87D00FA2812DAA84898
:10D0700090F87D00401CA64981F87D000AE0002060
:10D08000A2494874A249C87781F87D0002E00020D7
:10D090009E4948740A98012803D1A9F1010000F0C3
:10D0A000FF09BAF1010F06D0BAF1020F08D0BAF1A8
:10D0B000030F4BD11FE0A9EB0A0000F0FF094AE083
:10D0C0000A9810B1012810D107E092490020091BED
:10D0D000A84101DA4FF0010A07E08F490020091B3F
:10D0E000A84101DA4FF0010A00BF00BFA9EB0A0016
:10D0F00000F0FF092FE00A9810B1012820D10FE0BD
:10D1000084490020091BA84102DA4FF0010A06E019
:10D1100081490020091BA84101DA4FF0020A0FE003
:10D120007D490020091BA84102DA4FF0010A06E000
:10D130007A490020091BA84101DA4FF0020A00BF1A
:10D1400000BFA9EB0A0000F0FF0904E0A9F102000A
:10D1500000F0FF0900BF00BFBAF1010F06D0BAF11D
:10D16000020F07D0BAF1030F0CD107E09820FDF7AA
:10D170002AFA0BE0A820FDF726FA07E0B820FDF711
:10D1800022FA03E0A820FDF71EFA00BF00BF1CE052
:10D1900048463AF013FC02460B46CDE90001002058
:10D1A00058493BF0C7F9CDE90401204629463AF039
:10D1B00012FCCDE90201DDE904233AF0F9FACDE9E8
:10D1C00006013AF081FC04460D4648463AF0F6FB6B
:10D1D00002460B46CDE9000100204A493BF0AAF97E
:10D1E000CDE90401204629463AF0F5FBCDE90201DC
:10D1F000DDE904233AF0DCFA00221346CDE906010A
:10D200003AF0CAFCC4D90A220023204629463AF043
:10D21000C9F8D0B20C900A220023204629463AF0E1
:10D22000C1F804460D461AE0A9F10101A1EB0B017A
:10D230000DAA0C9850540BF1010000F0FF0B0A22CC
:10D240000023204629463AF0ADF8D0B20C900A22CD
:10D250000023204629463AF0A5F804460D46002151
:10D260000846091BA841DFDBA9F10101A1EB0B0175
:10D270000DAA0C9850540BF1010000F0FF0B002296
:10D280004FF0804310461F493BF054F9CDE90401AB
:10D29000384641463AF09FFBCDE90201DDE904231F
:10D2A0003AF0FEFACDE906013AF00EFC04460D46CE
:10D2B000002618E00A220023204629463AF072F898
:10D2C000D0B20C900A220023204629463AF06AF890
:10D2D00004460D4609EB0A01491E891B0DAA0C984C
:10D2E0005054701CC6B25645E4DB00261FE0000017
:10D2F00040548900804A5D05A0BB0D00905F01008D
:10D300002E00000000002440EA2D0020581D0020BF
:10D31000901900207F9698003F420F009F860100E1
:10D320001F993144C8B2FFF713FC701CC6B2A9EBB9
:10D330000B00B042F4DC0A98012841D1A9EB0B00A4
:10D34000C0B209901E98401EC0B21E9009980728CE
:10D3500021D2DFE800F004080C1014181C00112082
:10D36000FDF731F91BE01A20FDF72DF917E0FA203F
:10D37000FDF729F913E0E920FDF725F90FE0D120A9
:10D38000FDF721F90BE0CA20FDF71DF907E0B220F7
:10D39000FDF719F903E01120FDF715F900BF00BFF3
:10D3A000099E09E00DAA915D1F9A3244521CD0B229
:10D3B000FDF746F9701CC6B21E988642F2DB0FE0FC
:10D3C000A9EB0B00C6B208E00DAA915D1F9A32448A
:10D3D000D0B2FDF735F9701CC6B21E988642F3DB59
:10D3E00014B0BDE8F09F2DE9FF5F90B082460020A9
:10D3F0000D900E900F90AFF2F8000B9000200A9065
:10D40000DDF8789000221346DDE912013AF0ACFB1A
:10D4100009D201200A9000200146DDE912233AF0EA
:10D42000C7F9CDE912014FF0000B0AF102003AF002
:10D43000B4FA02460B46CDE902010020FE493BF05A
:10D4400079F8CDE90401DDE912233AF0B7F9CDE925
:10D4500006013AF039FB0746884664220023384625
:10D46000414639F09FFF63214A401A4302D17F1C95
:10D4700048F100080AF102003AF08FFA02460B4622
:10D48000CDE900010020EC493BF054F8CDE904015E
:10D49000384641463AF09FFACDE90201DDE904231E
:10D4A0003AF0FEF9CDE906013AF00EFB04460D46CE
:10D4B0000A98012803D1A9F1010000F0FF09BAF18F
:10D4C000010F06D0BAF1020F08D0BAF1030F4FD105
:10D4D00020E0A9EB0A0000F0FF094EE00A9810B125
:10D4E000012811D107E0D5490020091BA84101DA24
:10D4F0004FF0010A08E042F20F710020091BA84119
:10D5000001DA4FF0010A00BF00BFA9EB0A0000F0EA
:10D51000FF0932E00A9810B1012823D110E0C74971
:10D520000020091BA84102DA4FF0010A07E042F28D
:10D530000F710020091BA84101DA4FF0020A11E027
:10D5400042F20F710020091BA84102DA4FF0010AD4
:10D5500007E040F2E7310020091BA84101DA4FF053
:10D56000020A00BF00BFA9EB0A0000F0FF0904E0B7
:10D57000A9F1020000F0FF0900BF00BFBAF1010FDE
:10D5800006D0BAF1020F07D0BAF1030F0CD107E0B1
:10D590009F20FDF718F80BE0AF20FDF714F807E027
:10D5A000BF20FDF710F803E0AF20FDF70CF800BF37
:10D5B00000BF1CE048463AF001FA02460B46CDE9AE
:10D5C000000100209C493AF0B5FFCDE90401204656
:10D5D00029463AF000FACDE90201DDE904233AF0E8
:10D5E000E7F8CDE906013AF06FFA04460D464846E1
:10D5F0003AF0E4F902460B46CDE9000100208E49DD
:10D600003AF098FFCDE90401204629463AF0E3F9C3
:10D61000CDE90201DDE904233AF0CAF800221346FD
:10D62000CDE906013AF0B8FAC4D90A22002320460F
:10D63000294639F0B7FED0B20C900A2200232046CA
:10D64000294639F0AFFE04460D461AE0A9F1010162
:10D65000A1EB0B010DAA0C9850540BF1010000F046
:10D66000FF0B0A2200232046294639F09BFED0B248
:10D670000C900A2200232046294639F093FE0446E6
:10D680000D4600210846091BA841DFDBA9F1010175
:10D69000A1EB0B010DAA0C9850540BF1010000F006
:10D6A000FF0B00224FF08043104663493AF042FFDF
:10D6B000CDE90401384641463AF08DF9CDE9020141
:10D6C000DDE904233AF0ECF8CDE906013AF0FCF983
:10D6D00004460D46002618E00A220023204629466B
:10D6E00039F060FED0B20C900A2200232046294671
:10D6F00039F058FE04460D4609EB0A01491E891B04
:10D700000DAA0C985054701CC6B25645E4DB002696
:10D7100006E01F993144C8B2FFF71AFA701CC6B26E
:10D72000A9EB0B00B042F4DC0A98012837D1A9EB31
:10D730000B00C0B209901E98401EC0B21E900998FE
:10D7400030B1012809D002280BD0032811D10CE0F8
:10D750004FF48370FCF737FF10E0ED20FCF733FF48
:10D760000CE0DE20FCF72FFF08E0C620FCF72BFFC3
:10D7700004E04FF48370FCF726FF00BF00BF099E52
:10D7800009E00DAA915D1F9A3244521CD0B2FCF7F9
:10D7900057FF701CC6B21E988642F2DB0FE0A9EB61
:10D7A0000B00C6B208E00DAA915D1F9A3244D0B2B8
:10D7B000FCF746FF701CC6B21E988642F3DB14B01D
:10D7C000BDE8F09F2DE9FF5F86B0174698464FF001
:10D7D000000B00221346384641463AF0C5F909D2FB
:10D7E0004FF0010B3A4643460020014639F0E0FF76
:10D7F000074688460698002879D1BBF1000F47D12B
:10D800000F49611A75F100003EDB0E48807AC0F3C3
:10D81000400080B30C48407C012874D001200A49A4
:10D82000487406210A202FF001FD0648807AC0F3D3
:10D830004000002867D009E0000024409F860100D6
:10D8400040548900EA2D0020581D0020F84890F827
:10D850007D00022802DA0120F549C877F44890F8E3
:10D860007D00FA284FDAF24890F87D00401CF0491C
:10D8700081F87D0047E0FFE70020EE494874EC495D
:10D88000C87781F87D003EE00020EA4948743AE01C
:10D89000E9490020091BA84132DBE848807AC0F33F
:10D8A000400028B3E348407C01282CD00120E14906
:10D8B000487406210A202FF0B9FCE048807AC0F3B2
:10D8C000400000B3DA4890F87D00022802DA012017
:10D8D000D749C877D64890F87D00FA2813DAD4489B
:10D8E00090F87D00401CD24981F87D000BE029E1D1
:10D8F0000020D0494874CE49C87781F87D0002E005
:10D900000020CC494874BBF1000F71D103E0CC4A30
:10D91000A41A65F10005CA49631A65F100000022E6
:10D920001146D21A8141F2DB0A2200232046294601
:10D9300039F038FD02F0FF0A0A220023204629466A
:10D9400039F030FD04460D4618E0C9F1060003A980
:10D9500001F800A009F1010000F0FF090A220023EC
:10D960002046294639F01EFD02F0FF0A0A22002354
:10D970002046294639F016FD04460D46002108468A
:10D98000091BA841E1DBC9F1060003A901F800A0C9
:10D9900009F1010000F0FF090022AA4B3846414678
:10D9A00039F00CFFCDE900013AF08EF804460D463F
:10D9B0000A2200232046294639F0F4FCD0B28DF823
:10D9C00013000022A04B3846414639F0F7FECDE95E
:10D9D00000013AF079F804460D460A220023204659
:10D9E000294639F0DFFCD0B28DF81400002606E09D
:10D9F00018E0311DC8B2FFF7ABF8701CC6B2C9F110
:10DA00000700B042F5DCC9F10700C6B207E003AA7F
:10DA1000915D321DD0B2FCF713FE701CC6B2092E08
:10DA2000F5DB8BE05220FCF7CEFD03E0874AA41A19
:10DA300065F100058549621A65F1000000239A1A14
:10DA400073EB0001F2DB0A222046294639F0AAFCDA
:10DA500002F0FF0A0A2200232046294639F0A2FCE0
:10DA600004460D4618E0C9F1050003A901F800A01D
:10DA700009F1010000F0FF090A220023204629468F
:10DA800039F090FC02F0FF0A0A22002320462946C2
:10DA900039F088FC04460D4600210846091BA841C0
:10DAA000E1DBC9F1050003A901F800A009F10100BB
:10DAB00000F0FF090022634B3846414639F07EFEF4
:10DAC000CDE900013AF000F804460D460A22002391
:10DAD0002046294639F066FCD0B28DF812000022AB
:10DAE000594B3846414639F069FECDE9000139F01D
:10DAF000EBFF04460D460A2200232046294639F052
:10DB000051FCD0B28DF81300002605E0711DC8B29B
:10DB1000FFF71EF8701CC6B2C9F10600B042F5DC72
:10DB2000C9F10600C6B207E003AA915D721DD0B22A
:10DB3000FCF786FD701CC6B2082EF5DBA820FCF7AA
:10DB400042FDD2E1BBF1000F3AD13B49611A75F1B8
:10DB5000000031DB3948807AC0F3400020B33548FB
:10DB6000407C012879D001203249487406210A20DE
:10DB70002FF05CFB3148807AC0F34000F8B12C48AC
:10DB800090F87D00022802DA01202949C877284848
:10DB900090F87D00FA2860DA254890F87D00401C56
:10DBA000234981F87D0058E000202249487420492B
:10DBB000C87781F87D0050E000201E4948744CE091
:10DBC00023490020091BA84144DB1C48807AC0F38C
:10DBD000400020B31748407C01283ED00120154961
:10DBE000487406210A202FF021FB1448807AC0F3E4
:10DBF0004000E0B10E4890F87D00022802DA0120D2
:10DC00000B49C8770A4890F87D00FA2825DA0848B9
:10DC100090F87D00401C064981F87D001DE0002041
:10DC2000044948740249C87781F87D0015E014E082
:10DC300090190020581D0020A0BB0D00EA2D0020E7
:10DC400080969800000024400000594040420F0098
:10DC5000905F01000020FB494874BBF1000F7DD1AB
:10DC600003E0F949641A65F10005F749621A65F1A4
:10DC7000000000239A1A73EB0001F2DB0A2220460F
:10DC8000294639F08FFB02F0FF0A0A2200232046C2
:10DC9000294639F087FB04460D4618E0C9F1050016
:10DCA00003A901F800A009F1010000F0FF090A2210
:10DCB00000232046294639F075FB02F0FF0A0A22AC
:10DCC00000232046294639F06DFB04460D4600210D
:10DCD0000846091BA841E1DBC9F1050003A901F8C9
:10DCE00000A009F1010000F0FF090022D74B3846DF
:10DCF000414639F063FDCDE9000139F0E5FE044607
:10DD00000D460A2200232046294639F04BFBD0B2AB
:10DD10008DF812000022CE4B3846414639F04EFDB8
:10DD2000CDE9000139F0D0FE04460D460A22002359
:10DD30002046294639F036FBD0B28DF81300002278
:10DD4000C44B3846414639F039FDCDE9000139F080
:10DD5000BBFE04460D460A22002300E021E02046D7
:10DD6000294639F01FFBD0B28DF81400002605E0DB
:10DD7000311DC8B2FEF7ECFE701CC6B2C9F1060038
:10DD8000B042F5DCC9F10600C6B207E003AA915D16
:10DD9000321DD0B2FCF754FC701CC6B2092EF5DB64
:10DDA000A0E05220FCF70FFC03E0AB4AA41A65F197
:10DDB0000005A949621A65F1000100239A1A73EB64
:10DDC0000100F2DB0A222046294639F0EBFA02F084
:10DDD000FF0A0A2200232046294639F0E3FA0446C6
:10DDE0000D4618E0C9F1040003A901F800A009F1EB
:10DDF000010000F0FF090A2200232046294639F0DD
:10DE0000D1FA02F0FF0A0A2200232046294639F0FF
:10DE1000C9FA04460D4600210846091BA841E1DB6A
:10DE2000C9F1040003A901F800A009F1010000F004
:10DE3000FF090022854B3846414639F0BFFCCDE949
:10DE4000000139F041FE04460D460A220023204617
:10DE5000294639F0A7FAD0B28DF8110000227C4B88
:10DE60003846414639F0AAFCCDE9000139F02CFED4
:10DE700004460D460A2200232046294639F092FA2C
:10DE8000D0B28DF812000022724B3846414639F06C
:10DE900095FCCDE9000139F017FE04460D460A2233
:10DEA00000232046294639F07DFAD0B28DF81300C0
:10DEB000002605E0711DC8B2FEF74AFE701CC6B20E
:10DEC000C9F10500B042F5DCC9F10500C6B207E0B2
:10DED00003AA915D721DD0B2FCF7B2FB701CC6B2F2
:10DEE000082EF5DBB820FCF76EFB0AB0BDE8F09F0A
:10DEF0002DE9F04F87B08346174698464FF000094A
:10DF00003846414639F0E0FD04460D46BBF1020FAC
:10DF100078D104E042F21072A41A65F1000542F2D1
:10DF20001071621A65F1000000239A1A73EB000168
:10DF3000F0DB0A222046294639F034FA02F0FF0AC3
:10DF40000A2200232046294639F02CFA04460D46C1
:10DF500018E0C9F1030004A901F800A009F10100CB
:10DF600000F0FF090A2200232046294639F01AFA58
:10DF700002F0FF0A0A2200232046294639F012FA4D
:10DF800004460D4600210846091BA841E1DBC9F102
:10DF9000030004A901F800A009F1010000F0FF0945
:10DFA00000222A4B3846414639F008FCCDE90201EF
:10DFB00039F08AFD04460D460A22002320462946F0
:10DFC00039F0F0F9D0B28DF814000022214B384618
:10DFD000414639F0F3FB00221C4BCDE9000139F03A
:10DFE0005FFCCDE9020139F06FFD04460D460A22BF
:10DFF00000232046294639F0D5F9D0B28DF8150016
:10E00000002607E02AE006F10D01C8B2FEF7A0FDE8
:10E01000701CC6B2C9F10400B042F4DCC9F10400BE
:10E02000C6B208E004AA915D06F10D02D0B2FCF779
:10E0300007FB701CC6B2062EF4DBBF20FCF7C3FA48
:10E04000BDE00000581D002040420F0000002440A9
:10E050000000594000408F40A086010004E04FF4CA
:10E060007A72A41A65F100054FF47A71621A65F1AB
:10E07000000100239A1A73EB0100F0DB0A2220460C
:10E08000294639F08FF902F0FF0A0A2200232046C0
:10E09000294639F087F904460D4618E0C9F1020017
:10E0A00004A901F800A009F1010000F0FF090A220B
:10E0B00000232046294639F075F902F0FF0A0A22AA
:10E0C00000232046294639F06DF904460D4600210B
:10E0D0000846091BA841E1DBC9F1020004A901F8C7
:10E0E00000A009F1010000F0FF090022FC4B3846B6
:10E0F000414639F063FBCDE9020139F0E5FC044605
:10E100000D460A2200232046294639F04BF9D0B2A9
:10E110008DF813000022F34B3846414639F04EFB90
:10E120000022EF4BCDE9000139F0BAFBCDE9020145
:10E1300039F0CAFC04460D460A220023204629462F
:10E1400039F030F9D0B28DF814000022E64B384691
:10E15000414639F033FB0022E14BCDE9000139F0B3
:10E160009FFBCDE9020139F0AFFC04460D460A22BF
:10E1700000232046294639F015F9D0B28DF8150054
:10E18000002606E006F10D01C8B2FEF7E1FC701CA6
:10E19000C6B2C9F10300B042F4DCC9F10300C6B253
:10E1A00008E004AA915D06F10D02D0B2FCF748FA2E
:10E1B000701CC6B2062EF4DBD720FCF704FA07B0B9
:10E1C000BDE8F08F2DE9FC4782460E460024A046AC
:10E1D0000025002000900190BAF1090F2ED2DFE84F
:10E1E0000AF0052E4CBCFD4DBDFCFB000521084688
:10E1F000FCF726FA1320FCF7E6F91820FCF7E3F900
:10E20000F020FCF7E0F9C820FCF7DDF9A820FCF7C6
:10E21000DAF9002410E0325D11096200921DD0B2DB
:10E22000FCF70EFA325D02F00F016200D21DD0B28F
:10E23000FCF706FA601CC4B2042CECDB82E1E92096
:10E24000FCF7C1F9B220FCF7BEF9002412E0325D00
:10E25000110904EB4402921DD0B2FCF7F1F9325DD2
:10E2600002F00F0104EB4402D21DD0B2FCF7E8F932
:10E27000601CC4B2032CEADB64E100BF1220FCF78F
:10E28000A2F91020FCF79FF93B20FCF79CF93A20FB
:10E29000FCF799F91920FCF796F91B20FCF793F984
:10E2A0001A20FCF790F94FF48170FCF78CF94FF4C9
:10E2B0008070FCF788F9C820FCF785F9002449E054
:10E2C000375D0A2097FBF0F100FB117000F0FF09A9
:10E2D0000A2097FBF0F700250FE0C5F102000DF8CA
:10E2E0000090681CC5B20A2097FBF0F100FB11708A
:10E2F00000F0FF090A2097FBF0F7002FEDDCC5F1D5
:10E3000002000DF80090681CC5B2012D02D0022D4C
:10E3100008D103E000208DF8010000BF00208DF837
:10E32000000000E000BF00BF4FF000080DE01DF846
:10E33000081008F10702032303FB0422D0B2FCF704
:10E340007FF908F1010000F0FF08B8F1030FEEDBE0
:10E35000601CC4B2022CB3DBF4E000BF0B20FCF75E
:10E3600032F91220FCF72FF90920FCF72CF90A20CA
:10E37000FCF729F91120FCF726F91320FCF723F903
:10E380001820FCF720F93178707801EB00270A207B
:10E3900097FBF0F100FB117000F0FF090A2097FBDA
:10E3A000F0F70FE0C5F104000DF80090681CC5B24D
:10E3B0000A2097FBF0F100FB117000F0FF090A2022
:10E3C00097FBF0F7002FEDDCC5F104000DF800908D
:10E3D000681CC5B2012D02E04EE02FE02DE006D012
:10E3E000022D08D0032D0AD0042D10D10BE00020FF
:10E3F0008DF8030000BF00208DF8020000BF002050
:10E400008DF8010000BF00208DF8000000E000BF83
:10E4100000BFC5F1050000F0FF080AE01DF8081074
:10E4200008F10602D0B2FCF70BF908F1010000F088
:10E43000FF08B8F1050FF1DB84E000BF307800F091
:10E440000F010520FCF7FCF8002412E0621CB25C0E
:10E4500011096200921DD0B2FCF7F2F8621CB25CA6
:10E4600002F00F016200D21DD0B2FCF7E9F8601C87
:10E47000C4B2042CEADB65E008210520FCF7E0F8D3
:10E480003B20FCF7A0F83A20FCF79DF81920FCF798
:10E490009AF81B20FCF797F81A20FCF794F805214E
:10E4A0000720FCF7CDF8F220FCF78DF8F020FCF700
:10E4B0008AF8F0780006B17840EA0140717840EAC5
:10E4C0000120317840EA01070A2097FBF0F100FBB8
:10E4D000117000F0FF090A2097FBF0F716E000002A
:10E4E0000000244000408F400088C340C5F1050073
:10E4F0000DF80090681CC5B20A2097FBF0F100FBF4
:10E50000117000F0FF090A2097FBF0F7002FEDDCF7
:10E51000C5F105000DF80090681CC5B2C5F10600F4
:10E5200000F0FF080AE01DF8081008F10802D0B258
:10E53000FCF786F808F1010000F0FF08B8F1060FBB
:10E54000F1DB00BF00BFBDE8FC872DE9FC47824638
:10E550000D460024A0460026002000900190BAF14C
:10E56000090F3BD2DFE80AF0053B5DB0B25EB1B304
:10E57000C900FD20FCF727F8FE20FCF724F840F244
:10E580000710FCF720F840F20510FCF71CF84FF4D8
:10E590008370FCF718F8F520FCF715F8F720FCF766
:10E5A00012F8D720FCF70FF8002410E02A5D1109BB
:10E5B00062000F32D0B2FCF743F82A5D02F00F017F
:10E5C00062001032D0B2FCF73BF8601CC4B2022CDF
:10E5D000ECDB285D01091320FCF732F8DCE0E520D4
:10E5E000FBF7F1FFE720FBF7EEFFC420FBF7EBFFA3
:10E5F000BF20FBF7E8FF002410E02A5D110962004C
:10E600000E32D0B2FCF71CF82A5D02F00F01620056
:10E610000F32D0B2FCF714F8601CC4B2032CECDB50
:10E62000BAE000BFD720FBF7CEFF002449E02F5D02
:10E630000A2097FBF0F100FB117000F0FF090A209F
:10E6400097FBF0F700260FE0C6F102000DF80090EE
:10E65000701CC6B20A2097FBF0F100FB117000F0AD
:10E66000FF090A2097FBF0F7002FEDDCC6F102004E
:10E670000DF80090701CC6B2012E02D0022E08D1F7
:10E6800003E000208DF8010000BF00208DF800009D
:10E6900000E000BF00BF4FF000080DE01DF80810BB
:10E6A00008F10E02032303FB0422D0B2FBF7C8FFDC
:10E6B00008F1010000F0FF08B8F1030FEEDB601C69
:10E6C000C4B2022CB3DB67E000BF65E000BF0024EA
:10E6D00010E02A5D110962000E32D0B2FBF7B0FFE4
:10E6E0002A5D02F00F0162000F32D0B2FBF7A8FFE3
:10E6F000601CC4B2042CECDB4EE005210E20FBF7BD
:10E700009FFFF520FBF75FFFF720FBF75CFF2F78FB
:10E710000A2097FBF0F100FB117000F0FF090A20BE
:10E7200097FBF0F70FE0C6F102000DF80090701CA7
:10E73000C6B20A2097FBF0F100FB117000F0FF0950
:10E740000A2097FBF0F7002FEDDCC6F102000DF870
:10E750000090701CC6B2012E02D0022E08D103E038
:10E7600000208DF8010000BF00208DF8000000E0BF
:10E7700000BF00BF4FF000080AE01DF8081008F1C4
:10E780000F02D0B2FBF75CFF08F1010000F0FF08B8
:10E79000B8F1030FF1DB00BF00BFBDE8FC87024604
:10E7A0000B4600207047704738B50546992D1FDC91
:10E7B00055B9002405E0611CC8B2FEF7C9F9601C18
:10E7C000C4B2022CF7DB13E005F00F008DF8010056
:10E7D000C5F307108DF80000002407E01DF80410B1
:10E7E000621CD0B2FBF72CFF601CC4B2022CF5DB1C
:10E7F00038BD38B5054655B9002405E0A11CC8B29E
:10E80000FEF7A6F9601CC4B2022CF7DB12E005F09B
:10E810000F008DF8010028118DF80000002407E09A
:10E820001DF80410E21CD0B2FBF70AFF601CC4B252
:10E83000022CF5DB38BD10B5044634B1012C09D0EB
:10E84000022C0BD0032C0ED109E04FF48A70FBF799
:10E85000BAFE09E03F20FBF7B6FE05E004E05720D2
:10E86000FBF7B1FE00E000BF00BF10BD10B50446CD
:10E8700034B1012C09D0022C0BD0032C0ED109E0AD
:10E880004FF48A70FBF7B8FE09E03F20FBF7B4FEB7
:10E8900005E004E05720FBF7AFFE00E000BF00BF3B
:10E8A00010BD10B504462046FBF78DFEFE48FBF771
:10E8B0004AFE10BD10B5002404E0FF20FA490855B7
:10E8C000601C84B2232CF8DBF748FBF73CFE10BD3C
:10E8D00010B504462046FBF78FFEF348FBF733FEE6
:10E8E00010BD10B500244FF48A70FBF76CFE3C207D
:10E8F000FBF769FE4320FBF766FE4420FBF763FE4F
:10E90000EA4890F86300012803D14220FBF75BFE40
:10E9100007E0E64890F86300022802D14920FBF79F
:10E9200052FEE34890F8090110B14020FBF74BFE7E
:10E93000E0488079C0F3401018B14FF48970FBF7BC
:10E9400042FEDC48C0790221B1EB901F03D140F2B6
:10E950001110FBF738FED548007C012803D1482070
:10E96000FBF731FE02E04820FBF746FED248007B71
:10E9700000F00400042804D140F20D10FBF723FE40
:10E9800003E04FF48670FBF71EFE40F21510FBF714
:10E990001AFEC648407E462810DD4FF48770FBF70C
:10E9A00012FE40F20F10FBF70EFE40F21710FBF7BD
:10E9B0000AFE4FF48B70FBF706FE25E0BB48407E55
:10E9C00028280CDD4FF48770FBF7FDFD40F20F1097
:10E9D000FBF7F9FD40F21710FBF7F5FD14E0B34823
:10E9E000407E142808DD4FF48770FBF7ECFD40F201
:10E9F0000F10FBF7E8FD07E0AC48407E002803DD80
:10EA00004FF48770FBF7DFFDAC48807810B9062023
:10EA1000FBF7D9FDA948407804282FD006DC01284F
:10EA200009D002280ED0032854D117E0052835D08C
:10EA300063284FD140E00520FBF7C5FD0720FBF719
:10EA4000C2FD48E00520FBF7BEFD0420FBF7BBFD3F
:10EA50009A49B1F80B00FFF7A7FE3CE00520FBF751
:10EA6000B2FD9548007B00F0010018B10720FBF7CC
:10EA7000AAFD02E00720FBF7BFFD2CE00520FBF715
:10EA8000A2FD8D48007B00F0010018B10420FBF7C7
:10EA90009AFD02E00420FBF7AFFD1CE08648007BF6
:10EAA00000F00200022803D10520FBF78CFD02E0F4
:10EAB0000520FBF7A1FD0EE07F48007B00F004007D
:10EAC000042803D10520FBF77EFD02E00520FBF7BB
:10EAD00093FD00E000BF00BF7748C07C0A2833DA0E
:10EAE00000241DE07448C17C70484630405C50B141
:10EAF0005720FBF768FD7049CA7C6C494631885C39
:10EB0000FFF777FE0EE06C48C07C401C6A49C87471
:10EB10000846C07C0A2801DB0020C874601CC4B20F
:10EB20000A2CDFDB00BF6448007B00F00100D0B995
:10EB30006148C07C401C6049C8740846C07C0A28F3
:10EB400011DB0020C8740EE000205B49C8745748F0
:10EB500090F8460038B15720FBF735FD534991F83E
:10EB60004600FFF746FE4720FBF72DFD5448C079CD
:10EB700019280FDD4620FBF726FD4520FBF723FD76
:10EB80004D20FBF720FD4E20FBF71DFD4F20FBF72E
:10EB90001AFD40E04A48C079152810DB4848C07982
:10EBA00019280CDC4620FBF70EFD4520FBF70BFD7A
:10EBB0004D20FBF708FD4E20FBF705FD2BE04048FC
:10EBC000C07910280DDB3E48C079142809DC4620A6
:10EBD000FBF7F9FC4520FBF7F6FC4D20FBF7F3FCB7
:10EBE00019E03748C0790B280ADB3548C0790F286F
:10EBF00006DC4620FBF7E7FC4520FBF7E4FC0AE0D7
:10EC00002F48C079002806DD2D48C0790B2802DA8C
:10EC10004620FBF7D8FC2548007A01280CD129486A
:10EC2000807800F0010018B13F20FBF7CCFC0EE02B
:10EC30003F20FBF7E1FC0AE01C4890F8450018B9BA
:10EC40003F20FBF7C0FC02E03F20FBF7D5FC10BDE6
:10EC50002DE9FC410446052C7ED2DFE804F0450393
:10EC600086C0FB000320FBF7AEFC8320FBF7ABFC68
:10EC70004FF48470FBF7A7FC8520FBF7A4FC8420ED
:10EC8000FBF7A1FC05200921CDE9001008488030E0
:10EC9000056843682A460220FEF760F90449D1F866
:10ECA000880038F08BFE0FE0D20F0020A216002063
:10ECB0008E220020D22D0020581D0020D947002090
:10ECC0003A1F00200C00002007460022CE4B38F0EF
:10ECD000E7FD05460B460E2007212A46CDE9001028
:10ECE0000320FEF780FBEFE00120FBF76CFC002027
:10ECF000FBF769FC8B20FBF766FC8220FBF763FCCB
:10ED00008E20FBF760FC8720FBF75DFC8620FBF77D
:10ED10005AFCBE4890F8090158B905200921CDE9EF
:10ED20000010BA48856AC36A2A460220FEF716F91F
:10ED30000AE005200921CDE90010B4498D6CCB6CA7
:10ED40002A460220FEF70AF9B049486F38F0F9FE6A
:10ED500005460B460E2000E0B5E007212A46CDE926
:10ED600000100220FEF73FFBAEE00120FBF72BFC7A
:10ED70000020FBF728FC8B20FBF725FC8220FBF70B
:10ED800022FC8120FBF71FFCA04890F8090158B92C
:10ED900005200921CDE900109C48856AC36A2A46EE
:10EDA0000220FEF7DBF80AE005200921CDE900107A
:10EDB00096498D6CCB6C2A460220FEF7CFF893491A
:10EDC000D1F8980038F0BDFE05460B460E2007210D
:10EDD0002A46CDE900100220FEF705FB74E0012071
:10EDE000FBF7F1FB0020FBF7EEFB8B20FBF7EBFBC7
:10EDF0008220FBF7E8FB8C20FBF7E5FB834890F8CB
:10EE0000090158B905200921CDE900107F48856A1C
:10EE1000C36A2A460220FEF7A1F80AE0052009216C
:10EE2000CDE900107948856CC36C2A460220FEF7B4
:10EE300095F87649D1F89C0038F083FE05460B46DC
:10EE40000E2007212A46CDE900100220FEF7CBFA5A
:10EE50003AE0FFE70220FBF7B6FB0020FBF7B3FB2D
:10EE60008220FBF7B0FB8720FBF7ADFB8620FBF78A
:10EE7000AAFB664890F8090158B905200921CDE997
:10EE8000001062490D6A4B6A2A460220FEF766F8B6
:10EE90000AE005200921CDE900105C48056C436CAF
:10EEA0002A460220FEF75AF85849086F38F049FE02
:10EEB00005460B460E2007212A46CDE90010022008
:10EEC000FEF791FA00E000BF00BFBDE8FC813CB551
:10EED00005465020FBF777FB092D7DD2DFE805F0D2
:10EEE000050F193C5223425C860049490020FFF778
:10EEF00069F94749491F0020FFF727FB81E0454991
:10EF00000120FFF75FF94349C91C0120FFF71DFBF2
:10EF100077E041490220FFF755F93F49891C02205B
:10EF2000FFF713FB6DE03D480078012809D13C490B
:10EF30000520FFF747F93A49891C0520FFF705FB33
:10EF400009E0374919310520FFF73CF934491B31F5
:10EF50000520FFF7FAFA54E02F49091D0320FFF7B7
:10EF600031F94EE02D480078012805D12C49091DC2
:10EF70000620FFF727F904E029491D310620FFF795
:10EF800021F93EE027490420FFF71CF92549491DD6
:10EF90000420FFF7DAFA34E02248413890F84D00B7
:10EFA0003038C0B28DF80000002411E06000001D70
:10EFB0001C490A31085C30386100C91C194A0A3200
:10EFC000515C00EB0110C1B2601C0DF80010C4B21E
:10EFD000072CEBDB694600E012E00720FFF7F2F8B0
:10EFE0000DF105010720FFF7B0FA0AE00E490820ED
:10EFF000FFF7E8F80C49491E0820FFF7A6FA00E0E1
:10F0000000BF00BF3CBD00000088C3408E2200202E
:10F0100096270020140000203D2C0020F046002000
:10F020002645002061270020E900002008B50120C6
:10F03000ADF8000010208DF8030003208DF80200C9
:10F040006946FE4801F0D8FD08BD08B50120ADF8BD
:10F05000000000208DF8030003208DF802006946AF
:10F06000F64801F0C9FD08BD08B54020ADF8000024
:10F0700048208DF8030003208DF802006946EF4810
:10F0800001F0BAFD08BD08B54020ADF80000002031
:10F090008DF8030003208DF802006946E74801F06F
:10F0A000ABFD08BD08B50420ADF800008DF80300E5
:10F0B00003208DF802006946E04801F09DFD08BD7F
:10F0C00008B50420ADF8000000208DF803000320EF
:10F0D0008DF802006946D94801F08EFD08BD08B5DB
:10F0E0004FF40070ADF8000010208DF803000320ED
:10F0F0008DF802006946D24801F07EFD08BD08B5D2
:10F100004FF48060ADF8000010208DF8030003205C
:10F110008DF802006946CA4801F06EFD08BD08B5C9
:10F120004FF40070ADF8000000208DF803000320BC
:10F130008DF802006946C24801F05EFD08BD08B5C1
:10F140004FF48060ADF8000000208DF8030003202C
:10F150008DF802006946BA4801F04EFD08BD10B5B1
:10F16000FFF7BDFF0120B74908604FF4FA70F9F7C7
:10F1700098F90020B449C1F8A40110BD10B5FFF7FB
:10F18000AEFF0120AF49086010BD10B5FFF7A7FF23
:10F190000020AC49086010BD10B5FFF7B0FF01209A
:10F1A000A849091D08604FF4FA70F9F77AF90020B0
:10F1B000A549C1F8A80110BD10B5FFF7A0FF0120B7
:10F1C000A049091D086010BD10B5FFF798FF002089
:10F1D0009C49091D086010BD9848806800F0040132
:10F1E000890809B9002070470120FCE710B597484D
:10F1F000807A012802D19549087402E000209349E1
:10F2000008749248407A01280FD19048408A30B95A
:10F2100001208E49C8734FF46160488208E08B4832
:10F22000408A401E8949488202E00020874948827E
:10F230008648007C012802D1FFF7A0FF05E00020EE
:10F24000834981F83400FFF7A0FF8048C07B012884
:10F2500026D17F4890F835000F2807DA7C4890F8CF
:10F260003500401C7A4981F8350006E000207749D6
:10F27000C8730F20764981F83500754890F835003D
:10F28000032802DAFFF7A0FF10E0714890F835007C
:10F290000D2802DAFFF790FF08E0FFF795FF05E081
:10F2A00000206B4981F83500FFF78EFF10BD2DE976
:10F2B000F05F6648807A012803D1002064494876CF
:10F2C00085E06248407A012861D160488079012850
:10F2D00016D15F49498E46F2A862501A38F05DFB9C
:10F2E000804600225B4B38F069FA064600225A4BF2
:10F2F00038F0D6FA044638F0CEFB5549487637E068
:10F3000052484079012833D15148B0F81700534989
:10F31000097801EB8101B0EB410F26DC4F490978F8
:10F320004E4A5278891A01EB8101480038F035FBCA
:10F3300004460D464649B1F81710484A527802EB88
:10F340008202A1EB420038F028FB06460022444B23
:10F3500038F034FA804622462B4638F0A1FA82462D
:10F3600038F099FB3A49487602E01420384948764B
:10F370003748407E142802DD142035494876344849
:10F38000407E002823DA0020314948761FE03048CB
:10F39000408E46F2A861884216DA2D49498E46F21F
:10F3A000A862501A38F0F9FA80460022294B38F04A
:10F3B00005FA06460022284B38F072FA044638F067
:10F3C0006AFB2349487602E000202149487620481C
:10F3D000407E642802DD64201D494876BDE8F09F28
:10F3E00070B52048007817280AD11E48407839287F
:10F3F00006D11C488078022802DA012013490870DF
:10F4000012480078012807D010484078012803D01E
:10F410000E48007B012806D101200C49887000208D
:10F4200008704870087309488078012830D107486F
:10F43000C0780A281BD10020044915E000100140C3
:10F4400000180140A401234200002342F60F0020CF
:10F45000A21600200000594000AAD940F200002066
:10F46000000034400C0000208870C87004E0F848A8
:10F47000C078401CF649C870F548C078012808D10A
:10F48000FFF7D4FD0120F9F70CF80120F1490860DD
:10F490009EE0EF48C0780228FAD1EF48B0F8170094
:10F4A000EE49097801EB8101B0EB410F0EDB04F06E
:10F4B00013F8E948B0F81700E849097801EB810131
:10F4C000B0EB410F04DA04F007F801E004F004F8AF
:10F4D0000020E0490860DE48407B022836D1002049
:10F4E000DB494873DC48B0F81700DC49497801EB88
:10F4F0008101B0EB410F21DDD548807B012867D029
:10F500000120D3498873122102202DF08FFE06F0CE
:10F510007AFBD34890F86D00022802DA0120D04926
:10F52000C873CF4890F86D00FA2851DACC4890F8AB
:10F530006D00401CCA4981F86D0049E00020C449B3
:10F540008873C749C87381F86D0041E0C048407BAB
:10F55000012823D10020BE494873C2480079C0F376
:10F560008000A8B3BC48B0F81700BC49497801EB4B
:10F570008101322202EB4101884229DDB448807BBF
:10F58000012825D10020B2498873B549C87381F894
:10F590006D00012102202DF049FE19E0FFF764FD06
:10F5A000AC4868380068012812D1A948807B01283E
:10F5B0000ED10A20F8F775FFA648683800680128C0
:10F5C00006D10020A2498873A549C87381F86D004F
:10F5D0009F48C07A01281FD100209D49C8729E49CA
:10F5E000B1F8170038F0EAF9044600229E4B38F0D3
:10F5F000D3FA11D8002142F66400FAF712FA00217A
:10F6000042F66800FAF70DFA00209349088648860A
:10F61000012102202DF00AFE8F48007CE8BB8E48B5
:10F62000008E401C8C4908860846008EB0F5616F3C
:10F630001BDB002008860846408E401C4886084692
:10F64000408E4FF6FA71884202DD002082494886DA
:10F650008148018E42F66400FAF7E3F97E48418E54
:10F6600042F66800FAF7DDF90EE07B48008E4FF4B1
:10F67000167190FBF1F201FB120028B97648018E59
:10F6800042F66400FAF7CDF97348408E4FF6FA71EE
:10F69000884202DD0020704948866F48B0F81700A4
:10F6A0006E49097801EB8101B0EB410F03DA0120CB
:10F6B000674948710EE06848B0F817006749097853
:10F6C00001EB8101142202EB4101884202DD00209E
:10F6D0005F4948716048B0F817006049497801EB0C
:10F6E0008101B0EB410F03DA01205949C8710EE0E6
:10F6F0005948B0F817005949497801EB81011422A3
:10F7000002EB4101884202DD00205149C871524894
:10F71000408E46F2A861884203DB01204C49087202
:10F7200011E04D49488E38F049F9044600224F4B0C
:10F7300038F032FA03D801204549887103E00020EF
:10F7400043490872887142488079012803D04048B3
:10F75000407901282CD14348007900F00100F8B12C
:10F760003B48407A01282ED00120394948721021A7
:10F7700002202DF05BFD3A4890F86100022802DA81
:10F7800001203749C870364890F86100FA281ADA23
:10F79000334890F86100401C314981F8610012E063
:10F7A00000202B4948722E49C87081F861000AE098
:10F7B0002748407A38B100202549487241F21001AB
:10F7C00002202DF033FD2248C079012803D02048C3
:10F7D000007A01282ED106F016FA22480079C0F3EB
:10F7E0004000F8B11A48807A01282ED0012018492B
:10F7F0008872112102202DF019FD194890F862003D
:10F80000022802DA012016490871154890F86200B2
:10F81000FA281ADA124890F86200401C104981F860
:10F82000620012E000200A4988720D49087181F8CF
:10F8300062000AE00648807A38B1002004498872E4
:10F8400041F2110102202DF0F1FCFFF730FD70BDF7
:10F85000F60F002080012242A2160020F2000020B4
:10F8600090190020EA2D002000001C400088D440A0
:10F8700010B500215D4803F048F84FF47A715B48F9
:10F8800003F058F80121594803F03FF810BD7047C4
:10F8900010B590B004460121880401F076FC0121E6
:10F8A000084601F058FC524802F05EFD0C9400201E
:10F8B000ADF83400ADF83600ADF83800ADF83C00D6
:10F8C0000C20ADF83A000CA9494802F090FD4748D9
:10F8D00002F04EFF4648001D01904648029000206D
:10F8E00003904FF47A7004900020059080200690D9
:10F8F000002007900890202009904FF440500A9073
:10F9000000200B9001A9394802F0D4FF01224021C8
:10F91000374802F029FE0121344802F0F6FF0121A8
:10F92000334802F0F0FD40F22661314802F006FF54
:10F9300010B010BD10B500212C4802F0E6FF4FF4C6
:10F940007A712A4802F0F6FF0121284802F0DDFF13
:10F950004FF47A71274837F082FD4FF480712648C2
:10F9600037F07DFD10BD2DE9F04104460D462746D8
:10F9700000260DE039781E4802F032FE7F1C00BFE1
:10F9800040211B4802F09AFE0028F9D0701C86B274
:10F99000AE42EFDBBDE8F0812DE9F04105460E46B1
:10F9A0002F461648C079012804D001201449086068
:10F9B000F8F777FD40210E4802F08DFE00240DE09F
:10F9C00039780B4802F00CFE7F1C00BF402108482C
:10F9D00002F074FE0028F9D0601C84B2B442EFDB60
:10F9E000002007490860BDE8F081000030000240B7
:10F9F000004800400C10002004480020A2160020FF
:10FA0000880123420146FE48405C70470146FD489C
:10FA1000405C7047F8B5002429E0002000EB84002A
:10FA2000F9490968085C002101EB8401F74A505448
:10FA3000012000EB8400F4490968085C012101EB16
:10FA400084015054022000EB8400EF490968085CEF
:10FA5000022101EB84015054032000EB8400EA49A9
:10FA60000968085C032101EB84015054641C042CD8
:10FA7000D3D378E0002507E0601E05EB8000E34962
:10FA8000085C0DF805006D1C042DF5D304F003008F
:10FA900088BB9DF800609DF801008DF800009DF87E
:10FAA00002008DF801009DF803008DF802008DF82A
:10FAB00003609DF80000FFF7A5FF8DF800009DF89A
:10FAC0000100FFF79FFF8DF801009DF80200FFF78E
:10FAD00099FF8DF802009DF80300FFF793FF8DF862
:10FAE00003009DF80000CA4901EB940109784840E1
:10FAF0008DF8000001E0FFE700BF201F002101EBAF
:10FB00008000C249085C9DF800104840002101EBCC
:10FB10008401BE4A5054201F012101EB8000114690
:10FB2000085C9DF801104840012101EB840150540C
:10FB3000201F022101EB80001146085C9DF8021095
:10FB40004840022101EB84015054201F032101EBA6
:10FB500080001146085C9DF803104840032101EB2A
:10FB600084015054641C2C2C84D3F8BD10B502467B
:10FB7000002018E0002112E0130103EB80030B4486
:10FB8000A24CE35CA34C246804EB8004645C6340F7
:10FB9000A04C246804EB800463544B1CD9B20429A4
:10FBA000EADB431CD8B20428E4DB10BD70B50024A6
:10FBB00013E000250DE09749096801EB8501085D18
:10FBC000FFF720FF9349096801EB85010855681C80
:10FBD000C5B2042DEFDB601CC4B2042CE9DB70BDA0
:10FBE0008C49096848788B4909684979894A1268BB
:10FBF0005170884909684A7A864909684A71854975
:10FC000009684A7B834909684A72824909684873CE
:10FC10008049096888787F490968897A7D4A12682D
:10FC200091707C49096888727A49096888797949AC
:10FC300009688A7B774909688A71764909688873F7
:10FC400074490968C87873490968C97B714A1268A0
:10FC5000D17070490968CA7A6E490968CA736D49DA
:10FC60000968CA796B490968CA726A490968C87122
:10FC700070470146C80900EBC00000EB400080EA75
:10FC80004100C0B270472DE9F041002488E061488E
:10FC9000006810F824705F48006810F824005D497F
:10FCA000096801EB8401497848405A49096801EB29
:10FCB0008401897848405749096801EB8401C97873
:10FCC00080EA01055348006810F82400514909688A
:10FCD00001EB8401497880EA01063046FFF7C9FF4D
:10FCE00006464C48006810F8240086EA05014840A2
:10FCF0004849096801F824004648006800EB840080
:10FD000040784449096801EB8401897880EA01065A
:10FD10003046FFF7AEFF06463E48006800EB840021
:10FD2000407886EA050148403A49096801EB8401B8
:10FD300048703848006800EB8400807835490968CD
:10FD400001EB8401C97880EA01063046FFF791FF94
:10FD500006463048006800EB8400807886EA05019A
:10FD600048402C49096801EB8401887029480068E3
:10FD700000EB8400C07880EA07063046FFF779FF81
:10FD800006462448006800EB8400C07886EA050136
:10FD900048402049096801EB8401C870601CC4B266
:10FDA000042CFFF674AFBDE8F08130B589B00020B7
:10FDB000089059E217480168089811F82000079048
:10FDC00014480168089801EB8000407806901148BB
:10FDD0000168089801EB8000807805900D48016863
:10FDE000089801EB8000C07804900798FFF741FF66
:10FDF00004460798FFF73DFF0390FFF73AFF0BE03B
:10FE000008450508084605082C00002014150020A8
:10FE1000084705082800002044400798FFF729FFFD
:10FE20000290FFF726FF0390FFF723FF4440079857
:10FE3000FFF71FFF0190FFF71CFF0290FFF719FF6C
:10FE40000390FFF716FF0698FFF713FF0546069885
:10FE50004540FFF70EFF0390FFF70BFF0698FFF7F3
:10FE600008FF0290FFF705FF0390FFF702FF4540F0
:10FE70000698FFF7FEFE0190FFF7FBFE0290FFF7EA
:10FE8000F8FE0390FFF7F5FE6C400598FFF7F1FED2
:10FE900005980546FFF7EDFE0390FFF7EAFE4540A3
:10FEA0000598FFF7E6FE0290FFF7E3FE0390FFF7E9
:10FEB000E0FE45400598FFF7DCFE0190FFF7D9FE14
:10FEC0000290FFF7D6FE0390FFF7D3FE6C40049834
:10FED000FFF7CFFE04980546FFF7CBFE0390FFF730
:10FEE000C8FE0498FFF7C5FE0290FFF7C2FE03901C
:10FEF000FFF7BFFE45400498FFF7BBFE0190FFF7F8
:10FF0000B8FE0290FFF7B5FE0390FFF7B2FE6C401B
:10FF1000FE480168089801F820400798FFF7A9FEFD
:10FF200007980446FFF7A5FE0390FFF7A2FE079887
:10FF3000FFF79FFE0290FFF79CFE0390FFF799FEEC
:10FF400044400798FFF795FE0190FFF792FE02905C
:10FF5000FFF78FFE0390FFF78CFE0698FFF789FEF0
:10FF600005460698FFF785FE0390FFF782FE4540A1
:10FF70000698FFF77EFE0290FFF77BFE0390FFF7E7
:10FF800078FE45400698FFF774FE0190FFF771FE7A
:10FF90000290FFF76EFE0390FFF76BFE6C40059832
:10FFA000FFF767FE054605984540FFF762FE0390A0
:10FFB000FFF75FFE0598FFF75CFE0290FFF759FE22
:10FFC0000390FFF756FE45400598FFF752FE01905B
:10FFD000FFF74FFE0290FFF74CFE0390FFF749FE3C
:10FFE0006C400498FFF745FE04980546FFF741FE74
:10FFF0000390FFF73EFE45400498FFF73AFE02905B
:020000040801F1
:10000000FFF737FE0390FFF734FE45400498FFF7F3
:1000100030FE0190FFF72DFE0290FFF72AFE0390BD
:10002000FFF727FE6C40B9480168089801EB800093
:1000300044700798FFF71DFE07980446FFF719FE66
:100040000390FFF716FE44400798FFF712FE029058
:10005000FFF70FFE0390FFF70CFE44400798FFF7F1
:1000600008FE0190FFF705FE0290FFF702FE0390E5
:10007000FFF7FFFD0698FFF7FCFD06980546FFF722
:10008000F8FD0390FFF7F5FD0698FFF7F2FD0290EB
:10009000FFF7EFFD0390FFF7ECFD45400698FFF7F3
:1000A000E8FD0190FFF7E5FD0290FFF7E2FD039008
:1000B000FFF7DFFD6C400598FFF7DBFD054605986F
:1000C000FFF7D7FD0390FFF7D4FD45400598FFF7F4
:1000D000D0FD0290FFF7CDFD0390FFF7CAFD45402C
:1000E0000598FFF7C6FD0190FFF7C3FD0290FFF7EB
:1000F000C0FD0390FFF7BDFD6C400498FFF7B9FD0C
:10010000054604984540FFF7B4FD0390FFF7B1FDA5
:100110000498FFF7AEFD0290FFF7ABFD0390FFF7E9
:10012000A8FD45400498FFF7A4FD0190FFF7A1FD4D
:100130000290FFF79EFD0390FFF79BFD6C40734814
:100140000268089802EB800084700798FFF791FD21
:10015000044607984440FFF78CFD0390FFF789FDA4
:100160000798FFF786FD0290FFF783FD0390FFF7E6
:1001700080FD44400798FFF77CFD0190FFF779FD73
:100180000290FFF776FD0390FFF773FD0698FFF7E7
:1001900070FD06980546FFF76CFD0390FFF769FDBB
:1001A00045400698FFF765FD0290FFF762FD03905A
:1001B000FFF75FFD45400698FFF75BFD0190FFF7F5
:1001C00058FD0290FFF755FD0390FFF752FD6C407C
:1001D0000598FFF74EFD05980546FFF74AFD039089
:1001E000FFF747FD0598FFF744FD0290FFF741FD3B
:1001F0000390FFF73EFD45400598FFF73AFD01905B
:10020000FFF737FD0290FFF734FD0390FFF731FD54
:100210006C400498FFF72DFD05460498FFF729FD73
:100220000390FFF726FD45400498FFF722FD02905A
:10023000FFF71FFD0390FFF71CFD45400498FFF7F3
:1002400018FD0190FFF715FD0290FFF712FD0390D6
:10025000FFF70FFD6C402D480268089802EB800004
:10026000C4700898401C089008980428FFF6A2ADB6
:1002700009B030BD70B5002413E000250DE023491E
:10028000096801EB8501085DFFF7C0FB1F4909689C
:1002900001EB85010855681CC5B2042DEFDB601C1D
:1002A000C4B2042CE9DB70BD18490968487B1749C2
:1002B00009684A7A154909684A73144909684A79EC
:1002C000124909684A72114909684A780F49096850
:1002D0004A710E49096848700C49096888780B49C9
:1002E0000968897A094A1268917008490968887210
:1002F000064909688879054909688A7B03490968BC
:100300008A71024909688873004901E028000020C9
:100310000968C8783C490968C9793B4A1268D170B4
:1003200039490968CA7A38490968CA713649096879
:10033000CA7B35490968CA7233490968C87370476E
:1003400010B500240020FFF711FC01240AE0FFF79C
:100350002DFCFFF745FCFFF796FC2046FFF706FC57
:10036000601CC4B20A2CF2DBFFF720FCFFF738FC5C
:100370000A20FFF7FBFB10BD10B500240A20FFF791
:10038000F5FB09240AE0FFF78FFFFFF773FF204614
:10039000FFF7ECFBFFF709FD601EC4B2002CF2DC96
:1003A000FFF782FFFFF766FF0020FFF7DFFB10BDBE
:1003B0000246002003E00B5C1354431CD8B2102803
:1003C000F9DB704770B505460E46144629462046AF
:1003D000FFF7EEFF0C4804600C480660FFF71AFBBD
:1003E000FFF7AEFF70BD70B505460E4614462946B0
:1003F0002046FFF7DDFF0448046004480660FFF76D
:1004000009FBFFF7B9FF70BD280000202C00002079
:1004100010B54FF4A06000F0F9F810BD704700BFB0
:10042000FEE700BFFEE700BFFEE700BFFEE7704744
:1004300070477047704700000CB500200190009095
:100440005E48006840F480305C49086000BF5B484B
:10045000006800F4003000900198401C0190009862
:1004600018B90198B0F5A06FF1D15448006800F4B4
:10047000003010B10120009001E0002000900098B1
:10048000012828D14E48006840F010004C4908600F
:100490000846006820F0030008600846006808600D
:1004A00046484068454948600846406848600846F4
:1004B000406848600846406820F0030048600846ED
:1004C000406840F00100486000BF3C48406800F0D0
:1004D0000C000428F9D10CBD10B5FFF7ADFF10BD1D
:1004E00010B53648006840F00100344908600846FD
:1004F000406834490840314948600846006832493C
:1005000008402E4908600846006820F480200860F2
:100510000846406820F4FE0048604FF41F008860E1
:10052000FFF7DAFF4FF000602849086010BD10B5F2
:10053000002100200022214B5B6803F00C0121B157
:10054000042906D0082928D107E0214B214C23603B
:1005500027E0214B1F4C236023E0184B5B6803F41A
:100560007010164B5B6803F48032022303EB90405B
:1005700022B91A4B4343174C23600DE00F4B5B68C5
:1005800003F4003323B1164B4343124C236003E0C2
:10059000114B43430F4C236003E00D4B0D4C236084
:1005A00000BF00BF054B5B68C3F303130D4CE15C58
:1005B000084B1B68CB40074C236010BD0010024065
:1005C000002002400000FFF8FFFFF6FE08ED00E00B
:1005D00000127A0030000020001BB70000093D0027
:1005E000808D5B00340000200648804706480047A5
:1005F000FEE7FEE7FEE7FEE7FEE7FEE7FEE7FEE7D3
:10060000FEE7FEE7E10401083181000831490143BA
:10061000314A1160704770B5002100230F22C47861
:1006200004B32D4C246804F4E064C4F5E064210AAA
:10063000C1F10403CA40447804FA03F184781440F9
:1006400021430901254C0678A155047804F01F05C3
:100650000124AC4005786D11AD0005F1E025C5F829
:10066000004109E0047804F01F050124AC401C4D52
:100670000678761145F8264070BD1A4A0A400243B2
:10068000154B1B1F1A60704739B1134A121D1268AF
:100690000243114B1B1D1A6006E00F4A121D12681F
:1006A00082430D4B1B1D1A607047042808D14FF080
:1006B000E021096941F004014FF0E022116107E0F7
:1006C0004FF0E021096921F004014FF0E0221161AF
:1006D000704700000000FA050CED00E000E400E0C7
:1006E00080E100E080FFFF1F10B50446FA48844215
:1006F00008D10121401500F055FD0021601500F0E2
:1007000051FD17E0F548844208D10121001500F0A1
:1007100049FD0021201500F045FD0BE0F048844222
:1007200008D10121C80300F03DFD00214FF4004035
:1007300000F038FD10BD30B502460020002350689F
:10074000E84C20400D790C6844EA052420435060B1
:100750009068E54C2040D1E902542C434D7944EA9D
:10076000450420439060D06A20F470000C7C641E25
:10077000E4B2234340EA0350D06230BD002101605F
:10078000017141718160C16001210174704721B123
:10079000826842F00102826003E0826822F0010276
:1007A0008260704721B1826842F48072826003E007
:1007B000826822F480728260704710B50023CBB249
:1007C0001AB144681C43446002E044689C4344609E
:1007D00010BD816841F0080181607047014600202A
:1007E0008A6802F008020AB1012000E00020704788
:1007F000816841F0040181607047014600208A68E9
:1008000002F004020AB1012000E00020704721B18B
:10081000826842F4A002826003E0826822F4A002AF
:1008200082607047014600208A6802F480020AB1A3
:10083000012000E00020704710B50A460021002387
:10084000416821F46041531E41EA4331416010BDCB
:1008500021B1426842F40062426003E0426822F43F
:10086000006242607047F0B504460D46002000214A
:10087000092D11DDE068A5F10A0606EB46070726FB
:1008800006FA07F18843A5F10A0606EB460603FAC5
:1008900006F10843E0600CE0206905EB45070726F8
:1008A00006FA07F1884305EB450603FA06F108430B
:1008B0002061072A0FDA606B561E06EB86071F269B
:1008C00006FA07F18843561E06EB860605FA06F17E
:1008D0000843606322E00D2A0FDA206BD61F06EB77
:1008E00086071F2606FA07F18843D61F06EB860601
:1008F00005FA06F10843206310E0E06AA2F10D0654
:1009000006EB86071F2606FA07F18843A2F10D06BB
:1009100006EB860605FA06F10843E062F0BD21B158
:10092000826842F48012826003E0826822F48012BE
:10093000826070470146C86C80B2704766484C3090
:100940000068704721B1426842F48062426003E06F
:10095000426822F480624260704721B1426842F4EA
:100960008052426003E0426822F480524260704745
:100970000A460021816821F4E041114381607047FB
:1009800021B1826842F40042826003E0826822F46E
:1009900000428260704721B1826842F40212826094
:1009A00003E0826822F40212826070470146002050
:1009B0008A6802F400120AB1012000E000207047AA
:1009C000F0B504461546002000220026092911DD55
:1009D000E068A1F10A0707EB470C072707FA0CF2BA
:1009E0009043A1F10A0707EB470703FA07F2104308
:1009F000E0600CE0206901EB410C072707FA0CF2DC
:100A0000904301EB410703FA07F210432061A06B0A
:100A1000C0F30156EF1C06F1010CA7EB0C0707EB26
:100A2000870C1F2707FA0CF29043EF1C06F1010C0C
:100A3000A7EB0C0707EB870701FA07F21043A06347
:100A4000F0BD10B50A4600210023816B21F440114E
:100A5000531E41EA0351816310BD08B50023009382
:100A60000090009B0B440093009B1A6008BD08B5E2
:100A7000024600200090009201F12800009B1844DB
:100A800000900098006880B208BD0A4600214168C5
:100A9000164B1940114341607047416282627047B2
:100AA0000A460021416821F01F011143416070474F
:100AB00040B109490831096841F40001064A083289
:100AC000116007E004490831096821F40001024A75
:100AD00008321160704700000024014000280140E6
:100AE000003C0140FFFEF0FFFDF7F1FFFFFD3FFF7F
:100AF0000246002013680B400BB1012000E00020EB
:100B00007047CA430260704770B502460020002358
:100B100000240B125568CEB205EA060415681D4084
:100B200015B10CB1012000E0002070BD00220A12B6
:100B3000D34303607047000010B50446CC4884429C
:100B400008D10121042000F02DFB0021042000F039
:100B500029FB46E0C748844208D10121082000F063
:100B600021FB0021082000F01DFB3AE0C24884422E
:100B700008D10121102000F015FB0021102000F009
:100B800011FB2EE0BD48844208D10121202000F055
:100B900009FB0021202000F005FB22E0B848844238
:100BA00008D10121402000F0FDFA0021402000F092
:100BB000F9FA16E0B348844208D10121802000F000
:100BC000F1FA0021802000F0EDFA0AE0AE488442FC
:100BD00007D10121801500F0E5FA0021A01500F0F1
:100BE000E1FA10BD10B50121084600F0DBFA002142
:100BF000012000F0D7FA10BD2DE9F0410246002592
:100C00000026002000230024002791F803C00CF0E8
:100C10000F0591F803C00CF0100CBCF1000F03D0CD
:100C200091F802C04CEA050591F800C0BCF1000F34
:100C300031D0146800202BE04FF0010C0CFA00F3C7
:100C4000B1F800C00CEA03069E4220D183004FF0A9
:100C50000F0C0CFA03F7BC4305FA03FC4CEA04043E
:100C600091F803C0BCF1280F06D14FF0010C0CFA2B
:100C700000FCC2F814C00AE091F803C0BCF1480FB0
:100C800005D14FF0010C0CFA00FCC2F810C0401C5A
:100C90000828D1D31460B1F800C0BCF1FF0F34DDD7
:100CA000546800202EE000F1080C4FF0010808FA0B
:100CB0000CF3B1F800C00CEA03069E4221D1830078
:100CC0004FF00F0C0CFA03F7BC4305FA03FC4CEA97
:100CD000040491F803C0BCF1280F05D100F1080C01
:100CE00008FA0CF8C2F8148091F803C0BCF1480F60
:100CF00007D100F1080C4FF0010808FA0CF8C2F80F
:100D00001080401C0828CED35460BDE8F0814FF617
:100D1000FF710180022181700421C1707047024679
:100D2000002093680B400BB1012000E000207047C9
:100D30000146886880B2704702460020D3680B40A5
:100D40000BB1012000E0002070470146C86880B266
:100D5000704701617047416170470AB1016100E06D
:100D600041617047C16070474FF480320A4382612D
:100D70008161826182698269704702460020434B2B
:100D800018684FF68073184040EA021008433F4B42
:100D9000186070473E49C8617047F0B50A460023A5
:100DA00000240021002500F00046B6F1004F02D1DA
:100DB000364EF16901E0354E7168C0F3034583B2E8
:100DC00000F44016B6F5401F08D121F070612F4E97
:100DD000766826F070662D4F7E6012E000F4801673
:100DE000B6F5801F06D1032606FA05F4A14341F0AB
:100DF000706106E0460D360103FA06F6B14341F094
:100E0000706122B1460D360103FA06F6314300F057
:100E10000046B6F1004F02D11C4EF16101E01B4EBD
:100E20007160F0BD30B500228B071C0F0F2303FA51
:100E300004F2164B08338C1053F824309343134CB0
:100E400008348D1044F8253023468C1053F8243094
:100E50008C07240F00FA04F423430C4C08348D1043
:100E600044F8253030BD0A49DC3108607047000085
:100E700000080140000C0140001001400014014036
:100E800000180140001C014000200140000001400A
:100E900000002042DF48006840F00100DD490860A2
:100EA00008464068DC490840DA494860084600685E
:100EB000DA490840D74908600846006820F48020D5
:100EC00008600846406820F4FE0048604FF41F00A8
:100ED00088607047CF49096821F48031CD4A11609C
:100EE0001146096821F480211160B0F5803F03D0DC
:100EF000B0F5802F0ED106E0C649096841F4803173
:100F0000C44A116007E0C349096841F4A021C14AFD
:100F1000116000E000BF00BF704710B5014600221D
:100F2000002300204A11012A02D1BA4C236806E0AE
:100F3000022A02D1B74C236A01E0B64C636A01F081
:100F40001F02012494401C400CB1012000E000204D
:100F500010BD38B5002000900024002500BF3120CE
:100F6000FFF7DBFF05460098401C00900098B0F5A5
:100F7000A06F01D0002DF2D03120FFF7CEFF08B1D5
:100F8000012400E00024204638BD01460020A14A8B
:100F9000106820F0F80040EAC10010607047A049D6
:100FA00008607047024600209A4B586820F47C1075
:100FB00042EA01031843974B586070479849086606
:100FC000704701460020934A506820F00300084310
:100FD000506070478F48406800F00C007047014631
:100FE00000208C4A506820F0F000084350607047A1
:100FF00001460020874A506820F4E06008435060B2
:10100000704701460020834A506820F4605040EA4F
:10101000C1005060704729B17E4A527A02437D4B2D
:101020005A7204E07B4A527A82437A4B5A72704772
:101030007B49D8310860704701460020754A5068E6
:1010400020F440400843506070470021714A20322C
:101050001170704A82F82010012802D004280AD1A9
:1010600004E001216B4A2032117005E00521694A34
:101070002032117000E000BF00BF7047694908606E
:1010800070476449096A0143624A116270476549C1
:1010900044390860704730B5002100220024002345
:1010A0005C4D6D6805F00C0121B1042905D00829BB
:1010B00023D105E05C4D056022E05C4D05601FE03A
:1010C000544D6D6805F47012524D6D6805F480340E
:1010D000022505EB92421CB9554D554305600BE0C6
:1010E0004C4D6D6805F400351DB1524D55430560FA
:1010F00002E04E4D5543056002E04B4D056000BFD8
:1011000000BF444D6D6805F0F00109094A4D6B5C64
:101110000568DD4045603F4D6D6805F4E061090AF2
:10112000454D6B5C4568DD4085603A4D6D6805F462
:101130006051C90A404D6B5C4568DD40C560354D66
:101140006D6805F44041890B3C4D6B5CC568B5FB8F
:10115000F3F5056130BD29B12E4A526902432D4B8A
:101160005A6104E02B4A526982432A4B5A61704704
:1011700029B1284A92690243264B9A6104E0254A24
:1011800092698243234B9A61704729B1214AD269FF
:101190000243204BDA6104E01E4AD26982431D4BB0
:1011A000DA61704729B11B4AD2680243194BDA60F1
:1011B00004E0184AD2688243164BDA60704729B1BE
:1011C000144A12690243134B1A6104E0114A12696E
:1011D0008243104B1A6170471249403908607047CA
:1011E0000F49C86470470B49C87170470948406A85
:1011F00040F0807007494862704701460020054A68
:1012000092680A400AB1012000E0002070470149BD
:1012100088727047001002400000FFF8FFFFF6FEE2
:10122000000042428004424200127A00001BB700D4
:1012300000093D00808D5B00440000205400002028
:1012400010B50446FE48844208D10121C014FFF7BE
:10125000A9FF0021E014FFF7A5FFC4E0B4F1804F1F
:1012600008D101210846FFF7AAFF00210120FFF75E
:10127000A6FFB8E0F348844208D101210220FFF71D
:101280009EFF00210220FFF79AFFACE0EE48844267
:1012900008D101210420FFF792FF00210420FFF76D
:1012A0008EFFA0E0E948844208D101210820FFF721
:1012B00086FF00210820FFF782FF94E0E448844283
:1012C00008D101211020FFF77AFF00211020FFF73D
:1012D00076FF88E0DF48844208D101212020FFF713
:1012E0006EFF00212020FFF76AFF7CE0DA4884428D
:1012F00008D101214014FFF755FF00216014FFF7CA
:1013000051FF70E0D548844209D10121C804FFF79C
:1013100049FF00214FF40020FFF744FF63E0D0486D
:10132000844209D101210805FFF73CFF00214FF459
:101330008010FFF737FF56E0CA48844209D10121E7
:101340004805FFF72FFF00214FF40010FFF72AFF99
:1013500049E0C548844208D101214020FFF72FFF12
:1013600000214020FFF72BFF3DE0C048844208D118
:1013700001218020FFF723FF00218020FFF71FFFBE
:1013800031E0BB48844208D101218015FFF717FFE7
:101390000021A015FFF713FF25E0B648844209D1CC
:1013A00001210804FFF7FEFE00214FF48030FFF713
:1013B000F9FE18E0B048844209D101214804FFF742
:1013C000F1FE00214FF40030FFF7ECFE0BE0AB48DC
:1013D000844208D101218804FFF7E4FE00214FF484
:1013E0008020FFF7DFFE10BD00220288944B984258
:1013F0000ED0994B98420BD0B0F1804F08D0914B52
:10140000984205D0904B984202D0904B984204D11C
:101410004FF68F731A404B881A438D4B984207D072
:101420008C4B984204D04FF6FF431A40CB881A43A6
:1014300002808B8883850B880385814B98420BD073
:10144000854B984208D08B4B984205D08A4B9842E6
:1014500002D08A4B984201D10B7A03860123838202
:10146000704770B5002400220023058C4FF6FE76ED
:1014700035400584028C8388048B4FF68F752C4091
:10148000B51E2C400D882C43751E2A400D892A4319
:101490004D882A436A4DA8420BD06F4DA84208D010
:1014A000744DA84205D0744DA84202D0734DA84295
:1014B00013D14FF6F7752A404D892A434FF6FB7535
:1014C0002A408D882A434FF6FF652B404FF6FF5583
:1014D0002B408D892B43CD892B4383800483CD887A
:1014E0008586028470BD70B5002400220023058C1F
:1014F0004FF6EF7635400584028C8388048B48F6DE
:10150000FF752C404FF6FF452C400D884FF6FF76B7
:1015100006EA05252C434FF6DF752A400D8906EAB9
:1015200005152A434D8806EA05152A43444DA8426D
:1015300002D0494DA8421DD14FF67F752A404D89F2
:101540004FF6FF7606EA05152A434FF6BF752A4087
:101550008D8806EA05152A434FF6FF352B404FF2DA
:10156000FF752B408D8906EA85052B43CD8906EA58
:1015700085052B4383800483CD880587028470BD55
:1015800070B5002400220023058C4FF6FF6635401D
:101590000584028C8388848B4FF68F752C404FF620
:1015A000FC752C400D882C434FF6FF552A400D89C1
:1015B0004FF6FF7606EA05252A434D8806EA0525FB
:1015C0002A431F4DA84202D0234DA8421DD14FF2FD
:1015D000FF752A404D894FF6FF7606EA05252A4316
:1015E0004FF6FF352A408D8806EA05252A434EF638
:1015F000FF752B404DF6FF752B408D8906EA0515CA
:101600002B43CD8906EA05152B4383808483CD883F
:101610008587028470BD70B5002200230024058CEC
:101620004EF6FF7635400584038C8488828B48F61D
:10163000FF752A404FF6FF452A400D8820E0000044
:10164000002C01400004004000080040000C004055
:10165000001000400014004000340140004C0140E4
:10166000005001400054014000180040001C0040A0
:10167000002000400040014000440140004801407B
:101680004FF6FF7606EA05252A434DF6FF752B40F7
:101690000D8906EA05352B434D8806EA05352B43AF
:1016A000FA4DA84202D0FA4DA84208D14BF6FF7578
:1016B0002C408D894FF6FF7606EA85152C438480F1
:1016C0008283CD88A0F84050038470BD828B4FF296
:1016D000FF331A408283828B4FF6FF7303EA0123A4
:1016E0001A4382837047F0B50C461546002200214C
:1016F0000026078C4EF6FF7C07EA0C070784828BD6
:10170000018C4FF6FF7707EA043640F6FF473A4070
:101710004FF6FF7707EA05273A434FF6FF7707EAC8
:1017200003373A43D94FB8420ED0D94FB8420BD005
:10173000B0F1804F08D0D74FB84205D0D64FB8424D
:1017400002D0D64FB84206D14DF6FF77394046F465
:101750008057394305E047F6FF57394044F4805736
:10176000394382830184F0BD828B4FF6F3731A40B4
:101770008283828B0A4382837047F0B50C461546FC
:10178000002200210026078C4FF6FF6C07EA0C07A9
:101790000784828B018C4FF6FF7707EA04264FF609
:1017A0000C773A404FF6FF7707EA03172F433A4387
:1017B000B64FB8420ED0B64FB8420BD0B0F1804F02
:1017C00008D0B44FB84205D0B34FB84202D0B34F9F
:1017D000B84206D14FF6FF57394046F48077394377
:1017E00005E04FF2FF57394044F480773943828354
:1017F0000184F0BD028B4FF2FF331A400283028B4B
:101800004FF6FF7303EA01231A4302837047F0B5D2
:101810000C461546002200210026078C4FF6EF7C6F
:1018200007EA0C070784028B018C4FF6FF7707EA63
:10183000041640F6FF473A404FF6FF7707EA0337B2
:101840003A434FF6FF7707EA05273A438F4FB842EE
:101850000ED08F4FB8420BD0B0F1804F08D08D4FD3
:10186000B84205D08C4FB84202D08C4FB84206D156
:101870004FF6DF77394046F01007394305E04FF661
:101880005F77394044F01007394302830184F0BD8B
:10189000028B4FF6F3731A400283028B0A430283D2
:1018A0007047F0B50C46154600220021068C4FF615
:1018B000FE773E400684028B018C4FF60C76324058
:1018C0007E1C06EA03162E433243704EB0420ED001
:1018D0006F4EB0420BD0B0F1804F08D06D4EB04289
:1018E00005D06D4EB04202D06C4EB04206D14FF6DC
:1018F000FD76314044F00106314305E04FF6F576C0
:10190000314044F00106314302830184F0BD70B5DB
:1019100005460C465D4885420ED05D4885420BD099
:10192000B5F1804F08D05B48854205D05A488542C2
:1019300002D05A48854200D100E000BF208850B94B
:101940002389A28861882846FFF7ABFFE1882846F3
:10195000FFF79EFF25E0208804280AD12389A2886A
:1019600061882846FFF753FFE1882846FFF742FFCA
:1019700017E0208808280AD12389A2886188284690
:10198000FFF7FBFEE1882846FFF7EEFE09E023891A
:10199000A28861882846FFF7A6FEE1882846FFF75F
:1019A00095FE70BD2DE9F04105460C460026012745
:1019B000608808B9022600E00026A088012801D12D
:1019C000022700E001272088A0B92389A288618826
:1019D0002846FFF766FFE1882846FFF759FF23896D
:1019E0003A4631462846FFF712FFE1882846FFF7BE
:1019F00001FF13E02389A28861882846FFF707FFCB
:101A0000E1882846FFF7F6FE23893A463146284604
:101A1000FFF747FFE1882846FFF73AFFBDE8F0816E
:101A20000A884B881A438B881A43CB881A430B8940
:101A30001A434B891A438B891A43A0F844207047F4
:101A40004FF6FF71818000210180C18041800172C9
:101A500070470021018041808180C18001814181E6
:101A60008181C181704700210180418001218180F5
:101A70000021C18001817047002101804180818067
:101A8000C18001814181818170470000002C0140AB
:101A9000003401400004004000080040000C0040F9
:101AA00021B1028842F00102028004E002884FF670
:101AB000FE731A400280704731B1B0F8442042F4FE
:101AC0000042A0F8442005E0B0F84420C2F30E0222
:101AD000A0F8442070471AB183890B43838102E048
:101AE00083898B43838170478182704741EA020377
:101AF000A0F8483070471AB183890B43838102E014
:101B000083898B438381704701894FF6F8721140B6
:101B1000018170470A46002101894FF68F731940F1
:101B200011430181704730B504460D4629462046D1
:101B3000FFF7F0FF208940F00700208130BD2DE93C
:101B4000F04104460D4616461F46602D06D13B4621
:101B5000012231462046FFF75AFE05E03B460122AE
:101B600031462046FFF79DFE29462046FFF7D2FF6B
:101B7000208940F007002081BDE8F08130B50C4697
:101B800000210189C9B24FF6FF7505EA0325154307
:101B900025432943018130BD2DE9F04105460E461C
:101BA00017469846002443463A4631462846FFF7F2
:101BB000E5FF2C894FF6F870044044F007044FF617
:101BC0008F70044044F070042C81BDE8F081F0B5C2
:101BD00004460D4616461F463B46324629462046D9
:101BE000FFF7CCFF208940F480402081F0BD0185C3
:101BF000828270470A46002101884FF68F73194090
:101C0000114301807047F0B50C4615461E46002171
:101C1000002200230189028B038C4FF6F8773940AC
:101C200021434FF6FC473A4040F201173A434FF642
:101C3000DD773B404FF6FF7707EA06172F433B431C
:101C4000018102830384F0BD0A460021018B4FF617
:101C50008F7319401143018370470A460021018B9D
:101C600048F6FF7319404FF6FF7303EA0223194346
:101C7000018370470A460021818B4FF68F7319400C
:101C80001143818370470A460021818B48F6FF7318
:101C900019404FF6FF7303EA02231943818370470B
:101CA00021B1028842F08002028004E002884FF6EF
:101CB0007F731A400280704721B1828842F004028B
:101CC000828004E082884FF6FB731A40828070475E
:101CD00021B1828842F00802828004E082884FF6B7
:101CE000F7731A408280704721B1828842F0010266
:101CF000828004E082884FF6FE731A40828070472B
:101D00000A460021018B4FF6F773194011430183F6
:101D100070470A460021018B4FF2FF7319404FF6BE
:101D2000FF7303EA02231943018370470A46002127
:101D3000818B4FF6F77319401143818370470A4630
:101D40000021818B4FF2FF7319404FF6FF7303EAB6
:101D500002231943818370470A460021018B4FF605
:101D6000FB7319401143018370470A460021018B20
:101D70004FF6FF3319404FF6FF7303EA022319436E
:101D8000018370470A460021818B4FF6FB7319408F
:101D90001143818370470A460021818B4FF6FF3340
:101DA00019404FF6FF7303EA0223194381837047FA
:101DB0000A460021018B4FF67F73194011430183BE
:101DC00070470A460021018BC1F30E014FF6FF73E5
:101DD00003EA02231943018370470A460021818BDD
:101DE0004FF67F7319401143818370470A460021E3
:101DF000818BC1F30E014FF6FF7303EA02231943EF
:101E0000818370470A460021018C4FF6FD7319400B
:101E10001143018470470A460021018C4FF6F77385
:101E200019401143018470470A460021018C4FF686
:101E3000DF7319404FF6FF7303EA0213194301845D
:101E400070470A460021018C4FF67F7319404FF608
:101E5000FF7303EA02131943018470470A46002105
:101E6000018C4FF6FF5319404FF6FF7303EA02232C
:101E70001943018470470A460021018C4FF2FF7319
:101E800019404FF6FF7303EA022319430184704798
:101E90000A460021018C4DF6FF7319404FF6FF737F
:101EA00003EA023319430184704730B5002301244B
:101EB0008C40A3B2048C9C430484048C02FA01F588
:101EC000ADB22C43048430BD30B5002304248C40D3
:101ED000A3B2048C9C430484048C02FA01F5ADB2D5
:101EE0002C43048430BD70B50346002000241846FE
:101EF000183001258D40ACB21D8CA5431D8409B15D
:101F0000082909D100EB6100056825F0700505601E
:101F10000568154305600EE00D1FC5F34E05284406
:101F2000056825F4E045056005684FF6FF7606EA8A
:101F300002263543056070BD21B1028842F00202DD
:101F4000028004E002884FF6FD731A400280704759
:101F500021B1028842F00402028004E002884FF6B8
:101F6000FB731A400280704721B1828842F08002E0
:101F7000828004E082884FF67F731A408280704727
:101F800002884FF6F7731A40028002880A430280E3
:101F9000704782884FF68F731A40828082880A4386
:101FA0008280704702894FF6F8731A4002810289D5
:101FB0000A430281704702894FF67F731A400281FB
:101FC00002890A4302817047818470478185704786
:101FD000818670470187704781877047A0F840105D
:101FE000704702884FF6FF431A40028002880A4376
:101FF000028070470146888E70470146088F7047FF
:102000000146888F70470146B1F84000704701468D
:10201000888C70470146088D704702460020138A5D
:102020000B400BB1012000E000207047CA43028240
:10203000704730B50246002000230024158A05EAC7
:102040000103958905EA010413B10CB1012000E0F8
:10205000002030BDCA4302827047000010B504461C
:10206000BE48844208D101218014FFF79BF800216B
:10207000A014FFF797F816E0B948844208D101216F
:102080000014FFF79CF800212014FFF798F80AE0ED
:10209000B448844207D10121C013FFF790F8002112
:1020A000E013FFF78CF810BD10B50022028802F48F
:1020B00041520B884C8823438C882343CC8823438C
:1020C0000C8923434C8923438C892343CC892343A4
:1020D0001A430280838B4FF2FF74234083830B8A61
:1020E000038210BD2DE9F04F85B005460C464FF038
:1020F000000902274FF000084FF0010B0026B246FE
:10210000A88B4FF240010840A88302202884B5F82C
:102110001C90A068022801D100BF38E0A08810B947
:102120004FF0010B01E04FF0020B8D48854200D1CA
:1021300000E000BF6846FEF7AEFFDDF800A0E088D3
:10214000B0F5007F0AD14FEA1A2000EB8000400072
:10215000A168B0FBF1F0401D86B20BE04FEA4B10D6
:10216000BAFBF0F000EB80004000A168B0FBF1F09A
:10217000401D86B20A20B6FBF0F606F00108A6EB79
:102180000800C0F34F074FF6FF7000EA0828022F3F
:1021900001DBFF2F02DD02274FF00008E08840EA54
:1021A000080038432884A088A1890843618808432F
:1021B0002188084340F4006040EA0909A5F81C9012
:1021C00005B0BDE8F08F0021018041808180C18091
:1021D000018141818181C1810721018270470021F4
:1021E000018041808180C180022181600021818144
:1021F000704721B1028842F04002028004E0028868
:102200004FF6BF731A400280704721B1828B42F4AF
:102210008062828304E0828B4FF6FF331A40828310
:10222000704730B5002400230C110125A540ABB246
:102230001AB185881D43858002E085889D4385808D
:1022400030BD1AB183880B43838002E083888B43BF
:1022500083807047818170470146888970474FF6B7
:10226000FF62914204D0028842F48072028004E04E
:1022700002884FF6FF631A400280704721B18288BE
:1022800042F00402828004E082884FF6FB731A4019
:102290008280704702884FF2FF731A4002800288E2
:1022A0000A4302807047018841F4805101807047E1
:1022B00021B1028842F40052028004E002884DF607
:1022C000FF731A400280704702460020012901D0A6
:1022D000108B00E0908A70470146088A7047B1F57C
:1022E000804F04D1028842F48042028004E00288D8
:1022F0004BF6FF731A400280704702460020138994
:102300000B400BB1012000E000207047CA4302815E
:102310007047F0B50246002000240023002501F09C
:102320000F070126BE40B4B20B1101269E40B3B286
:10233000968806EA03051689264016B10DB10120DC
:1023400000E00020F0BD10B5002201F00F040123D1
:10235000A3409AB2D343038110BD00000030014076
:1023600000380040003C004010B50446FB48844261
:1023700009D101218803FEF715FF00214FF48040A9
:10238000FEF710FF32E0F648844209D101214804EB
:10239000FEF715FF00214FF40030FEF710FF25E097
:1023A000F048844209D101218804FEF708FF00218A
:1023B0004FF48020FEF703FF18E0EB48844209D178
:1023C0000121C804FEF7FBFE00214FF40020FEF7B8
:1023D000F6FE0BE0E548844208D101210805FEF72E
:1023E000EEFE00214FF48010FEF7E9FE10BD2DE94E
:1023F000F04786B005460E460024A24600BFA1461F
:102400000027B08900B100BF2F462C8A4CF6FF7020
:102410000440F08804432C82AC894EF6F31004404B
:10242000B08831890843718908430443AC81AC8A80
:102430004FF6FF400440B0890443AC8201A8FEF788
:102440002AFEC648874202D1DDF810A001E0DDF87F
:102450000CA0A88900F4004040B10AEBCA0000EBD0
:102460000A1031684900B0FBF1F807E00AEBCA0036
:1024700000EB0A1031688900B0FBF1F86420B8FB6A
:10248000F0F004012009642101FB1089A88900F4FF
:10249000004040B1322000EBC900B0FBF1F000F089
:1024A0000700044308E0322000EB09106421B0FB70
:1024B000F1F000F00F0004432C8106B0BDE8F08776
:1024C0004FF41651016000218180C18001810C21EF
:1024D000418100218181704710B502460020108A99
:1024E0004FF2FF0318400B884C8823438C8823430A
:1024F000CC8823431843108210BD00210180418005
:102500008180C180704721B1828942F4005282816A
:1025100004E082894DF6FF731A4082817047F0B55E
:102520000346002400260025002040F66A17B94221
:1025300000D100BF1846C1F3421401F01F06012765
:1025400007FA06F5012C01D10C3004E0022C01D170
:10255000103000E014301AB107682F43076002E022
:102560000768AF430760F0BD1AB1838A0B438382CB
:1025700002E0838A8B4383827047028A4FF6F073AE
:102580001A400282028A0A430282704782894FF20D
:10259000FF731A40828182890A438281704721B188
:1025A000828942F00202828104E082894FF6FD7343
:1025B0001A4082817047028A4FF6DF731A40028206
:1025C000028A0A430282704721B1028A42F48042A1
:1025D000028204E0028A4BF6FF731A4002827047BF
:1025E000C1F308028280704701468888C0F3080062
:1025F0007047818941F0010181817047028BD2B21D
:102600000283028B42EA012202837047028B02F4AA
:102610007F420283028B0A430283704721B1828A80
:1026200042F02002828204E0828A4FF6DF731A4071
:102630008282704721B1828A42F01002828204E0D5
:10264000828A4FF6EF731A408282704721B1828AE4
:1026500042F00802828204E0828A4FF6F7731A4041
:102660008282704721B1828942F40042828103E074
:102670008289C2F30E028281704721B1828A42F4BC
:102680000062828204E0828A4FF2FF731A408282E3
:102690007047828A4FF6FB731A408282828A0A430D
:1026A0008282704721B1828A42F00202828204E073
:1026B000828A4FF6FD731A408282704702460020DC
:1026C000B1F5007F00D100BF13880B400BB1012092
:1026D00000E00020704701F40072B2F5007F00D1E5
:1026E00000BFCA430280704770B502460024002331
:1026F0000025002040F66A16B14200D100BFC1F3A8
:10270000421501F01F03012606FA03F3012D02D141
:102710009689334006E0022D02D1168A334001E04B
:10272000968A33400C12012606FA04F416883440C7
:1027300013B10CB1012000E0002070BD10B50022E3
:10274000002340F66A14A14200D100BF0A120124FE
:102750009440A3B2DC43048010BD00000038014067
:102760000044004000480040004C00400050004041
:1027700001684FF6FE721140016000210160416066
:102780008160C1608D49884208D18C490839496807
:1027900041F00F01894A083A51608AE087491431B3
:1027A000884208D185490839496841F0F001834AD7
:1027B000083A51607DE081492831884208D17F493B
:1027C0000839496841F470617C4A083A516070E008
:1027D0007A493C31884208D178490839496841F43E
:1027E0007041764A083A516063E07449503188423A
:1027F00008D172490839496841F470216F4A083A92
:10280000516056E06D496431884208D16B490839FE
:10281000496841F47001694A083A516049E06749E2
:102820007831884208D165490839496841F07061BA
:10283000624A083A51603CE06149884206D1011F72
:10284000096841F00F01021F116032E05C49143148
:10285000884208D15A49091F096841F0F001584AD5
:10286000121F116025E056492831884208D1544989
:10287000091F096841F47061514A121F116018E084
:102880004F493C31884208D14D49091F096841F43C
:1028900070414B4A121F11600BE049495031884288
:1028A00007D14749091F096841F47021444A121FA2
:1028B0001160704710B50022026847F6F0739A4322
:1028C0000C6A8B6823430C6923434C6923438C694E
:1028D0002343CC6923434C6A23438C6A23431A4322
:1028E0000260CB6843600B6883604B68C36010BDB7
:1028F0000021016041608160C160016141618161CD
:10290000C161016241628162704721B1026842F097
:102910000102026004E002684FF6FE731A40026092
:1029200070471AB103680B43036002E003688B43EE
:1029300003607047416070470146486880B2704745
:1029400001460020002201F080531BB11C4B083BC4
:102950001A6802E0194B083B1A6802EA01030BB13E
:10296000012000E00020704700F0805119B11449A7
:10297000091F086002E011490839486070470146A4
:102980000020002201F080531BB10D4B083B1A6858
:1029900002E00A4B083B1A6802EA01030BB101206E
:1029A00000E00020704700F0805119B10449091F70
:1029B000086002E001490839486070470800024099
:1029C0000804024010B501210807FEF7F8FB0021BA
:1029D0004FF08050FEF7F3FB10BD2A4908627047A4
:1029E00028490861704701460020274A106820F0F6
:1029F000E0000843106070472249A031086070472A
:102A000010B502460020204B186820F00300104348
:102A100018601E4B1B6843F004031C4C2360012903
:102A200001D130BF00E020BF184B1B6823F0040326
:102A3000164C236010BD1448006840F00400124991
:102A400008600846006840F0020008600F4800680F
:102A500040F004000D49086000BF00BF30BF704760
:102A600001460020084A52680A400AB1012000E0ED
:102A7000002070470449096841EA8001024A116058
:102A80007047000000000E420070004010ED00E0B2
:102A900001460020FE4A106800F03800084310602C
:102AA0007047FB49096821F00801F94A1160114695
:102AB0000968014311607047F549096821F0100168
:102AC000F34A116011460968014311607047F148EB
:102AD000EF494860F04848607047EE48EC4948606C
:102AE000ED4848607047EA48006940F08000E849D6
:102AF00008617047E648006940F08000E4490861D9
:102B000070470420E249C96801F0010109B10120C0
:102B10000EE0DF49C96801F0040109B1022007E0B5
:102B2000DB49C96801F0100109B1032000E004206D
:102B3000704700B502460423FFF7E3FF034603E0B6
:102B4000FFF7DFFF0346521E012B01D1002AF7D108
:102B500002B90523184600BD30B5044604254FF4DC
:102B60003020FFF7E6FF0546042D17D1C84800695D
:102B700040F00200C649086108464461006940F01F
:102B8000400008614FF43020FFF7D3FF0546C048EE
:102B9000006941F6FD710840BD490861284630BD15
:102BA00010B504244FF43020FFF7C3FF0446042C73
:102BB00016D1B748006940F00400B54908610846DD
:102BC000006940F0400008614FF43020FFF7B1FF8A
:102BD0000446AF48006941F6FB710840AC49086102
:102BE000204610BD00B502460423FFF78AFF0346C6
:102BF00003E0FFF786FF0346521E012B01D1002A96
:102C0000F7D102B90523184600BD10B504244FF4CE
:102C10003020FFF7E7FF0446042C16D19C480069DA
:102C200040F004009A4908610846006940F04000FD
:102C300008614FF43020FFF7D5FF0446944800693F
:102C400041F6FB71084092490861204610BD002002
:102C50008F49C96901F0020109B1012000E000209B
:102C6000704730B5A5250424FFF7F1FF00B100251A
:102C70004FF43020FFF75DFF0446042C3AD185481D
:102C800083498860844888600846006940F02000D5
:102C900008610846006940F0400008614FF43020A8
:102CA000FFF747FF0446042C1BD17948006941F621
:102CB000DF710840764908610846006940F010005D
:102CC000086176480580E002FFF733FF0446052CD3
:102CD00010D06F48006941F6EF7108406C490861F7
:102CE00008E0052C06D06A48006941F6EF710840FB
:102CF00067490861204630BD78B506460C46042574
:102D000000200090E802FFF714FF0546042D24D1AF
:102D10005F48006940F001005D4908613480E802C5
:102D2000FFF707FF0546042D10D1B01C0090200CC2
:102D300000990880E802FFF7FCFE05465448006948
:102D400041F6FE7108405249086106E050480069AA
:102D500041F6FE7108404E490861284678BD70B5BD
:102D600004460D460426F002FFF7E3FE0646042E55
:102D700011D14748006940F00100454908612580AC
:102D8000F002FFF7D6FE06464148006941F6FE71A3
:102D900008403F490861304670BD70B505460E4693
:102DA0000424E002FFF7C5FE0446042C17D139487D
:102DB00037498860384888600846006940F010004C
:102DC00008612E80E002FFF7B4FE0446052C06D011
:102DD0002F48006941F6EF7108402D4908612046EF
:102DE00070BD2DE9F04304464FF6FF763746B046F6
:102DF000B1460425E443E6B2C4F30727C4F3074809
:102E00004FEA1469E802FFF794FE0546042D49D104
:102E100020481F498860204888600846006940F0C3
:102E200010000861FF2E06D01C4808300680E8021A
:102E3000FFF77FFE0546042D08D1FF2F06D0174867
:102E40000A300780E802FFF774FE0546042D0AD118
:102E5000B8F1FF0F07D011480C30A0F80080E8024D
:102E6000FFF767FE0546042D0AD1B9F1FF0F07D021
:102E70000A480E30A0F80090E802FFF75AFE054617
:102E8000052D0FD00248006941F6EF71084007E0B8
:102E90000020024023016745AB89EFCD00F8FF1FFA
:102EA000664908612846BDE8F08330B5054604242C
:102EB0004FF43020FFF73DFE0446042C41D160481A
:102EC0005E4988605F4888600846006940F02000DD
:102ED00008610846006940F0400008614FF4302066
:102EE000FFF727FE0446042C22D15448006941F61E
:102EF000DF710840514908610846006940F0100040
:102F000008611DB100205049088002E0A5204E490B
:102F100008804FF43020FFF70CFE0446052C10D03B
:102F20004648006941F6EF7108404449086108E0ED
:102F3000052C06D04148006941F6DF7108403F4941
:102F40000861204630BDF0B505460E4617460424FC
:102F50003B483A4988603B488860E002FFF7E9FD5A
:102F60000446042C19D13548006940F0100033495B
:102F7000086147F0F800304328433349891C088032
:102F8000E002FFF7D6FD0446052C06D02B48006969
:102F900041F6EF710840294908612046F0BD2748F5
:102FA000C069800870472548006A7047002023499F
:102FB000096801F0200109B1012000E000207047FC
:102FC00029B11E4A126902431C4B1A6104E01B4AD4
:102FD00012698243194B1A6170470146002001298A
:102FE00008D1164AD26902F001020AB1012008E0B4
:102FF000002006E0114AD2680A400AB1012000E030
:10300000002070470D49C860704704200B49C9680B
:1030100001F0010109B101200EE00849C96801F081
:10302000040109B1022007E00449C96801F0100158
:1030300009B1032000E00420704700000020024096
:1030400023016745AB89EFCD00F8FF1F00204449FD
:103050000860091D0860091D0860091D08604148D5
:103060003F4914310860704700213D498279002AA8
:103070003AD00A46126803689A430B461A600A1D42
:10308000126803689A430B1D1A60027911440A689A
:1030900003681A430A60324A0832126803689A4386
:1030A0002F4B08331A601A1D126803689A432C4B81
:1030B0000C331A604279102A0ED11A1F1268036865
:1030C0001A43274B08331A601A1D126803681A4303
:1030D000234B0C331A600DE02149427911440A68F0
:1030E00003681A430A6005E0027911440A6803681C
:1030F0009A430A6070470021016001710C214171FF
:103100000021817170471649103109680143144A42
:1031100010321160704701460020114A14321268C3
:103120000A400AB1012000E0002070470C49143128
:1031300008607047014600200022094B1B6803EA23
:103140000102074B14331B680B4013B10AB1012075
:1031500000E0002070470249143108607047000009
:1031600000040140FFFF0F000E49086070470D4941
:10317000486070470B49886070474AF6AA200949A1
:10318000086070474CF6CC4006490860704701461D
:103190000020044AD2680A400AB1012000E0002061
:1031A0007047000000300040F0B5034600201C4688
:1031B0000D4608E026782F78F61B301E00D004E07C
:1031C000641C6D1C521E002AF4D800BFF0BD70B5FF
:1031D00004460D46002305E026782E706D1C641C05
:1031E0005E1CB3B29342F7DB70BDF0B505460E46E8
:1031F000144663B929463246002005E00F7817705F
:10320000521C491C471CB8B2A042F7DB0EE0012B50
:103210000CD12F19791E3246002005E00F78177067
:10322000521C491E471CB8B2A042F7DBF0BD10B5D6
:103230000346002204E000241C705B1C541CE2B214
:103240008A42F8DB10BD10B5024600231078992899
:1032500012DC507880B1507812280DDC907858B18B
:103260009078312808DCD078232805DC107959289B
:1032700002DC5079592801DD002010BD087899281A
:1032800012DC487880B1487812280DDC887858B173
:103290008878312808DCC878232805DC0879592883
:1032A00002DC4879592801DD0020E6E710780C7827
:1032B000A04201DD002342E010780C78A0423DD10D
:1032C00050784C78A04201DD002338E050784C78EB
:1032D000A04231D190788C78A04201DD00232EE00D
:1032E00090788C78A04225D1D078CC78A04201DDAE
:1032F000002324E0D078CC78A04219D110790C7941
:10330000A04201DD00231AE010790C79A0420DD112
:1033100050794C79A04201DD002310E050794C79BE
:10332000A04201D101230AE0022308E0022306E0C3
:10333000022304E0022302E0022300E002231846F5
:103340009BE701460878992812DC487880B14878D4
:1033500012280DDC887858B18878312808DCC878C4
:10336000232805DC0879592802DC4879592801DD31
:10337000002070470120FCE7704730B50146084641
:10338000CC1701EB14742411A1EB04140A46CD17D9
:1033900001EB15752D1105EB850504EB4504E3B232
:1033A000184630BD01460A2291FBF2F302FB1313CB
:1033B00091FBF2F203EB0212D0B270472DE9FC4709
:1033C00004460D4616464FF00009002213462046DB
:1033D000294634F0C9FB03D24FF0010985F00045BE
:1033E0002046294634F057FB0190019834F0E6FA64
:1033F000074622462B4634F0DEF904460D460022ED
:10340000FE4B2046294634F0D9F904460D462046A5
:10341000294634F040FB80B20090B9F1010F03D18E
:10342000019840F000400190022231466846FFF7C3
:10343000CEFE0422B11C01A8FFF7C9FEBDE8FC873F
:103440002DE9F04104460D46164622462B463046ED
:10345000F6F7AAFA3046F6F757FA074688463A468C
:1034600043462046294634F07FFB02D10020BDE8C8
:10347000F0810120FBE770B504460D462146284641
:10348000F6F738FA2846F6F780F906463146204620
:1034900034F0B6FB01D1002070BD0120FCE770B50F
:1034A00004460D4621462846F6F7A2FA2846F6F7C6
:1034B00087FA0646A64201D1002070BD0120FCE734
:1034C00010B5F5F797FAF4F7ADFFF5F712FCF5F73D
:1034D000A2FC07F089FD10BD2DE9F04100210D206F
:1034E000F5F742F9054634F053FA0446204634F025
:1034F00028FB0546C24AC34B34F060F9074634F056
:1035000063FB0446204634F093FAC1B2BE4881758D
:103510000146887D34F03CFA0746214634F034F801
:103520000646BA4934F033F8054634F081FAB64914
:1035300048750846807DA1F817000846B0F81700C6
:1035400000EBC00101EB00104FF6FF7101EA8000B3
:10355000AD49A1F817000846B0F81700497D0844A6
:10356000A949A1F81700BDE8F08170B5FBF79AFDF5
:103570000120F4F796FFFBF72FFE0446FBF7A0FDB2
:10358000FBF754FD0120F4F78CFF0120A0490860EF
:103590004FF4FA70F4F785FF4FF400619D48FDF792
:1035A000CBFB08B9012000E0002005462A464FF475
:1035B00000619848FDF7D1FB4FF4FA70F4F771FF02
:1035C0004FF400619348FDF7B7FB08B9012000E014
:1035D000002005462A464FF400618E48FDF7BDFBEA
:1035E000FFF77AFF00208A4908604CB9012086491C
:1035F000087408204874062088700120087008E0CC
:1036000006208149C870002008740220087001203B
:10361000487400207C49887007F084FB07F0A2FB07
:103620007D480068012812D17C484078C0F3C00072
:1036300038B17B48407801280DD001207849487086
:1036400009E00020764948704870087003E00020C7
:1036500073494870087070481C380068012814D1FC
:103660006E484078C0F3001038B16D48C07801282A
:103670000FD001206A49C8700BE000206849C8706B
:103680006849487481F86F0003E000206449C870FD
:10369000887007F057FB07F074FB70BD10B529F078
:1036A00015FC07216048FCF777F90120F4F7F9FED3
:1036B00000205E490860FFF758FF10BD00205C49FC
:1036C00008704870C87088700871C87308744882A0
:1036D000888270470020574981F8680081F86900A6
:1036E00081F86B0081F86A0081F86C0081F86D0048
:1036F00081F86F0081F870000866704770472DE907
:10370000FF5F4D4908684D4933F041FF4C49C1F80E
:103710001A0049494868494933F039FF4849C1F816
:103720001E0045498868454933F031FF4449C1F8D6
:1037300022004FF47A703449A1F81F00012008706C
:10374000002040498870404A10605060002191601C
:10375000D160114681F809013C4908700120487187
:10376000002088713A4948700320114681F8A00072
:1037700001203849087048703748C088488036486A
:10378000C1883448A0F80D103348C1783148017120
:103790003148C1782F48C1731046026A416A104609
:1037A00034F012FA2B49C1F8050027498A6AC96A20
:1037B000104634F009FA2749C1F809002248026A84
:1037C000416A104634F000FA224908611E48826AB4
:1037D000C16A104634F0F8F91E4948611E48C078A5
:1037E00008761D48C1781B4880F822101A480179D4
:1037F000184841761848017916482FE00088C340E0
:10380000B6BE4868CBB9643FA21600200000C8428B
:10381000800122420008014030012342EA2D0020AD
:103820006700002090190020074805088481224283
:10383000F60F00201F190020912D002000007A446F
:10384000D91800205F1A00208E220020581D002069
:1038500070000020E31700200C00002080F82310E7
:10386000F8490A6A496A104634F0AEF9F649C1F8D7
:103870001A00F448826AC16A104634F0A5F9F24988
:10388000C1F81E00EF48026A416A104634F09CF904
:10389000ED494862EB48826AC16A104634F094F9F7
:1038A000E94988620A20E94988740020E8490872D9
:1038B000C871E849088834F06BF8E749C1F8160088
:1038C000E449488834F064F8E349C1F81A00E14952
:1038D000888834F05DF8E049C1F80E00DD49C888F9
:1038E00034F056F8DC49C1F82200DA49088934F08E
:1038F0004FF8D949C1F81200D649488934F048F840
:10390000D549C1F81E0015F0F1FF16F0BFF816F00A
:10391000EBF816F0C0F9D1490869D14933F069FED6
:10392000D049C1F842000020CF49C87116F05BFDB4
:103930000120C64981F85500FFF7E0FEDFF82CB3FF
:103940004FF0000A08E000208BF800000BF1010B9B
:103950000AF1010000F0FF0ABAF1030FF3D3BE49E8
:10396000D1F8060034F0EDF804460D46BA49D1F816
:10397000060034F0E6F80646BD4ABE4B33F01EFFA3
:1039800022462B46CDE9000133F018FF8046002285
:10399000B94B33F085FFCDE9020134F015F9AE499A
:1039A000C1F80A000020A9494872C87108720120B4
:1039B00008750020A64908714FF40061AF48FDF773
:1039C000BBF908B9012000E00020044622464FF46C
:1039D0000061AA48FDF7C1F94FF07E50A149C863C4
:1039E0000220A74908700020984981F83600A549AF
:1039F0000870FFF76FFEFFF761FE0DF096FF16F0FF
:103A000013FE2FF0A4FEBDE8FF9F10B50BF0F1FEF2
:103A100010BD10B5FFF754FD4FF400619748FDF756
:103A20008BF908B9012000E00020044622464FF43B
:103A300000619248FDF791F94FF4FA70F4F731FD07
:103A40004FF400618D48FDF777F908B9012000E0D7
:103A50000020044622464FF400618848FDF77DF9B6
:103A60004FF4FA70F4F71DFDF6F76EFB4FF40061AA
:103A70008248FDF761F908B9012000E00020044602
:103A800022464FF400617D48FDF767F915F0D0FA42
:103A90004FF400617948FDF74FF908B9012000E0C3
:103AA0000020044622464FF400617448FDF755F9A2
:103AB00015F005FD16F0D4FA29F0A3FA4FF40061D1
:103AC0006E48FDF739F908B9012000E000200446EE
:103AD00022464FF400616948FDF73FF929F0A3FE43
:103AE0004FF400616548FDF727F908B9012000E0AF
:103AF0000020044622464FF400616048FDF72DF98E
:103B00004FF400615D48FDF717F908B9012000E0A6
:103B10000020044622464FF400615848FDF71DF985
:103B2000FFF773FF4FF400615448FDF705F908B93A
:103B3000012000E00020044622464FF400614F4877
:103B4000FDF70BF9FFF7DBFD4FF400614B48FDF784
:103B5000F3F808B9012000E00020044622464FF4A3
:103B600000614648FDF7F9F8FFF798FD4FF4006152
:103B70004248FDF7E1F808B9012000E000200446C2
:103B800022464FF400613D48FDF7E7F800203E492A
:103B9000087010BD70472E4880792D49487108463D
:103BA00040793C2803DD0120C871002088717047EE
:103BB00027488079FA2804DC25488079401C24496C
:103BC000887170472DE9F04706468946154600275B
:103BD0000024A046C8212D4833F041FCC82D02D94D
:103BE0000120BDE8F087002724E04FF00008C8213D
:103BF000264833F034FC2A464946304612F045FD4B
:103C00002A464946214812F04BFD002409E0305D68
:103C10001E49095D884202D04FF0010803E0601C94
:103C200084B2AC42F3DB00BFB8F1010F00D003E077
:103C3000781C87B2032FD8DB00BFB8F1010F27D162
:103C40000120CEE78E220020E3170020A2160020DC
:103C50009D180020BA2D002098230020DB2B002087
:103C600000006145D91800207C1D0020FE000020C6
:103C70006F1283C0CA2109400000104000080140B3
:103C8000FB0000206600002006010020FE1A002034
:103C90000020A6E700B59BB000210191029103919D
:103CA0000491059106910791089109910A910020CC
:103CB0000B900C900D910E910F901090119012900E
:103CC00013911491FE48CDE9151042F2107017902F
:103CD00000201890FB481990FB481A900120FB49DE
:103CE00008700020C1F80100012240F63E51F7485B
:103CF000FFF768FF012240F63F51F448FFF762FFEB
:103D000001224FF45461F148FFF75CFF68224FF441
:103D10007F7101A812F0B9FC682240F2924101A81B
:103D200012F0B3FC68224FF4A56101A812F0ADFCBB
:103D3000042240F2BE51E548401C12F0A6FC682265
:103D400040F2D65101A812F0A0FC682240F26C614A
:103D500001A812F09AFC682240F2027101A812F048
:103D600094FC04224FF4F361D848401C12F08DFCFF
:103D700068224FF4F66101A812F087FC682240F631
:103D8000460101A812F081FC682240F6DC0101A87E
:103D900012F07BFC042240F67211CC48401C12F059
:103DA00074FC682240F68A1101A812F06EFC6822A9
:103DB0004FF4226101A812F068FC682240F6B62197
:103DC00001A812F062FC042240F64C31BF48401CAE
:103DD00012F05BFC682240F6643101A812F055FC39
:103DE000682240F6FA3101A812F04FFC68224FF425
:103DF000496101A812F049FC042240F62651B3485B
:103E0000401C12F042FCB24ADDE901109162D0621E
:103E1000DDE9031011625062DDE905019063D163B1
:103E2000DDE9071011635063DDE909019064D16495
:103E3000DDE90B0110645164DDE90D019065D16588
:103E4000DDE90F1011655065DDE911019066D1665D
:103E5000DDE91301106651668032DDE9151011604D
:103E600050609B491798C1F888001898C1F89400D1
:103E700098481999416697491A98C1F82E001BB0C5
:103E800000BD2DE9F05F81460F4690461C464FF07D
:103E9000000A4846F5F779FC05463846F5F775FC03
:103EA00006464046F5F771FC83463146284633F016
:103EB000A7FE06D15946304633F0A2FE01D1256057
:103EC00015E03146284633F09BFE04D0594628467B
:103ED00033F096FE01D1256009E05946304633F0B3
:103EE0008FFE01D1266002E025604FF0010A5046A6
:103EF000BDE8F09F2DE9F05F8246884691461D4659
:103F00004FF0000B5046F5F75BFD04464046F5F7D1
:103F100057FD06464846F5F753FD0746B44203D120
:103F2000BE4201D12C600CE0B44201D0BC4201D1B0
:103F30002C6006E0BE4201D12E6002E02C604FF002
:103F4000010B5846BDE8F09F2DE9FF4F81B08B462D
:103F50009A46002000900198F5F7D6FC04460D46DD
:103F60005846F5F7D1FC06460F460398F5F7CCFC0A
:103F70008046894632463B462046294633F0F4FDCA
:103F800009D142464B463046394633F0EDFD02D169
:103F9000CAE900451EE032463B462046294633F03A
:103FA000E3FD06D042464B462046294633F0DCFD71
:103FB00002D1CAE900450DE042464B46304639463B
:103FC00033F0D2FD02D1CAE9006703E0CAE9004537
:103FD00001200090009805B0BDE8F08F00B59FB0BB
:103FE0001CAB4FF4A56240F292414FF47F70FFF793
:103FF000ABFF012818D11CAB4FF4A56240F29241EF
:104000004FF47F70FFF7A0FF012808D1324890F8E5
:10401000500040F00100304981F8500008E0DDE92F
:104020001C01CDE9000103E0DDE91C01CDE900013F
:104030001CAB4FF4A66240F29A4140F20440FFF7F5
:1040400083FF012818D11CAB4FF4A66240F29A41BD
:1040500040F20440FFF778FF012808D11E4890F88D
:10406000500040F002001C4981F8500008E0DDE9F2
:104070001C01CDE9020103E0DDE91C01CDE90201EB
:104080001CAB4FF4A76240F2A24140F20C40FFF794
:104090005BFF012827D11CAB4FF4A76240F2A2417D
:1040A00040F20C40FFF750FF012817D10A4890F862
:1040B000500040F00400084981F8500017E000006B
:1040C000000059400000A0419A99CA42D500002042
:1040D0008E220020F6150020A2160020DDE91C012A
:1040E000CDE9040103E0DDE91C01CDE904011CABCD
:1040F0004FF4A86240F2AA4140F21440FFF724FFB7
:10410000012818D11CAB4FF4A86240F2AA4140F23A
:104110001440FFF719FF012808D1FC4890F850001F
:1041200040F00800F94981F8500008E0DDE91C0181
:10413000CDE9060103E0DDE91C01CDE906011CAB78
:104140004FF4A96240F2B24140F21C40FFF7FCFE7E
:10415000012818D11CAB4FF4A96240F2B24140F2E1
:104160001C40FFF7F1FE012808D1E84890F8500004
:1041700040F01000E54981F8500008E0DDE91C013D
:10418000CDE9080103E0DDE91C01CDE908011CAB24
:104190004FF4AA6240F2BA4140F22440FFF7D4FE45
:1041A000012818D11CAB4FF4AA6240F2BA4140F288
:1041B0002440FFF7C9FE012808D1D44890F85000E8
:1041C00040F01000D14981F8500008E0DDE91C0101
:1041D000CDE90A0103E0DDE91C01CDE90A011CABD0
:1041E0004FF4AB6240F2C24140F22C40FFF7ACFE0C
:1041F000012818D11CAB4FF4AB6240F2C24140F22F
:104200002C40FFF7A1FE012808D1C04890F85000CB
:1042100040F01000BD4981F8500008E0DDE91C01C4
:10422000CDE90C0103E0DDE91C01CDE90C011CAB7B
:104230004FF4AC6240F2CA4140F23440FFF784FED2
:10424000012818D11CAB4FF4AC6240F2CA4140F2D5
:104250003440FFF779FE012808D1AC4890F85000AF
:1042600040F01000A94981F8500008E0DDE91C0188
:10427000CDE90E0103E0DDE91C01CDE90E011CAB27
:104280004FF4AD6240F2D24140F23C40FFF75CFE99
:10429000012818D11CAB4FF4AD6240F2D24140F27C
:1042A0003C40FFF751FE012808D1984890F8500093
:1042B00040F01000954981F8500008E0DDE91C014C
:1042C000CDE9100103E0DDE91C01CDE910011CABD3
:1042D0004FF4AE6240F2DA4140F24440FFF734FE60
:1042E000012818D11CAB4FF4AE6240F2DA4140F223
:1042F0004440FFF729FE012808D1844890F8500077
:1043000040F01000814981F8500008E0DDE91C010F
:10431000CDE9120103E0DDE91C01CDE912011CAB7E
:104320004FF4AF6240F2E24140F24C40FFF70CFE26
:10433000012818D11CAB4FF4AF6240F2E24140F2C9
:104340004C40FFF701FE012808D1704890F850005A
:1043500040F020006D4981F8500008E0DDE91C01C3
:10436000CDE9140103E0DDE91C01CDE914011AAB2C
:104370004FF4B06240F2EA4140F25440FFF7BAFD18
:10438000012816D11AAB4FF4B06240F2EA4140F274
:104390005440FFF7AFFD012808D15C4890F8500069
:1043A00040F02000594981F8500004E01A98169016
:1043B00001E01A9816901BAB40F2845240F2EE4195
:1043C0004FF48B60FFF75DFD012816D11BAB40F267
:1043D000845240F2EE414FF48B60FFF752FD01280A
:1043E00008D14A4890F8500040F04000474981F811
:1043F000500004E01B98179001E01B9817901BAB2E
:104400004FF4B16240F2F24140F25C40FFF739FDF7
:10441000012816D11BAB4FF4B16240F2F24140F2D9
:104420005C40FFF72EFD012808D1384890F8500075
:1044300040F08000354981F8500004E01B98189046
:1044400001E01B9818901BAB40F28C5240F2F641F1
:104450004FF48C60FFF715FD012816D11BAB40F21D
:104460008C5240F2F6414FF48C60FFF70AFD0128B0
:1044700008D1264890F8500040F08000234981F888
:10448000500004E01B98199001E01B981990204AF5
:10449000DDE900019062D162DDE902011062516242
:1044A000DDE904109163D063DDE906101163506308
:1044B000DDE908019064D164DDE90A1011645064FB
:1044C000DDE90C109165D065DDE90E1011655065D0
:1044D000DDE910109166D066DDE9120110665166C3
:1044E0008032DDE914101160506009491698C1F856
:1044F00088001798C1F89400064818994166054944
:104500001998C1F82E001FB000BD0000A2160020AF
:104510008E220020F61500202DE9FE4F05468B4621
:1045200016461F460C9C4FF0000800200290814662
:10453000824601900090C821F74832F090FFC821D0
:10454000F64832F08CFFC821F54832F088FFC82CBD
:1045500001D800D802D90120BDE8FE8F4FF0000835
:1045600061E04FF00009CA46002001900090224609
:104570005946E94812F094F822463146E74812F0CD
:104580008FF822463946E64812F08AF82246E34977
:10459000E14832F088FF08B1012000E000208146A8
:1045A0002246DF49DC4832F07EFF08B1012000E0FE
:1045B000002082462246DA49D84832F074FF08B11A
:1045C000012000E000200190B9F1000F09D1BAF1FB
:1045D000000F06D1002322462946CF48FEF705FEEC
:1045E00024E0B9F1000F02D0BAF1000F06D1002388
:1045F00022462946C848FEF7F8FD17E0019830B971
:10460000002322462946C548FEF7EFFD0EE00023B1
:1046100022462946C048FEF7E8FD0120009008F137
:1046200001001FFA80F8B8F1030F9ADB00BF009871
:10463000012800D190E700208EE7F0B59BB0012063
:104640004FF454635A1E511E0090B648FFF764FFA2
:10465000B448007818B1B3480078052814DD01206B
:10466000B0490870012240F63E51AE48FFF7AAFA61
:10467000012240F63F51AB48FFF7A4FA01224FF464
:104680005461A848FFF79EFAA6480078062831D260
:10469000DFE800F030030C151E274FF47F7440F262
:1046A00092454FF4A56640F2BE5724E040F2D6543E
:1046B00040F26C6540F202764FF4F3671BE04FF472
:1046C000F66440F6460540F6DC0640F6721712E046
:1046D00040F68A144FF4226540F6B62640F64C3771
:1046E00009E040F6643440F6FA354FF4496640F686
:1046F000265700E000BF00BF042239468948401C0D
:1047000011F0CEFF8748D0F801008749884209D9C7
:1047100000208449C1F80100042239468148401C28
:1047200011F0B3FF682033462A462146009001A8C5
:10473000FFF7F2FE7D4ADDE901109162D062DDE90A
:10474000031011625062DDE905109163D063DDE969
:10475000071011635063DDE909019064D164DDE95C
:104760000B1011645064DDE90D019065D165DDE940
:104770000F1011655065DDE911109166D066DDE915
:104780001310116650668032DDE91510116050601B
:1047900066491798C1F888001898C1F894006448D1
:1047A0001999416662491A98C1F82E001BB0F0BDF4
:1047B00010B500215F4A116051609160D1601161B4
:1047C00051619161D1610020106250629162D162A9
:1047D000116351639163D163116451649164D16435
:1047E000116551659065D065106650669066D0661B
:1047F000106750679167D16780321160516008324D
:1048000010605060083211605160083210605060D2
:104810000832106050600832116051600832116037
:1048200051600832116051600832116051600832E5
:1048300011605160083211605160083210605060A0
:104840000832106050600832116051600832116007
:104850005160083210605060F83AC2F80011C2F896
:104860000411C2F80811C2F80C11C2F81011C2F8F4
:104870001411C2F81811C2F81C114FF490724FF4C1
:104880005C612C4811F001FF10BD10B54FF490721F
:104890004FF45C61274811F003FF10BD2DE9F0478C
:1048A000804689469246DDE908670025002406E037
:1048B000601CC4B2032C02DB681CC5B206E0424691
:1048C00030463946FEF7BCFD0128F1D000BF002478
:1048D00006E0601CC4B2032C02DB681CC5B206E013
:1048E0004A4630463946FEF7ABFD0128F1D000BFFD
:1048F000002406E0601CC4B2032C02DB681CC5B2B5
:1049000006E0524630463946FEF79AFD0128F1D0BE
:1049100000BF2846BDE8F087FE1A0020C61B002015
:104920008E1C0020D5000020809698008E2200204A
:10493000F6150020232800202DE9F0470646894679
:10494000174698460025002406E0601CC4B2032CDC
:1049500002DB681CC5B205E031464046FEF78BFD20
:104960000128F2D000BF002406E0601CC4B2032C72
:1049700002DB681CC5B205E049464046FEF77BFDF8
:104980000128F2D000BF002406E0601CC4B2032C52
:1049900002DB681CC5B205E039464046FEF76BFDF8
:1049A0000128F2D000BF2846BDE8F0872DE9F04786
:1049B00006468946174698460025002406E0601CF6
:1049C000C4B2032C02DB681CC5B205E03146404688
:1049D000FEF765FD0128F2D000BF06E0601CC4B2FE
:1049E000032C02DB681CC5B205E049464046FEF7D1
:1049F00056FD0128F2D000BF06E0601CC4B2032CB3
:104A000002DB681CC5B205E039464046FEF747FDAB
:104A10000128F2D000BF2846BDE8F0872DE9F04319
:104A20009BB04FF46168F8480078062831D2DFE87F
:104A300000F030030C151E274FF47F7440F29245AE
:104A40004FF4A56640F2BE5724E040F2D65440F23F
:104A50006C6540F202764FF4F3671BE04FF4F664A6
:104A600040F6460540F6DC0640F6721712E040F6C6
:104A70008A144FF4226540F6B62640F64C3709E01A
:104A800040F6643440F6FA354FF4496640F626574E
:104A900000E000BF00BFDD48816AC06ACDE90110B7
:104AA000DA49086A496ACDE90301D848816BC06BCD
:104AB000CDE90510D548016B406BCDE90710D3480F
:104AC000816CC06CCDE90910D049086C496CCDE906
:104AD0000B01CE48816DC06DCDE90D10CB48016D45
:104AE000406DCDE90F10C949886EC96ECDE911013D
:104AF000C649086E496ECDE91301C448803001688B
:104B00004068CDE91510C148D0F888001790BF481B
:104B1000D0F894001890BE48406E1990BC48D0F868
:104B20002E001A906822214601A8FFF74BF8682250
:104B3000294601A8FFF746F86822314601A8FFF789
:104B400041F8B148D0F80100401CAF49C1F801005C
:104B500004223946AC48401C11F097FDAA48D0F811
:104B6000010040457ED3F4F777F94FF40061A9487E
:104B7000FCF7E2F808B9012000E0002081464A462F
:104B80004FF40061A348FCF7E8F89F480078401C08
:104B90009D49087008460078052801DD012008704D
:104BA00099480078062831D2DFE800F030030C1570
:104BB0001E274FF47F7440F292454FF4A56640F2F1
:104BC000BE5724E040F2D65440F26C6540F20276C3
:104BD0004FF4F3671BE04FF4F66440F6460540F6E9
:104BE000DC0640F6721712E040F68A144FF4226594
:104BF00040F6B62640F64C3709E040F6643440F6FD
:104C0000FA354FF4496640F6265700E000BF00BF72
:104C10007E49886AC96ACDE901017C48016A406A17
:104C2000CDE903107949886BC96BCDE90501774956
:104C3000086B496BCDE907017449886CC96CCDE9F3
:104C400009017248016C406CCDE90B106F48816D11
:104C5000C06DCDE90D106D48016D406DCDE90F10AF
:104C60006A4800E048E0816EC06ECDE911106748E7
:104C7000016E406ECDE913106448803001684068D1
:104C8000CDE915106148D0F8880017905F48D0F83A
:104C9000940018905E48406E19905D48D0F82E0040
:104CA0001A906822214601A8FEF78CFF6822294647
:104CB00001A8FEF787FF6822314601A8FEF782FFB0
:104CC00001205149C1F80100042239464E48401CD8
:104CD00011F0DBFC012240F63E514B48FEF772FF1B
:104CE000012240F63F514848FEF76CFF01224FF485
:104CF00054614548FEF766FF6420F3F7D2FB1BB012
:104D0000BDE8F08338B54448407908B900240CE088
:104D100041484079012801D1012406E03E4840790C
:104D2000022801D1022400E000243B480094D0F87E
:104D3000013001780022104631F04CFB31F00FFCBD
:104D400038BD36480078012806D10420344908705F
:104D500000203249087015E032480078012803D15C
:104D600003202F4908700DE02E480078022809D151
:104D70002B48007C012802D12949087002E002205A
:104D800027490870704710B527484078042813DB7E
:104D9000254800783C280FDC2148C07918B901204B
:104DA0001F49C87105E0002011F072F800201C496D
:104DB000C87100201C4948701948C07901280AD1DF
:104DC00000201A49086001201949C1F89C010020FF
:104DD00011F0C6F805E00020144908601449C1F834
:104DE0009C0110BD10B51048407804282BDB0E48FC
:104DF00000783C2827DC15F017FC0948C079C8B9B1
:104E000001200749C8711BE0D50000208E22002038
:104E1000F615002000080140E8000020FE000020F8
:104E2000A2160020FB000020581D00208481224291
:104E300000002342012011F02BF80020FE49C87128
:104E40000020FE494870FC48C079012809D10020A3
:104E5000FB4908600120FB49C1F89C0111F080F872
:104E600008E00120F64908600020F649C1F89C01DD
:104E700028F037F8F048007B022805DB4FF461602A
:104E8000ED49A1F80D000BE0EB48B0F80D0000284B
:104E900006DDE948B0F80D00401EE749A1F80D0015
:104EA000E548007B092829DD4620E7490870602095
:104EB0004870672088708921E348C1704320E24927
:104EC00008718621E04841716820DF4988716821B6
:104ED000DD48C1715220DC4908728621DA484172EE
:104EE0007520D94988729721D748C1720C2242F2A5
:104EF000300111F0CAFB0020CF49087310BD10B576
:104F000005F010FF05F02EFFD0480068012834D1CD
:104F1000CF48007802282ADDCE484078C0F3C00090
:104F2000F8B1CB48407801282BD00120C8494870FF
:104F30000321072028F07AF9C74890F86E0002286C
:104F400002DA0120C4490874C34890F86E00FA28B8
:104F500017DAC14890F86E00401CBF4981F86E0016
:104F60000FE00020BA4948704870087009E0B8485E
:104F70000078401CB649087003E00020B44948702E
:104F80000870B2481C380068012836D1B0488078D3
:104F900002282CDDAF484078C0F30010F8B1AC48CF
:104FA000C07801282DD00120A949C870042107200C
:104FB00028F03CF9A84890F86F00022802DA012096
:104FC000A5494874A44890F86F00FA2819DAA24855
:104FD00090F86F00401CA04981F86F0011E000209C
:104FE0009B49C8709C49487481F86F0009E0984853
:104FF0008078401C9649887003E000209449C8706E
:10500000887005F09FFE05F0BCFE10BD10B5FAF7E4
:1050100049F80120F3F745FAFAF7DEF80446FAF703
:105020004FF8A4BB00208449C87008468078052842
:1050300025DD012008700846007C012824D00120CD
:10504000087484484078C0F34000E8B1022106208B
:1050500028F0ECF8804890F86000042802DA01207B
:105060007D4988707C4890F86000FA280CDA7A480C
:1050700090F86000401C784981F8600004E06E48B8
:105080008078401C6C4988706B48807833E0FFE77B
:105090000020694988700846C078052824DD022070
:1050A00008700846007C20B30020087469484078E6
:1050B000C0F34000E8B10221062028F0B7F86648A6
:1050C00090F86000042802DA022063498870624880
:1050D00090F86000FA280CDA5F4890F86000401CF5
:1050E0005D4981F8600004E05348C078401C524993
:1050F000C8705148C078FFF702FF10BD2DE9F0419C
:10510000044656498979A1F5FA61C8B2FEF74AF911
:1051100020705249C878FEF745F960704F49087908
:10512000FEF740F9A0704D490878FEF73BF9E070B2
:105130004A494878FEF736F9207148498878FEF7E1
:1051400031F96071A41C4649886AC96A6060A1602F
:105150004348016A406AE160206141488568C1684E
:105160000022404B284632F029FB074632F02CFD46
:1051700060613B480568416800223A4B284632F09E
:105180001DFB074632F020FDA0613548D0F898009D
:10519000E0613348D0F89C0020623148D0F88800A4
:1051A00060622F49803108684968A062E162A41EEC
:1051B000BDE8F0812DE9F041044628498979A1F53F
:1051C000FA61C8B2FEF7EEF820702449C878FEF7FD
:1051D000E9F8607021490879FEF7E4F8A0701F49EA
:1051E0000878FEF7DFF8E0701C494878FEF7DAF837
:1051F00020711A498878FEF7D5F860711848826ADC
:10520000C16A104632F047FCC4F806001448026A2E
:10521000416A104632F03FFCC4F80A001048826B25
:10522000C16B104632F037FCC4F80E000C48026B1C
:10523000416B104618E00000A2160020581D002007
:105240008481224200002342312C0020300123427D
:1052500067000020EA2D0020901900200C0000209B
:105260008E2200200020AC4032F015FCC4F8120061
:10527000FE480569416900221346284632F08CFC3D
:105280001AD2FA488569C1690022F94B284632F0E2
:1052900095FA074632F098FCC4F81600F348056901
:1052A00041690022F24B284632F088FA074632F074
:1052B0008BFCC4F81A0019E0EC488568C16800222C
:1052C000EC4B284632F07AFA074632F07DFCC4F8FF
:1052D0001600E648056841680022E64B284632F091
:1052E0006DFA074632F070FCC4F81A00DF48D0F8B7
:1052F0009800C4F81E00DD48D0F89C00C4F82200D5
:10530000DD48B0F817000A2190FBF1F084F8260080
:10531000D948B0F8170090FBF1F084F82700D7487F
:105320000168A1624168E16280682063BDE8F081A4
:105330002DE9F05F81464C46D1498979A1F5FA61A2
:10534000C8B2FEF72FF82070CD49C878FEF72AF8CA
:105350006070CB490879FEF725F8A070C849087835
:10536000FEF720F8E070C6494878FEF71BF8207178
:10537000C3498878FEF716F86071A41CBB48876A99
:10538000C16A0022BF4B384632F018FA054632F0A7
:10539000C0FB6060A160B548056A416A0022B94B54
:1053A000284632F00BFA074632F0B3FBE060216189
:1053B000AE48856BC16B0022B24B284632F0FEF935
:1053C000074632F0A6FB6061A161A848056B416BFE
:1053D0000022AC4B284632F0F1F9074632F099FB37
:1053E000E0612162A41EA84800780121B1EBD01F22
:1053F00053D19E480569416900221346284632F080
:10540000CBFB25D29948D0F818A0C1690022984B4F
:10541000504632F0D3F9074600229A4B32F0CEF9CB
:10542000054632F019FBC4F8260090480569416929
:1054300000228F4B284632F0C1F982460022914B60
:1054400032F0BCF9074632F007FBC4F82A0048E006
:1054500086498D68C9680022864B284632F0AEF92D
:1054600007460022874B32F0A9F9824632F0F4FA5F
:10547000C4F826007D480768416800227D4B384605
:1054800032F09CF9824600227E4B32F097F90546B5
:1054900032F0E2FAC4F82A0023E074498D68C96842
:1054A0000022744B284632F089F907460022754BDA
:1054B00032F084F9824632F0CFFAC4F826006B4904
:1054C0000D68496800226B4B284632F077F9074691
:1054D00000226C4B32F072F9824632F0BDFAC4F809
:1054E0002A006248D0F898002E3460605F48D0F8F7
:1054F0009C0020605D48D0F8B100A0605B48D0F807
:1055000088006061594980310D68496800225F4B0D
:10551000284632F053F9074632F0D6FAE0600E34EE
:10552000C4F802105449B1F8170032F047FA0746A0
:10553000574A584B32F042F9054632F0ACFAA072A5
:105540004D48407EE0724C49B1F8170032F036FA0F
:1055500007464F4A4F4B32F031F9054632F09BFA7D
:1055600020734548407E60734B4890F83000A0732C
:10557000494890F83200E073474890F834002074AE
:10558000454890F836006074434890F83800A0749D
:10559000414890F83A00E0743F4890F83C0020758C
:1055A0003D4890F83D0060753B4890F83E00A0757E
:1055B000394890F83F00E075374890F84000207671
:1055C000354890F841006076334890F84200A07664
:1055D000314890F84300E0762F4890F84400207757
:1055E0002D4890F8450060772B4890F84600A0774A
:1055F000294890F84700E07727480068206226484D
:105600004068606224488068A0622348C068E06205
:105610002148006920632048406960631E48406A51
:10562000A0631D48806AE0631B48C06A20641A4872
:10563000806C60641848C06CA0641748006DE0641A
:105640000E480088A4F850003C3C0C48418804F106
:105650008C00A4F88E100948818804F18C00A4F80D
:1056600090100648C18804F18C0017E08E220020BB
:105670000020ACC00020AC40A2160020C62D0020A7
:105680000C0000200088C340D22D002000408F4035
:105690009A9999999999B93F062E0020A4F89210E9
:1056A000FE48018904F18C00A4F89410FB4841895C
:1056B00004F18C00A4F89610BDE8F09F2DE9F041AC
:1056C000F7498979A1F5FA61C8B2FDF76BFEF54992
:1056D0000870F349C878FDF765FEF2494870F04953
:1056E0000879FDF75FFEEF498870ED490878FDF70E
:1056F00059FEEC49C870EA494878FDF753FEE9497C
:105700000871E7498878FDF74DFEE6494871E6489B
:105710000088C880E4484188E2480181E2488188E5
:10572000E0484181E048C188DE488181DE48018946
:10573000DC48C181DC484189DA480182DA48818944
:10574000D8484182D948836AC16AD64A1432184679
:10575000FDF734FED548036A416AD24A1A32184628
:10576000FDF72CFED148836BC16BCE4A2032184620
:10577000FDF724FECD48036B416BCA4A263218461A
:10578000FDF71CFECA4800780121B1EBD01F3ED1C5
:10579000C6480469416900221346204632F0FCF9EC
:1057A0001AD2C2488669C1690022C24B304632F023
:1057B00005F8044632F008FABA49C862BB490E69D6
:1057C00049690022BB4B304631F0F8FF044632F005
:1057D000FBF9B449086334E0B4498E68C968002213
:1057E000B54B304631F0EAFF044632F0EDF9AD49F1
:1057F000C862AE48066841680022AF4B304631F0BF
:10580000DDFF044632F0E0F9A649086319E0A74835
:105810008668C1680022A84B304631F0CFFF0446AD
:1058200032F0D2F99F49C862A04806684168002258
:10583000A14B304631F0C2FF044632F0C5F9994918
:1058400008639A48D0F89800964948639748D0F87A
:105850009C0088639548D0F8B100C8639748407DA4
:1058600081F840009548807D81F841009348407D53
:1058700081F842009148807D81F84300904890F87B
:10588000300081F844008E4890F8320081F84500DD
:105890008B4890F8340081F84600894890F836002B
:1058A00081F84700864890F8380081F8480084481D
:1058B00090F83A0081F84900814890F83C0081F85E
:1058C0004A007F4890F83D0081F84B007C4890F8F2
:1058D0003E0081F84C007A4890F83F0081F84D0076
:1058E000774890F8400081F84E00754890F84100E4
:1058F00081F84F00724890F8420081F850007048DB
:1059000090F8430081F851006D4890F8440081F808
:1059100052006B4890F8450081F85300684890F8B1
:10592000460081F85400664890F8470081F8550019
:1059300063480068C1F8560061484068C1F85A00E1
:105940005F488068C1F85E005D48C068C1F86200C9
:105950005B480069C1F8660059484069C1F86A00AF
:105960005748406AC1F86E005548806AC1F8720015
:105970005348C06AC1F876005148806CC1F87A007B
:105980004F48C06CC1F87E004D48006DC1F88200E0
:1059900042480088A1F88600404841884148A0F864
:1059A00088103E4881883F48A0F88A103B48C1884B
:1059B0003C48A0F88C10394801893A48A0F88E106C
:1059C000364841893748A0F89010BDE8F0812DE9AC
:1059D000F041044632498979A1F5FA61C8B2FDF770
:1059E000E1FC384908702E49C878FDF7DBFC3549E1
:1059F00048702B490879FDF7D5FC32498870284951
:105A00000878FDF7CFFC2F49C87025494878FDF785
:105A1000C9FC2C49087122498878FDF7C3FC294943
:105A200048712248856AC16A264A921D2846FDF7B8
:105A3000C5FC1E48056A416A224A0C322846FDF719
:105A4000BDFC1A498D68C96800221B4B284631F0FD
:105A5000B5FE07461B4A1832FDF7B0FC13490D6826
:105A600049680022144B284631F0A8FE0746154A23
:105A70001E32FDF7A3FC0D48D0F89800114948628A
:105A80000A48D0F89C0088620C48407D81F82C00C0
:105A90000A48807D81F82D00094815E0C62D0020B8
:105AA0000C000020531E0020DC2D00208E22002040
:105AB000D22D00200020ACC00020AC40A216002057
:105AC000062E00202B18002090F8300081F82E00C0
:105AD000FE4890F8340081F82F00FC4890F832001E
:105AE00081F83000F94890F8360081F83100F74825
:105AF00090F83C0081F83200F44890F83E0081F8BC
:105B00003300F24890F83D0081F83400EF4890F8F7
:105B10003F0081F83500ED48406AC1F83600EB4897
:105B2000806AC1F83A00E948806CC1F83E00E74855
:105B3000C06CC1F8420046222146E548FDF747FB0C
:105B4000BDE8F081F0B59BB00024002500260027B9
:105B5000E048407820B9DF48807808B9012500E0A6
:105B60000025DC48007838B9DA48407820B9D948AF
:105B7000807808B9012600E00026D648007901287F
:105B80000AD1D448007838B9D248407820B9D148F1
:105B9000807808B9012700E00027CF48008860B16D
:105BA000CC484078CC49098890FBF1F201FB120007
:105BB00018B9C848807800B90124012D06D10EA873
:105BC000FFF79CFA0EA9012013F08BFD012E06D1E0
:105BD0000EA8FFF793FA0EA9022013F082FD012F01
:105BE00006D10EA8FFF78AFA0EA9032013F079FD5B
:105BF000012C06D101A8FFF7DDFA01A9042013F05A
:105C000032FD1BB0F0BD10B5FEF708FF10BD10B59A
:105C10000024FDF7CDFFB148C079012803D0AF487B
:105C2000007A01280CD10020AC49C8710872012CFF
:105C300002D0FEF7F3FE01240020A949A1F82100BB
:105C4000A748B0F82100B0F5967F09DB012C02D0FF
:105C5000FEF7E4FE01240020A149A1F8210006E09E
:105C60009F48B0F82100401C9D49A1F8210010BDBB
:105C70002DE9F0419748407800287DD195488078FB
:105C80000028FAD19748046843689748066A416A31
:105C90002246304631F08CFD924AC03A1061516183
:105CA00002F1C800046843688F498E6AC96A2246B7
:105CB000304631F07DFD8B4AC03A9061D16102F1EE
:105CC000F000046843688848066B416B2246304602
:105CD00031F06EFD834AC03A1067516702F1F80057
:105CE000046843688048866BC16B2246304631F0B9
:105CF0005FFD7C4AC03A9067D16702F1D00004682A
:105D0000436879490E6A496A2246304631F050FDAF
:105D1000744AC03A1062516202F1D8010C684B68B3
:105D200071498E6AC96A2246304631F041FD6D4A9A
:105D3000C03A9062D1621046D0F80041D0F80431E8
:105D400069490E6B496B2246304631F031FD654A98
:105D5000403A10605160A2F18000D0F80841D0F8BC
:105D60000C3161498E6BC96B2246304631F020FD03
:105D70005C4A383A106000E04CE1516002F1580191
:105D80000C684B6858490E6A496A2246304631F021
:105D90000FFD544AC03A1064516402F1E8000468EF
:105DA00043685148866AC16A2246304631F000FD98
:105DB0004C4AC03A9064D1641046D0F81041D0F8F3
:105DC000143149490E6B496B2246304631F0F0FCE4
:105DD000444A203A10605160A2F1A001D1F8184164
:105DE000D1F81C314048866BC16B2246304631F0F9
:105DF000DFFC3C4A183A106051603B48016A406A37
:105E00001832116050603848816AC06A08321160E7
:105E100050603549086B496B283210605160324838
:105E2000816BC06B08321160506008224FF46861CA
:105E30002C4810F02AFC082240F6886129480830D6
:105E400010F023FC08224FF46B612648303010F02C
:105E50001CFC082240F6B8612248383010F015FCCE
:105E60001C48007800286ED11E48C038016A406A7C
:105E70001C4AC03A116350631146886AC96A90632C
:105E8000D16302F180010868496890321060516066
:105E9000A2F10800016840680832116050600021DA
:105EA000983A116251629162D16200208032106092
:105EB00050600832106050600B49086A496A4832E5
:105EC000106051600849886AC96A0FE0062E0020F8
:105ED0002B1800200C000020EE0000209D18002050
:105EE000A2160020E32800208E2200200832106035
:105EF0005160F848016B406BD83AC2F80011C2F803
:105F00000401F448816BC06BC2F80811C2F80C019F
:105F100008224FF46961F04810F0B7FB082240F600
:105F20009861ED48083010F0B0FB08224FF46C6126
:105F3000E948303010F0A9FB082240F6C861E64875
:105F4000383010F0A2FBE5480079012862D1E3481F
:105F5000007800285ED1E048D038016C406CDE4A01
:105F6000D03A116550651046816CC06C9165D06562
:105F700002F1A00001684068B03211605060A2F1E7
:105F80000800016840680832116050600021B83A8A
:105F9000116451649164D1640020A032106050609B
:105FA000083211605160CB48016A406A3832116092
:105FB0005060C848816AC06A083211605060C548A4
:105FC000016B406BE83AC2F81011C2F81401C148E5
:105FD000816BC06BC2F81811C2F81C0108224FF483
:105FE0006A61BD48103010F050FB082240F6A861ED
:105FF000B948183010F049FB08224FF46D61B648DB
:10600000403010F042FB082240F6D861B2484830D8
:1060100010F03BFBB148407850B9B0488078032875
:1060200006D1C0224FF45C61AB48D03810F02DFB94
:10603000BDE8F0812DE9FF478146A9490868A949D3
:1060400031F0D7FA0546494631F0DAFD31D8A64895
:10605000807AC0F3C00010B3A44890F86E00012805
:106060002BD00120A14981F86E006021052027F086
:10607000DDF89F4890F87E00022803DA01209C4951
:1060800081F820009A4890F87E00FA2815DA98489E
:1060900090F87E00401C964981F87E000DE00020BB
:1060A000924981F86E00924981F8200081F87E00C3
:1060B00003E000208D4981F86E008C4890F868005C
:1060C0008A4901EB8000C0F80090084690F868000B
:1060D000401C81F86800084690F86800142802D136
:1060E000002081F86800814890F8690014286FD179
:1060F0004FF0000A002409E07C4800EB84000168AE
:10610000504631F0ECF98246601CC4B2142CF3DB2B
:106110007849504631F06DFA7449C865704948684D
:10612000704931F066FA05467048C16D284631F075
:1061300067FD7DD200206D4981F86D00084690F81A
:106140006C000A2875DD6349D1F8D10031F0F9FC03
:1061500007460022684B31F031FB0022674BCDE946
:10616000000131F09DFB05460E466049C86D31F0D7
:10617000E8FC2A463346CDE9020131F00DFD32D26A
:106180005948807AC0F3401018B3584890F870000E
:1061900001281CD00120554981F87000622105209A
:1061A00027F044F8524890F88000022803DA0120D2
:1061B0004F4981F822004E4890F88000FA2870DAA2
:1061C0004B4890F88000401C494981F8800068E005
:1061D00060E00020454981F87000454981F82200BF
:1061E00081F880005DE00020404981F870003E4861
:1061F000807AC0F3001020B3084690F86F000128A1
:106200004FD0012081F86F006121052027F00EF8A2
:10621000374890F87F00022803DA0120344981F8DA
:106220002100334890F87F00FA283ADA304801E03C
:1062300019E010E090F87F00401C2D4981F87F00A4
:106240002FE00020294981F86F00294981F82100B9
:1062500081F87F0025E0254890F86C00401C234918
:1062600081F86C001DE00020204981F86C00084690
:1062700090F86D000A2805DD002081F8700081F893
:106280006F000EE0194890F86D00401C174981F826
:106290006D0006E0154890F86900401C134981F82C
:1062A0006900124890F86F00BDE8FF870020704732
:1062B000704710B52FF0FEFF1149087008460078AE
:1062C00038B1012030F06DF900200D49087001202F
:1062D00010BD17E08E220020F32800200C000020C3
:1062E000DB2B002000006145EA2D00201F19002053
:1062F000901900200000A0410000F43F0020AC40B5
:106300006C000020002010BD1CB5694601A82FF0CC
:1063100046FFFE4908709DF8040001280FD1084689
:10632000007848B1002030F03CF90020F7490870AF
:106330000120F749487202E00020F54948721CBD6F
:106340000020F4490870087148700120C8700020CE
:10635000C1F8050070470020EF490860EF49C1F817
:10636000AC01704770B505460C46264601203070DA
:1063700003207070281D81B22046F9F70DFB70BD17
:1063800010B50346002009E0441C145D0C54441C65
:10639000A0B2441E145D0C54441CA0B29842F3DB1E
:1063A00010BDDB48C079012800D17047D848007A79
:1063B000012801D10220F8E7D548007C012801D14D
:1063C0000320F2E7D2484079012801D10420ECE70C
:1063D000D3488078012801D10520E6E7CC488079B0
:1063E000012805D100BFCA4880790028FBD1DCE72D
:1063F0000020DAE7C648B0F86100102803D1032076
:10640000C34908707047C248B0F861005A2803D1E8
:106410000420BF490870F5E7BD48B0F861002028A6
:1064200007D1BB480078032803D10120B849087080
:10643000E8E7B7480078E5E7704700B5B548D0F819
:106440000500B0F5616F02D90220B6490870FEF769
:1064500078FCFFF7F1FF002000BD10B5F3F771FDE8
:10646000F2F747FCF2F7D7FC4FF4E130F2F732FED7
:1064700004F035FF08F047FE01200FF02DFD26F057
:1064800025FD14F0D1F809F0F7F90020A6490870AD
:1064900048709F49C871487208720846807C4874E9
:1064A000002081F8370081F8380081F8390081F840
:1064B0003E0081F845009D49087001204871002088
:1064C00088714870C87088759149A1F81D00A1F8BD
:1064D000210081F8270081F82800A1F82500A1F803
:1064E0002300052081F8290081F82A00084690F849
:1064F0002900801EA1F82500084690F82A00801E79
:10650000A1F8230008F040FB00208149A1F80D000C
:10651000C87485494871012088700020C8700871CE
:10652000834908700FF0B2FA012007F077FF78492D
:10653000B1F81F00F2F7C5FB10BD10B5F3F701FD70
:10654000F2F7D7FB00207B4908607B49C1F8BC010A
:10655000784920310860774914310860091F0860C4
:106560007149087048706A49C87148720872887227
:1065700001204874002081F8370081F8380081F844
:10658000390081F83E0081F8450068490870012013
:106590004871002088714870C8708875674981F813
:1065A00009015B4981F8280081F827003C2081F827
:1065B000290081F82A00084690F82900801EA1F8D9
:1065C0002500084690F82A00801EA1F8230008F054
:1065D000DBFA00204E4981F82C00A1F81D00A1F83B
:1065E0002100C87450494871012088700020C8708B
:1065F00008710FF04BFA08F086FD04F070FEFCF70E
:10660000BBFE00200FF068FC022007F007FF4049A6
:10661000B1F81F00F2F755FB6420F1F742FF10BDFF
:1066200038B5044640F2754084422DD040F28D408A
:10663000844202D109F020F926E040F29D408442D4
:1066400022D0801C84421FD0801C84421CD13C4834
:10665000407908B900250CE039484079012801D17A
:10666000012506E036484079022801D1022500E0E4
:10667000002533480095D0F80130017800221046FB
:106680002FF0A8FE2FF06BFF38BD704770477047A2
:106690007047704770477047704700B5FFF7F9FFC4
:1066A000FFF7F6FFFFF7F3FFFFF7EFFFFFF7EEFF50
:1066B000FFF7F0FFFFF7EFFF00BD7047002000BFBE
:1066C00006E000221F4901EB40010A80411CC8B2CC
:1066D0000728F6DB70471C4800781C490979884276
:1066E0007DD01A48007918490870002081F86000B0
:1066F00081F8610081F8620081F8630081F864002C
:1067000081F8650081F8660022E000006B0000203F
:10671000A21600205F1A0020BC0121420000234283
:1067200006010020FB00002004000020581D00206E
:106730006D0000208C012342000021428E220020A7
:10674000E80000201E1F0020901900200C000020EF
:1067500081F8670081F8680081F8690081F86A00B3
:1067600081F86B0081F86C0081F86D0081F86E0093
:1067700081F86F0081F8700081F8710081F8720073
:1067800081F8730081F8740081F8750081F8760053
:1067900081F8770081F8780081F8790081F87A0033
:1067A00081F87B0081F87C0081F87D0081F87E0013
:1067B00081F87F0081F8800081F8810081F88200F3
:1067C00081F8830081F8840081F8850081F88600D3
:1067D00081F8870081F8880081F8890000E029E0CD
:1067E00081F88A0081F88B0081F88C0081F88D0097
:1067F00081F88E0081F88F0081F8900081F8910077
:1068000081F8920081F8930081F8940081F8950056
:1068100081F8960081F8970081F8980081F8990036
:1068200081F89A0081F89C0081F89D0081F89E0013
:1068300081F89B00704710B50024FFF74CFF2BF048
:10684000CDFF012807D10124FB48807820F02000EB
:106850002030F94988702CF06EF8012807D1012406
:10686000F548807820F040004030F34988702CF0E3
:10687000F5F8012807D10124EF48807820F01000B6
:106880001030ED498870ED4890F8A100B42812D17D
:10689000EA4890F8A100401CE84981F8A100E848C6
:1068A000407800F0010000B30846007B01281CD0AE
:1068B0000120087319E0E14890F8A100FA2806DAEF
:1068C000DE4890F8A100401CDC4981F8A100DB48BB
:1068D00090F8A100012808D1D948407800F00100C3
:1068E00018B10121084626F0A1FCD448807A01287D
:1068F00022D10020D1498872D2480078C0F34010DC
:1069000038B1CD48007820F020002030CA49087006
:106910000124CD480078C0F3800068B1CA480078EF
:10692000C0F3C00020B1042163202DF0ADFF03E0CF
:10693000012163202DF0A8FFC048007B012812D15F
:10694000C048407800F0010050B1BB48407820F0CA
:106950000100401CB849487001240420BB498873D9
:106960000020B6490873B5488078012810D100206E
:10697000B2498870B3484078C0F3400050B3AE4885
:10698000407820F00200801CAB494870012426E0CA
:10699000AA488078022822D10020A8498870A948F6
:1069A0004078C0F3400038B1A348407820F002009E
:1069B000801CA14948700124A3480078C0F300104E
:1069C00040B1A1480078C0F3401020B104217020EC
:1069D0002DF05AFF03E0012170202DF055FF97485C
:1069E000007C012822D10020944908749548407801
:1069F000C0F3C00038B19048407820F0080008305B
:106A00008D49487001249048407800F0010068B139
:106A10008D484078C0F3400020B1042103202DF0C0
:106A200033FF03E0012103202DF02EFF8348407C3B
:106A3000012822D100208149487482484078C0F35F
:106A4000001038B17C48407820F0100010307A49AE
:106A5000487001247C484078C0F3800068B17A48CF
:106A60004078C0F3C00020B1042108462DF00CFF8F
:106A700003E0012104202DF007FF704890F83F004B
:106A8000012823D100206D4981F83F006D488078AE
:106A900000F0010038B16848807820F00100401C07
:106AA0006549887001246848807800F0010068B169
:106AB00065488078C0F3400020B1042170202DF09B
:106AC000E3FE03E0012170202DF0DEFE5B4890F82C
:106AD0003E0001281FD10020584981F83E00594846
:106AE000C07A00F0010018B101205349C872012496
:106AF0005548007D00F0010068B15348007DC0F3A7
:106B0000400020B1042171202DF0BEFE03E00121E0
:106B100071202DF0B9FE494890F84000012810D1AD
:106B20000020464981F8400046488078C0F3400084
:106B300038B14148807820F00200801C3E498870BE
:106B400001243E4890F83A00012810D100203B492A
:106B500081F83A003B48C078C0F3C00038B13648ED
:106B6000C07820F0080008303349C8700124334849
:106B700090F83B00012810D10020304981F83B00FB
:106B80003048C078C0F3001038B12B48C07820F0EE
